:020000040000FA
:040000006FD00400B9
:101000006F00507B000000000000000090200020D6
:10101000AA220020A9BDF9F56C23002000000000E1
:10102000000000006C230020902000200000000041
:101030000000000090200020000000009020002010
:101040000000000090200020902000209020002030
:101050009020002090200020242F00205E240020DB
:101060000000000090200020902000200424002098
:1010700090200020D22300209020002090200020EB
:101080009020002090200020902000209020002020
:101090009020002001A04111B7170040985F3AC688
:1010A000945F3247E39CE6FE3245410182800111A4
:1010B00013078008F337078093F787083EC20100C3
:1010C0000100B7170040930570052380B70413068D
:1010D00080FA2380C7040100010083C6B70493F699
:1010E000F60DA385D704238007049246F3A6068055
:1010F0000100010093760502D5CEF336078093F602
:10110000860836C4010001002380B7042380C70489
:1011100001000100B70614007D89558D88C70100C4
:1011200001000100010023800704A246F3A6068007
:101130000100010073370780137787083AC6010062
:1011400001002380B7042380C704010001000100CF
:1011500001003727004093061005A303D7802380A2
:101160000704B247F3A70780010001009307800836
:10117000F3B7078093F787083ECE01000100B71749
:101180000040130770052380E704130780FA2380CB
:10119000E7040100010003C7B70413670708A3852C
:1011A000E70423800704F247F3A70780010001004A
:1011B0000561828093760504BDC6F336078093F6F9
:1011C000860836C8010001002380B7042380C704C5
:1011D00001000100B7061400938606047D89558D31
:1011E00088C7010001000100010023800704C246F6
:1011F000F3A6068001000100733707801377870884
:101200003ACA010001002380B7042380C70401000B
:1012100001003727004093062005A303D7802380D1
:101220000704D24781B773370780137787083ACC12
:10123000010001002380B7042380C70401000100DE
:1012400098471367070C98C723800704E24719BF24
:101250000111814601468145114506CE97000000E7
:10126000E780005593078008F3B7078093F7870856
:101270003EC601000100B717004013077005238028
:10128000E704130780FA2380E7040100010003C785
:101290006704136717002383E70423800704B2471A
:1012A000F3A7078001000100F2400561828041112F
:1012B000814601468145114597000000E780404F77
:1012C00013078008F337078093F787083EC40100AF
:1012D0000100B7170040130670052380C70493066A
:1012E00080FA2380D70401000100FD552396B70240
:1012F00023800704A245F3A5058001000100733790
:101300000780137787083AC6010001002380C704CD
:101310002380D7040100010003C767041367170087
:101320002383E70423800704B247F3A70780010063
:10133000010001A0BD473305F50201007D1575FDD3
:101340008280411122C426C206C6AA8401446317C2
:101350009400B24022449244410182800504130566
:10136000803E420497000000E78000FD4180C5B741
:101370009305000273A04580824573901534924016
:101380002242B2424243D2436244F2440255925551
:101390002256B2564257D2576258F25806499649D9
:1013A000264AB64A464BD64B664CF64C065D965DD1
:1013B000265EB65E465FD65F09617300203041113C
:1013C000B7170040985F3AC6945F3247E39CE6FE49
:1013D000324541018280B71700401307000323887C
:1013E000E702854717170000232EF74273002030CD
:1013F000411122C406C637040020976000E0E78050
:10140000C0E41C408297D5BF373700408347470070
:101410009146BD8B6389D70099466394D700834773
:101420005740730020309736000083C6662C9387A0
:10143000160017360000230DF62A0347870097375A
:1014400000009387E71AB6972380E700B7E7040008
:10145000BC4F0946894517150000034565F482977E
:10146000C9B7B787004003C76700098B6309071036
:1014700003C777009306000313770703630DD708AC
:10148000173800000348586217360000130606613B
:101490000547B30606012380E60083C577001737AA
:1014A000000013072760429793F5F50F2300B7005C
:1014B00003C58700973500009385855EC295137537
:1014C000F50F2380A5000347070089451377F7032D
:1014D000630CB70C63E7E50A6306071A8545630CDE
:1014E000B7129737000083C7375C3307F60003470E
:1014F00007001377F70F19CB850793F7F70F0D4701
:101500006363F71A17370000A300F75AB787004044
:1015100009472383E700B787004083C77700E207C6
:10152000E18763DE07049737000083C7F757173753
:1015300000001307A7563E9785462300D7001737AC
:101540000000130727563E97930600032300D70099
:10155000173700001307C7543E97A146850723009D
:10156000D70093F7F70F0D476364F71417370000A0
:10157000A30CF752B787004009472383E7007300A5
:101580002030930610026300D70E930620026305F5
:10159000D70693060002E316D7F403C72702137792
:1015A000C70F13672700D5A803C767001377070481
:1015B00065CB03C7A702173800001308A82F1735FB
:1015C00000001305E526134707082385E70203C734
:1015D000A7021377370F136787002385E702814738
:1015E00013070004B305F5008C41B306F80091071A
:1015F0008CC2E399E7FEF5B503C7A70213470704BA
:101600002385E70203C7A7021377C70F13672700D5
:101610002385E702F9B503C767001377070449C3B9
:1016200003C76702173800001308881C173500002D
:101630001305C513134707082383E70203C767028F
:101640001377370F136787002383E7028147130758
:101650000004B305F5008C41B306F80091078CC275
:10166000E399E7FEBDBD03C7670213470704238361
:10167000E70203C767021377C70F136727002383A7
:10168000E70285B503C767001377070411CB03C7CB
:1016900027021377370F136787002381E70291B57D
:1016A000238006003DBD97370000A38F073EB9BDDC
:1016B00097370000A38A073E75BD230304801547B2
:1016C0002303E48001002302A480828083076480D6
:1016D000E3CE07FE23030480828083076480E3CE89
:1016E00007FE03454480828083076480E3CE07FEC3
:1016F0002302A4808280411126C44AC24EC006C67D
:101700001377F50BAD47AA892E899544630CF70032
:10171000194597000000E78080FA97000000E780F5
:1017200020FB8D444E8597000000E78040F9FD596D
:10173000FD1463983401B240A24412498249410128
:101740008280135509011375F50F97000000E7809B
:10175000E0F92209F1BF011126CC06CEB70408003A
:1017600097000000E780C0F6154597000000E7806D
:1017700000F597000000E78080F697000000E78002
:1017800000F62AC697000000E78080F43245937780
:10179000150089EB136515001375F50FF240E2444F
:1017A00005618280FD14E9F00145CDBF397126DC69
:1017B0004ADA4ED852D656D45AD25ED006DE62CE1F
:1017C00066CCB7E700E07D5783AA070022C603AACC
:1017D000470023A0E71823A2E718B7170040130714
:1017E00070052380E704130780FA2380E70483C78A
:1017F0004704930B75FFB684E20793FBFB0F854606
:10180000AA892E8B328937240040E187015763FA79
:1018100076016308D5008946130700026313D500DB
:101820000157D98F93F7F70FB71C00402382FC04B0
:1018300011472303E4801305F00F97000000E780B1
:1018400000E8094C97000000E78080E863657C159C
:10185000B7050700DA9537870700795563FEE50479
:10186000B3879500636AF704370B0800A94733EB89
:1018700065016395F90881E8814497000000E780DD
:1018800020E5268515A8DA85094597000000E78040
:10189000C0E605090345F9FFFD14050B970000009C
:1018A000E780C0E481C49377FB0FE5F79700000061
:1018B000E780A0EA69F17D55B7170040130770056E
:1018C0002380E704130780FA2380E70403C7470453
:1018D000418B2382E704F250B7E700E023A05711C1
:1018E00023A24711E25432445259C259325AA25AE1
:1018F000125B825B724CE24C21618280A547639B44
:10190000F90685691309F00FB3069900B3742B012A
:10191000B6941349F9FFB3749900856B3379690163
:10192000416B9387F9FFB3F7270199E363FC340117
:1019300093D94900C147E3E637FF3DBF0569C16957
:101940007D19D9B71305800D63886901130500025D
:101950006384790113051008CA8597000000E780A9
:10196000C0D997000000E78040DF31D54E99B3849D
:1019700034416DBFDA852D4597000000E780E0D740
:10198000CA94E30B99EE050997000000E78020D583
:10199000A30FA9FEFDB79387F9FF93F7F70F636DC8
:1019A000FC0C83C71C04130730086315F7063707C0
:1019B00008006361EB06B3079B00B706100063FBEA
:1019C000D704334BEB0089476399F9068980D549E1
:1019D000E38404EADA85094597000000E780E0D156
:1019E00011090327C9FF91472320E480030764807E
:1019F000E34E07FE23033481FD17EDFBFD14110BAD
:101A000081C49377FB0FE9FF97000000E780E0D4E3
:101A100061F155B5B717004003C75704B707080071
:101A20001377070219E3B78707007955E376FBE8D8
:101A300033079B00E3F9E7F841B58547E380F9F008
:101A4000DA852D4597000000E78020CB9389F4FFCD
:101A5000E38404E297000000E78060C893F7390050
:101A600091EB832604800327090093074900E3963E
:101A7000E6E03E89CE84D9BFB5476399F9001305E6
:101A8000900B97000000E78080C3FDB3B1471305BA
:101A9000B00AE388F9FE99476397F904B70508008F
:101AA000B365BB002D4597000000E78000C5814469
:101AB0008D4BA14997000000E78060C263967401D6
:101AC000832704802320F9008504E39534FF8327CE
:101AD000048013172B01635507002312F90069BB1B
:101AE0002322F90051BB9D47639FF90281451305ED
:101AF000B00497000000E78040C0BD4423200900E7
:101B000023220900FD5997000000E78040BD93F7AC
:101B10007400CA9703C70700FD14398D2380A700FE
:101B2000E39334FF91BBA1476397F9069700000048
:101B3000E780A0C28144630D0B008D479304C0036E
:101B40006308FB009304000563048B0193044004C5
:101B50001375C507E30295D2194597000000E78089
:101B600000B697000000E780A0B60545970000008A
:101B7000E780E0B4268597000000E78020B709459C
:101B800097000000E78080B697000000E780E0BC87
:101B9000E31405CE0DB39147639FF900130560066A
:101BA00097000000E780A0B197000000E78040B2F6
:101BB00013059009F9B5E38109CCF1547DB9BD66EF
:101BC0000147173600001306E613938606A68545DF
:101BD0008347060093F7F70F91C382800507E3F967
:101BE000E6FE97370000238FB710DDB77D1662063B
:101BF000618693178601E18763D4070001458280DF
:101C0000931726003307F500AE9718439C4363E70C
:101C1000E7007D16E37FF7FC7D55828005458280D5
:101C2000FD15E205E18513978501618793F7F50FAF
:101C300063480700FD15139725002A97584365D779
:101C4000138517006205618582803308B5021C4246
:101C500083A80600B335B502C29733B50701AE9825
:101C6000469585486367B5006394A50063E3070163
:101C700081480C43C6950CC388C21CC28280814730
:101C80001397870161876343B7008280139727000A
:101C90002A97232007008507E5B7814701479396D8
:101CA0008701E18663C5B6001335170082809396DD
:101CB0002700AA9694428507558FD5B793D75540EC
:101CC0008A07AA979C4305453315B5007D8D828010
:101CD00017F3FFDFE702A33D2A8497000000E780A7
:101CE00060F405C5931725003E940327C4FF814780
:101CF00011EB7D1516053E954205418517F3FFDF73
:101D00006700233D05838507E5B70145C5BF8147CA
:101D10001397870161876343C70082801397270069
:101D2000B386E50094422A97850714C3D5B77D167C
:101D300062066186014793178601E18763D5070034
:101D400013351700828093172600B306F500AE976F
:101D500094429C437D16B58F5D8FF1BF8A05AA958D
:101D600001476363B500828083A6C5FFF11593D751
:101D70001600D98F9CC11397F601E5B72A83014855
:101D8000014701456343D7008280B387050183A8DB
:101D90000700B30706019C43C697AA976384F8001F
:101DA00033B517010507B3080301620723A0F80044
:101DB00061871108C1BF2A8301478147014563C379
:101DC000D70082803388E50083280800330EE600C0
:101DD000032E0E003388A8403308C84163840801ED
:101DE00033B508018507B308E300E20723A0080123
:101DF000E1871107E9B717F3FFDFE702432B011172
:101E0000B286B2842E86AA850A8597000000E780F4
:101E1000C0FA2A84A6850A8597000000E78020E89A
:101E200033348000060413351500018D056117F366
:101E3000FFDF6700032A17F3FFDFE702C324411126
:101E4000AA89AE8A328BB68402C202C402C6014499
:101E5000131C8401135C8C4163499C02939B140006
:101E6000FD1B0549138CF4FFF15C33048901620406
:101E700061846340740792478E04CE9423AEF4FECF
:101E8000410117F3FFDF6700832313192400B30B0D
:101E90002B01014A93172A00D69783A50B0088438C
:101EA00078003400500097000000E78040DA050A0F
:101EB00093178A01E187F11BE35EFCFC92474E9980
:101EC00005042320F900A2473EC2B24702C63EC421
:101ED00041B7131A8901135A8A41131D240093171D
:101EE0008A01E18763CF970092470A044E941CC091
:101EF000A24705091379F90F3EC2B24702C63EC494
:101F0000ADB7B3079A0313152A0056950841780018
:101F100034005000050AEA97DA978C4397000000D6
:101F2000E780E0D26DBF0000197106C212C416C668
:101F30001AC81ECA22CC26CE2AD02ED232D436D6E9
:101F40003AD83EDA42DC46DECAC0CEC2D2C4D6C6D9
:101F5000DAC8DECAE2CCE6CEEAD0EED2F2D4F6D6C9
:101F6000FAD8FEDA971500009385458B8841E70083
:101F7000050092402242B2424243D2436244F244BC
:101F8000025592552256B2564257D2576258F258CD
:101F900006499649264AB64A464BD64B664CF64CFD
:101FA000065D965D265EB65E465FD65F096173008C
:101FB00020300000972100209381C1041751002098
:101FC0001301418417F5FFFF130505049705002051
:101FD00093854503171600201306C6FD63FAC50056
:101FE0008322050023A0550011059105E3EAC5FEF3
:101FF00017050200130545E097150020938585FB22
:10200000171600201306066563FAC5008322050033
:1020100023A0550011059105E3EAC5FE1715002020
:1020200013054563974500209385C5196377B5006F
:10203000232005001105E36DB5FEFD42739002BC3F
:102040008D4273904280B722000093828288739001
:102050000230970200209382E2FA93E232007390FA
:1020600052309752000093822299739012346FB0CD
:10207000347973002030397101436EC619A039716B
:1020800041536AC866CA62CC5ECE19A03971015349
:102090005AD056D252D44ED64AD826DA22DC06DEA0
:1020A00033016140828241114AC026C222C406C661
:1020B0008282B24D4101024D924C224CB24B410101
:1020C000024B924A224AB2494101024992442244B7
:1020D000B240410182803D432A876373C3029377F4
:1020E000F700BDEFADE5937606FF3D8ABA960CC3C7
:1020F0004CC30CC74CC74107E36BD7FE11E282808B
:10210000B306C3408A069702000096966780A60031
:102110002307B700A306B7002306B700A305B7003F
:102120002305B700A304B7002304B700A303B70037
:102130002303B700A302B7002302B700A301B7002F
:102140002301B700A300B7002300B700828093F5F6
:10215000F50F93968500D58D93960501D58D61B7C2
:10216000939627009702000096968682E78086FA6B
:102170009680C1171D8F3E96E374C3F8A5B73367E9
:10218000B500FD530D8B79E7B7877F7F9387F7F70E
:1021900010419441B372F6003363F600BE92B3E28D
:1021A00062006397720C6318D6065041D441B37233
:1021B000F6003363F600BE92B3E262006398720ADF
:1021C000631BD60410459445B372F6003363F600E2
:1021D000BE92B3E262006391720A631ED60250455A
:1021E000D445B372F6003363F600BE92B3E26200E8
:1021F000639A72086311D60210499449B372F600CB
:102200003363F600BE92B3E2620063937208510535
:10221000D105E30FD6F61317060193970601631C49
:10222000F7001357060193D706013305F74093755E
:10223000F50F91E982804183C1833305F74093759F
:10224000F50F91E182801377F70F93F7F70F3305BE
:10225000F74082800346050083C605000505850515
:102260006313D60065FA3305D640828011059105C7
:10227000E312D6FE014582802105A105E31CD6FCB0
:10228000014582803105B105E316D6FC0145828007
:102290004105C105E310D6FC01458280B717004017
:1022A00003C777051377E70FA38BE704130700F83D
:1022B000A38DE7043D47238CE70413075003A38C49
:1022C000E70403C7A7051377D70F238DE7048280A0
:1022D000B717004003C7E7020D8941111377C70FF5
:1022E000498F93068008F3B6068093F6860836C6B3
:1022F00001000100930670052380D704930680FA3D
:102300002380D704010001002387E702238007040C
:10231000B247F3A70780010001004101828041110B
:102320002A83014E930E407E130F0019930F40062F
:1023300063E56E129308001913034006B378150382
:10234000854E0D4FA14F337365020D89133515006E
:1023500063EFBE121308F6FF7946729842081358CD
:1023600008013307C70213D61700BE07329761462C
:10237000B3F6C60213068070B386C6023697A1660E
:10238000F58F42075D8FB716004083C7F60293F7BB
:102390000708A303F1000346710083C7F60293F711
:1023A0000708E394C7FE83477100B716004093F710
:1023B000F70F6388071293078008F3B7078093F736
:1023C00087083EC401000100B7170040930670055E
:1023D0002380D704930680FA2380D70401000100EC
:1023E00023AA070383C6170393E60608A388D70228
:1023F00023800704A247F3A70780010001001166AC
:10240000B71700407D16D45BC85F93854703A98E3C
:10241000F18EF5FA93068008F3B6068093F68608E7
:1024200036C601000100930670052380D704930689
:1024300080FA2380D7040100010098C103C7170365
:1024400013670704A388E70223800704B247F3A7B2
:10245000078001000100410182807D133368E3039E
:102460009308E016630E08003368F3039308D01650
:10247000630808009378330093B818009388D8163F
:1024800033081E01131E0801135E0E0155B5639338
:10249000E5030548638608000148630303002A88B2
:1024A00071087298FD15131E0801C205135E0E0116
:1024B000C18179BD13F8150063F4BF007908D5B761
:1024C00013381800E5BF83C7F60293F70708A30384
:1024D000F1000346710083C7F60293F70708E394FF
:1024E000C7FE8347710093F7F70FF1DFE9B531714C
:1024F0004AD966CB06DF22DD26DB4ED752D556D32E
:102500005AD15ECF62CD6AC96EC7AA8C02D8971025
:102510000000E78020B12A8993078008F3B707807D
:1025200093F787083EDA01000100B7170040130750
:1025300070052380E704130780FA2380E704010075
:10254000010003C7F7021377770FA387E70203C7DA
:10255000F70213678700A387E70223800704D25797
:10256000F3A7078001000100054597000000E78000
:1025700060D6130780C13347E902116A93070AE85E
:1025800093065002BD69930BA004814A014B1304CA
:102590008008930470057D1AB347F9023307D70208
:1025A0003EC0FD873ECC938709A69309803E334702
:1025B000F7023AC27D873AC4334739038549B39954
:1025C000990193D93940B306D702B30B7703B3C649
:1025D000F602B3CBFB0236C6FD8636C893D6FB4166
:1025E00036CEB7460F00938606243349D902856656
:1025F000938606FAB3969601B389E90213076055EC
:102600003309D90293060010B389E9023349D9028C
:10261000B3C9F9029316390036CA37190040FD864E
:1026200036D0930D090493D7F9413ED2F336048096
:1026300093F6860836DC01000100930770052380BD
:10264000FD00930680FA2380DD000100010083462F
:10265000390593F6860FA309D9048346390593E615
:102660001600A309D90423800D00E256F3A60680C4
:1026700001000100130C80FA116DF336048093F60B
:10268000860836DE01000100930770052380FD00F7
:1026900023808D010100010083463905216693E600
:1026A0000602A309D90483560905B3E6A601231837
:1026B000D90483560905D18E2318D90423800D002F
:1026C000F256F3A60680010001008346390593F611
:1026D00006026381061A03463905218A6DDE081851
:1026E00097100000E7800098733604801376860800
:1026F000B2C20100010023809D0023808D010100F2
:102700000100B717004003C637051376F60DA389FD
:10271000C70403C6370513660602A389C704835698
:1027200009052166B3E6A6012318D90483560905D5
:10273000D18E2318D90423800D009646F3A6068077
:10274000010001008346390593F60602638B0614E7
:1027500083463905A18AEDFE97000020E780A0930B
:10276000AA8636D497000020E780E092A256E30ABA
:10277000D5FE835609054255B3E6A6012318D904B0
:1027800097100000E780C08F83463905A18AEDDEEF
:10279000035609058346290582473376CA00B306E6
:1027A000DA0293D5F641B296B388F640E24733B8E1
:1027B000C6002E983308F840A247B3B61601330876
:1027C000D84063C70701631DF800924763FA1701F9
:1027D000C247634FF80E63950701B24763EAF80EEC
:1027E000894663E9660FF2469315180013D3F80182
:1027F0005E8613951800B365B30042D646D497C0E1
:102800000100E780A0883258050B137BFB0F63475C
:102810000001631A0838A2586387083813081500A6
:10282000B336A800B69513D6F5013298B336C80072
:10283000AE9613581800FE06B3E606017336048000
:1028400013768608B2C60100010023809D00238014
:102850008D01010001000356C902B296C206C18271
:102860002316D90223800D00B646F3A60680010088
:10287000010021B5F336048093F68608B6C0010046
:10288000010023809D0023808D010100010083460B
:10289000390593E60602A309D90423800D00864674
:1028A0000DB5F336048093F68608B6C40100010026
:1028B00023809D0023808D0101000100834639059E
:1028C00093E60602A309D90423800D00A646BDB5F0
:1028D000E30B0BF0F336048093F68608B6C80100CC
:1028E0000100930680FA23809D002380DD00010013
:1028F00001008346390593F5FC0F93F6860FA30973
:10290000D90483463905CD8EA309D90423800D004F
:10291000C646F3A6068001000100130580FA0346AF
:102920003905930639051D8A631C96297336048080
:1029300013768608B2CC01000100130680FA2380CA
:102940009D002380CD000100010003C60600137620
:10295000F60D2380C60003C6060013660602238018
:10296000C600835609051166D18E2318D9048356F3
:1029700009052166D18E2318D90423800D00E6466F
:10298000F3A6068001000100130680FA834639058C
:1029900093F606026380062683463905130C390533
:1029A000A18AFDDA081897000000E780A06BF336D3
:1029B000048093F68608B6D001000100930680FAE1
:1029C00023809D002380DD000100010083460C0070
:1029D000116693F6F60D2300DC0083460C0093E6A7
:1029E00006022300DC0083560905D18E2318D90482
:1029F000835609052166D18E2318D90423800D0042
:102A00008656F3A6068001000100130680FA83466D
:102A1000390593F60602638A062083463905A18AA2
:102A2000EDFE97F0FF1FE78000672A8C97F0FF1FED
:102A3000E7806066E30C85FF835609051166425501
:102A4000D18E2318D90497000000E7806063834685
:102A5000390513063905A18AFDDAF336048093F6A9
:102A60008608B6D401000100930680FA23809D00F9
:102A70002380DD00010001008346060093F6F60D79
:102A80002300D60023800D00A656F3A60680010081
:102A900001008356090503462905D247B376DA00BB
:102AA0003306CA021305800C9355F6413696330D52
:102AB000F6408257333CD6002E9C3336A601330CA9
:102AC000FC40330CCC403308850392564E86B33518
:102AD000A5033305A503C29597B00100E780005B0D
:102AE00063468001631E0C16630C0D161306150059
:102AF0003335A6002E959356F5013696B335D6009C
:102B0000AA959396F50105828585D18E6346B0001E
:102B1000639D051A638B061A0356C9021582330595
:102B2000D6003336C500B2956348B00063910524E2
:102B30001306F00F637DA622894663F356159307AB
:102B40008008F3B7078093F78708BED6010001001D
:102B500037170040930770052300F704930780FAA6
:102B60002300F704010001008356C702896781171B
:102B7000D58FC207C1832316F70223000704B65777
:102B8000F3A7078001000100FA506A54DA544A5949
:102B9000BA592A5A9A5A0A5BFA4B6A4CDA4C4A4D8D
:102BA000BA4D296182801308F5FF3335A800FD1561
:102BB0002E951356F5013298B336C800AA9695B9EA
:102BC000F336048093F68608B6CA0100010023801C
:102BD0009D002380AD000100010083463905CD8EA4
:102BE000A309D90423800D00D646F3A60680010070
:102BF000010035B3F336048093F68608B6CE0100A3
:102C0000010023809D002380CD0001000100834648
:102C1000390593E60602A309D90423800D00F64680
:102C2000F3A606800100010095B3F336048093F605
:102C30008608B6D20100010023809D002380CD00CC
:102C4000010001008346390593E60602A309D90471
:102C500023800D009656F3A606800100010045BBB7
:102C60009306F5FF33B5A600FD152E959355F50196
:102C7000AE96B3B5B600AA951396F501858269B5EF
:102C8000F336048093F68608B6D801000100930657
:102C900080FA23809D002380DD000100010083561F
:102CA000C9020566011693F6F60FD18EC206C182DF
:102CB0002316D90223800D00C656F3A60680010014
:102CC0000100850A93FAFA0F95B233E6B60045C2C1
:102CD0000356C9023305D0403338A000B305B040D5
:102CE000B385054115826345B000D1E16371A60843
:102CF000894663F0560593078008F3B7078093F77A
:102D00008708BEDA01000100B717004013077005FD
:102D10002380E704130780FA2380E7040100010001
:102D200003D7C7027D8B2396E70223800704D6577B
:102D300081BDF336048093F68608B6DC01000100FD
:102D4000930680FA23809D002380DD0001000100AE
:102D50008356C9020566011693F6F60FD18EC20698
:102D6000C1822316D90223800D00E656B9B7930716
:102D70008008F3B7078093F78708BEDE01000100E3
:102D800037170040930770052300F704930780FA74
:102D90002300F704010001000356C7029397560071
:102DA000B297C207C1832316F70223000704F65720
:102DB000C1BB914763EEB70217D70100130787180D
:102DC0008A05BA959C41BA978287B717004003A736
:102DD000470B1345F5FF698F23AAE70A03A7070BE3
:102DE000698F23A8E70A03A7070A798D23A0A70AFA
:102DF0008280B717004083A6470B1347F5FFF98E73
:102E000023AAD70A83A6070B558D23A8A70A83A652
:102E1000070A758F23A0E70A8280B717004003A72F
:102E2000470B498F23AAE70A03A7070B1345F5FFB2
:102E300045BFB717004083A6470B1347F5FF758FB3
:102E400023AAE70A03A7070A598D4DB7B717004011
:102E500003A7470B498FEDB7914763EEB70217D72A
:102E600001001307670F8A05BA959C41BA978287BC
:102E7000B717004003A7470D1345F5FF698F23AA35
:102E8000E70C03A7070D698F23A8E70C03A7070C1E
:102E9000798D23A0A70C8280B717004083A6470D29
:102EA0001347F5FFF98E23AAD70C83A6070D558D7E
:102EB00023A8A70C83A6070C758F23A0E70C82809C
:102EC000B717004003A7470D498F23AAE70C03A7B4
:102ED000070D1345F5FF45BFB717004083A6470D03
:102EE0001347F5FF758F23AAE70C03A7070C598D2D
:102EF0004DB7B717004003A7470D498FEDB779715C
:102F000022D43714004026D24AD0035924028354D5
:102F1000040206D64209C2044ECE52CC56CA1359F8
:102F20000901C1802DE11379F9F793F4F49F420967
:102F3000C20413590901C18093078008F3B70780C1
:102F400093F787083EC40100010093077005230032
:102F5000F404930780FA2300F40401000100231114
:102F600024032310940223000404A247F3A707803C
:102F700001000100B250225492540259F249624AAF
:102F8000D24A45618280B7F5070081463000B1051D
:102F9000194597000020E7806081A2471397270119
:102FA000E34A07FC1369090893E404409309800885
:102FB000F3B7098093F787083EC001000100930A28
:102FC000700523005405130A80FA2300440501000C
:102FD00001002311240323109402230004048247D8
:102FE000F3A7078001000100294597F0FF1FE78044
:102FF0006034F3B9098093F989084EC201000100D9
:1030000023005405230044050100010083570402F6
:1030100093E707202310F402230004049247B9B772
:10302000B71700408847420541819377050491EB2B
:103030009377F5013755E801130505803345F5020F
:1030400082809377050C130700046397E70093775A
:10305000F50137459C1CCDB72165130505D082804D
:1030600037E700E01C435443A183E206D58F1CC11F
:10307000FD572320F7182322F718828013178500A5
:10308000B7E700E023A0E710618123A2A7108280A8
:10309000B7F700E08847CC47828081473737004048
:1030A000A14663C4C700328582800345B740E38EE2
:1030B000A6FE3385F5000345050085072304A740D8
:1030C000CDB7970700209387E7EE9C431737002082
:1030D0001307470F3E95636EE5001737002013076F
:1030E00067526368A700170700202325A7EC3E85D9
:1030F0008280FD57EDBF8280411122C406C62A841A
:1031000097000000E78000F22947B307E502B240CC
:103110008D83B3D7870222449507B3D7E7023737A9
:103120000040C207C1832316F70041018280378522
:10313000030041111305054006C697000000E78013
:10314000E0FBB7370040130770F82381E7000D4715
:10315000A381E70013070004A380E7000547238746
:10316000E700B240410182803737004083472700A3
:103170001A0593F7F703C98F93F7F70F2301F700A9
:103180008280B737004003C7170019C9D98DA380C3
:10319000B70003C70700136787002380E70082801A
:1031A00093C5F5FFF98DA380B7008280AE872A878B
:1031B000B736004021463738004089E71703000042
:1031C0006700A3F383C8B600E30916FF0507834829
:1031D000F7FFFD17C20723041801C183F9BF41118E
:1031E00022C406C62A8497000000E780A0E329478E
:1031F000B307E502B2408D83B3D787022244950717
:10320000B3D7E70237370040C207C1832316F74020
:1032100041018280716541111305052006C69700A2
:103220000000E78000FCB7370040130770F82381E7
:10323000E7400D47A381E74013070004A380E74060
:1032400005472387E740B24041018280CC414111CC
:1032500006C6328503C6150083C5050022064D8EBD
:1032600042068D654186138875A2630C0611634B77
:10327000C804138845A26300060D634AC8009385FD
:1032800035A26301B6082390060029464DA0138895
:1032900055A26305060D938565A2E316B6FE8D451E
:1032A0001D4663E6E5081146198E63F3C7003E86A6
:1032B000B7E704002390C600FC4797D5010093852B
:1032C000E5CB9DA0138895A263030611634E060DFE
:1032D0001388A5A263000613938505A5E315B6FA26
:1032E00099451D4663E5E504198E63F3C7003E86E4
:1032F000B7E704002390C600FC479705002093859C
:10330000A5D51DA09D451D4663E3E5022146198E06
:1033100063F3C7003E86B7E70400FC472390C6006E
:103320009705002093858533BA9582970146B24070
:10333000328541018280AD451D46E3EAE5FE314616
:10334000198E63F3C7003E86B7E704002390C600DA
:10335000FC4797D501009385E5C4F9B7B1451D46F3
:10336000E3E7E5FC3546198E63F3C7003E86B7E711
:1033700004002390C600FC4797D50100938585C3C0
:1033800065B78D451D46E3E4E5FA1146198E63F3F2
:10339000C7003E86B7E704002390C600FC4797D5D8
:1033A0000100938565BE49B78D451D46E3E1E5F80B
:1033B0001146198E63F3C7003E86B7E704002390D9
:1033C000C600FC4797D50100938585C0B1BFA545D0
:1033D0001D46E3EEE5F42946198E63F3C7003E86E9
:1033E000B7E704002390C600FC4797D501009385FA
:1033F00065BA1DBFB5451D46E3EBE5F23946198EAA
:1034000063F3C7003E86B7E704002390C600FC477D
:1034100097D50100938585B501BFB7E7040003A3E5
:10342000071397060020938626C24146A545170537
:103430000020130565B80283797126D252CCAE8480
:103440002A8A97D501009385A5BA17D501001305DF
:10345000A5BC06D63AC622D44AD0368432894ECE8E
:1034600056CA97B00100E780A00DA28517D50100CC
:10347000130585BB97B00100E780800C294597B004
:103480000100E780C01083C7840093F70702E5E3DB
:1034900083C904008947054532476397F908D4403A
:1034A00083C7160083C60600A207D58FC1661386A0
:1034B00016FE638DC7028D166381D7088D669386CD
:1034C000269029456392D706B7E70400A2862254C6
:1034D00003A34714B250F249D24A4A86A68502593C
:1034E00092545285624A8547456102832D450DEF0E
:1034F00093070002354563E98702B7E70400FC47FC
:10350000C84413060002CA858297814997070020A4
:103510009387C72F9C43014581CB9C4391C74E8520
:103520002286CA8582970145B2502254925402598C
:10353000F249624AD24A456182802D4575F7130AE5
:10354000700F3545E3628AFEB7EA040083A7CA0418
:10355000C8442286CA858297E30A44FBC84483A7ED
:103560008A0433068A4081452295829745B72145D2
:1035700065BF2D455DE703C505000947631FE508E5
:1035800003A84500411106C60347180032850346CB
:10359000080022074168518F930828FE630717052A
:1035A00063E9E80005186303070323900600294533
:1035B00091A8130648FE630AC7041518E31707FF0E
:1035C00015463E87637BF600154701A813060002E7
:1035D0003E876374F60013070002B7E704002390E8
:1035E000E600FC471316070111A83E8691C3054665
:1035F000B7E70400FC472390C6004206CC45418251
:1036000082970145B24041018280130600083E873F
:10361000E375F6FC13070008C9B7239006000545BB
:1036200082808280416779176304E504411122C4D6
:1036300006C685472A84639FF500B7E70400228504
:103640002244B24003A38713970500209385451BAE
:103650004101028389476399F500B7E7040083A716
:10366000070B8545829771D9B2402244410182807F
:103670008280411122C437E404008327841326C2C8
:10368000AA84416506C697050020938565177D15B8
:1036900082978327C40A170500001305E5F885887B
:1036A000829795C0032304132244B24092449706A4
:1036B00000209386E6AB4146C5451705002013055B
:1036C000259A41010283B2402244924401454101BE
:1036D000828019C59707002023AAA712014582807E
:1036E000454582801147636AA70A97D601009386F1
:1036F000E68E0A0536951841411106C63697AE8703
:10370000B2850287130700026145639DE700B7E7B2
:103710000400FC471306000217050020130585F47A
:1037200082970145B2404101828005476145E39B94
:10373000E7FEB7E70400FC47054617050020130520
:1037400065F4F9BF1307700F6145E39DE7FCB7E728
:103750000400FC471306700F170500201305C5F27F
:10376000C1B7130700086145E39EE7FAB7E7040015
:10377000FC471306000817050020130565004DB728
:1037800015476145E390E7FAB7E70400FC471546A3
:10379000170500201305050761B70945828041110F
:1037A00026C2B7E4040083A7C41322C44AC006C6D5
:1037B0002E84970500209385A5042A898297058980
:1037C00005C5970700209387A78983D7A70BA285F4
:1037D00003A3440D2310F4002244B24092444A85CE
:1037E0000249014641010283B24022449244024907
:1037F00049454101828097070020238B07009707E6
:10380000002023A90700B717004003A7070CB7063D
:10381000C0FFFD16758F23A0E70C03A7070DB706A1
:103820004000558F23A8E70C03A7070C3D9B23A05E
:10383000E70C03A7070D1367070123A8E70C828095
:10384000B717004003A5470C83A7470C59811345C0
:103850001500C18B058999E31365250097070020A2
:1038600083C707FB6380A702970700202382A7FA7C
:1038700011C9970700209387E7F903A307006303A3
:10388000030002838280114517F3FFFF670063C6C0
:10389000411193962500AA852D4506C697F0FF1F76
:1038A000E780C0F0B240014541018280011122CC85
:1038B00006CE3714004026CA4AC84EC652C48344B6
:1038C0007405034AB405834984050349940597F0B8
:1038D000FFFFE780E09C8347A40593F4F40F137A7D
:1038E000FA0F93E71700230DF40493F9F90F1379F6
:1038F000F90FB717004003C7A705058B6DFF03D568
:10390000C705A38D4705238C3705A38C2705A38BFB
:103910009704F2406244D2444249B249224A0561C6
:10392000828041119397050122C406C626C2C18731
:103930002E8463DC0700B7E40400FC54829719C1AD
:10394000BC5482972165218D15A893F7150013C5E6
:1039500015008DE793F725009DC797000000E780CD
:1039600060EEB7E70400BC4F1306000A894517054F
:1039700000200345A5EA829713452400B240224463
:103980009244410182809397250163D80702B7E4EE
:10399000040083A7C41E829797000000E780E0EE32
:1039A000BC4C375607001306063089651705002002
:1039B0000345C5E68297096579B7939715010145D7
:1039C000E3DE07FA17C501001305056E97B0010085
:1039D000E780E0CEB7E70400BC4F130600649165B2
:1039E00017050020034585E382971165A9BF2D7156
:1039F000232A9110FD74E98C232C81102328211196
:103A0000232631112A84AE893289930600100A8652
:103A1000A6852D45232E111097F0FF1FE78000D9B2
:103A200013154401B7E70400FC4751810A051396BA
:103A30002900CA850A958297A6858566014625458F
:103A400097F0FF1FE78080D60A86A68593060010B0
:103A5000294597F0FF1FE78060D58320C11103241B
:103A6000811183244111032901118329C11015619A
:103A70008280B7F7070003C70701411106C622C4B9
:103A800026C24AC0A547631DF70097000000E780E3
:103A900040F6B240224492440249014541018280ED
:103AA00013942500AA843289A286AA850146254559
:103AB00097F0FF1FE78080CFA2864A86A68529451A
:103AC00097F0FF1FE78080CEE9B71D71A2CC37E4E5
:103AD00004005C5C485886CE494697C50100938532
:103AE0002558829711E917C501001305A55897B00D
:103AF0000100E780C0BC01A0B7F600E0795798CA82
:103B0000FD57DCCA0567B7E700E023A0E7101306FE
:103B1000F00290C223A0E71801000100370700203F
:103B200018471306000481459706002023A6E6CE19
:103B30004157A38AE7403C44080882979707002032
:103B40009387876A3EC8856713870740231AE10079
:103B50001D673ACC37070105130707103ACE938744
:103B600057D11307B00F2310E1022312F1020547CA
:103B700097F7FFFF938707522301E1023ED817070B
:103B80000000130727D197070000938767D2B7F586
:103B90000700BAC23EDC170700001307C7ED9707FE
:103BA0000000938787CE81463000E1051945BAC4ED
:103BB0003EDE97F0FF1FE78060BF180881479946F7
:103BC00030003E960346060085070507A30BC70095
:103BD000E398D7FEC24791C70357410185676373D6
:103BE000F70001A0B7E7040083A7470A08088297F7
:103BF000AA8511C917C501001305054997B0010031
:103C0000E780009401A0F64066442561828041115E
:103C100026C2B7E4040083A7040806C622C4170519
:103C20000000130545D0829717040020130404BF39
:103C30002300A40097000000E780800297000000A6
:103C4000E780A0BB03450400224403A38405B240DF
:103C5000924413060032896541010283797106D6C8
:103C600022D413078008F337078093F787083EC2F2
:103C700001000100B7170040930570052380B704C9
:103C8000130680FA2380C7040100010083C6F702EF
:103C900093F6A60FA387D702238007049246F3A6C4
:103CA00006800100010073370780137787083AC444
:103CB000010001002380B7042380C7040100010034
:103CC00003C7F70213672700A387E70223800704CF
:103CD000A247F3A7078001000100054597E0FFFF19
:103CE000E780405F97000000E78020BA01478146E7
:103CF0008147054685451305407E97E0FFFFE78035
:103D0000406237E404003C44680051468145829794
:103D1000B707C0A83EC8B787E803938707D03ECA55
:103D200097E7FF1F9387A7693EC67C586800829774
:103D3000B250225445618280411197D5010093858C
:103D4000E59C17C501001305252D06C697A00100A7
:103D5000E780007F17D50100130505B497A0010087
:103D6000E780007EB2402945410117B3010067009A
:103D70000382411197D501009385859A17C50100EB
:103D80001305852906C697A00100E780607B17D53B
:103D90000100130525AF97A00100E780607AB240CB
:103DA0002945410117A301006700637E411122C428
:103DB00006C6834705002A849DC797D501009385D1
:103DC000E59B17C501001305252597A00100E78095
:103DD00020774C4017D50100130545BA97A0010084
:103DE000E78000763DA058410DEF97D501009385FF
:103DF000E59817C501001305252297A00100E7806B
:103E0000207417D501001305E5B897A00100E780DD
:103E100020732244B2402945410117A301006700E5
:103E20000377A1679386D7036313D70297D5010061
:103E30009385C59417C501001305051E97A00100C1
:103E4000E780007017D501001305C5B57DBFED07EC
:103E500097D501009385859217C501001305C51BF1
:103E6000631BF70097A00100E780806D17D5010064
:103E7000130585B459BF97A00100E780606C4C40E2
:103E800017D50100130545B591BF411197D5010024
:103E90009385458A17C501001305051806C697A026
:103EA0000100E780E069B2402945410117A3010004
:103EB0006700E36D797122D426D24AD02E842A89F4
:103EC0008145B2844800714606D697E0FFFFE7803F
:103ED000C02097F7FF1F9387674ADC4783D7070007
:103EE000231421012313F10097500000E780608123
:103EF0009547A305F1009307401F3EC6FD572305D4
:103F0000A100230AF10097500000E780C0932686A5
:103F1000A285480097500000E7808081B25022546B
:103F20009254025945618280971700202391077CA3
:103F300097170020238A076AB7E70400BC4741119E
:103F400006C641468145170500201305651882976E
:103F500097200000E780A05697200000E780C0313E
:103F6000014597500000E780803217070020034783
:103F700027189307F00A6315F7029307F0F88945AD
:103F8000170500201305C516170700202302F71692
:103F900097070020A38E071497500000E780C059B0
:103FA00097500000E7808066814537050400970739
:103FB000002023AD071097070020239707109707CD
:103FC00000202384071097070020239507089707F0
:103FD000002023930706970700202396070E9707D4
:103FE0000020239F070E97300000E78040C5014561
:103FF00097500000E780405D97C5010093850576E6
:1040000017C501001305450197A00100E780405343
:1040100017D50100130585A297A00100E780405243
:10402000B2402945410117A30100670043564111E1
:1040300022C406C626C293F715002E84638F07108C
:10404000814617F6FF1F1306A63085451705002089
:10405000035545FE97C00000E78040C015C997C5CD
:1040600001009385657017C501001305E5FA97A057
:104070000100E780E04C17C501001305A51197A0CA
:104080000100E780E04B294597A00100E780205020
:1040900097C501009385456D17C501001305C5F748
:1040A00097A00100E780C04917C501001305C50F9F
:1040B00097A00100E780C048294597A00100E7804C
:1040C000004D17F5FF1F1305652B5C450547239031
:1040D000E70097300100E780C07097C50100938525
:1040E000A56817C50100130525F397A00100E78017
:1040F000204517C501001305650C97A00100E78056
:104100002044294597A00100E7806048930710F8F4
:1041100017070020230EF7FC9707002083D747F1ED
:1041200017070020A306F7FC17050020130545FC20
:10413000A183914517070020230DF7FA9707002068
:10414000A38907FA97500000E780003F1345140049
:10415000B240224492444101828093F72500E1C39A
:1041600017070020035747F645CB97060020938694
:10417000E6F5944297D701009387478E17060020F3
:104180000346A6F4814517050020130565F49770D2
:104190000000E78000CCAA8441C197C50100938547
:1041A000656317C50100130525E797A00100E780A7
:1041B0002039A68517C501001305C50197A0010088
:1041C000E7800038294597A00100E780403C970729
:1041D0000020239B07EE930710F817070020230900
:1041E000F7F09707002083D7A7E417070020A30163
:1041F000F7F0A18317070020230DF7EE91458D47B7
:10420000170500201305C5EE17070020A303F7EEDE
:1042100097500000E78040321345240015BF93F704
:104220004500D1C397C501009385C55A17C5010044
:10423000130585DE97A00100E780803017C50100D7
:10424000130505FB97A00100E780802F294597A063
:104250000100E780C033930720F8170700202309E7
:10426000F7E89707002083D7E7DE17070020A301B0
:10427000F7E8A18317070020230DF7E68547170706
:104280000020A308F7E697400000E780C05B170511
:1042900000201305E5E5914597500000E780C0290F
:1042A0001345440075B593F78500A9C797C501006C
:1042B0009385455217C50100130505D697A0010047
:1042C000E780002817C501001305C5F397A001007A
:1042D000E7800027294597A00100E780402B97073A
:1042E0000020239307DE97700000E78060C6134527
:1042F0008400B9BD93F70501D1C38545170500209A
:10430000035545D597500100E780807897C5010097
:104310009385454C17C50100130505D097A00100F2
:10432000E780002217C50100130505EF97A00100E3
:10433000E7800021294597A00100E78040259307E9
:1043400030F8170700202305F7DA9707002083D7F6
:1043500067D017070020A30DF7D817050020130515
:1043600025D9A1838D45170700202304F7D897503E
:104370000000E780601C13450401D9BB93F70502D8
:10438000D1C797C501009385E54417C50100130502
:10439000A5C897A00100E780A01A17C50100130562
:1043A000E5E997A00100E780A019294597A0010041
:1043B000E780E01D930740F817070020230AF7D293
:1043C0009707002083D747C717070020A302F7D21B
:1043D000A18317070020230EF7D085471707002079
:1043E000A309F7D097070020239807C4974000003F
:1043F000E780604517050020130585CF914597504C
:104400000000E78060131345040299B393F7050495
:10441000FDC397C501009385E53B17C50100130552
:10442000A5BF97A00100E780A01117C501001305E3
:1044300065E297A00100E780A010294597A0010040
:10444000E780E0149707002083C787CA1307700A24
:104450006386E7061307800A638CE7081307600A80
:104460006393E704930760F8170700202302F7C857
:104470009707002083D727C517070020A30AF7C690
:10448000A183170700202306F7C6854717070020DA
:10449000A305F7C6B14517050020130565C597505C
:1044A0000000E780600997400000E780C0391345AD
:1044B000040497070020239807C059B9930770F8A0
:1044C000170700202306F7C29707002083D7A7BF4E
:1044D00017070020A30EF7C0A18317070020230AA7
:1044E000F7C0854717070020A306F7C0994565B7B1
:1044F000930780F8F1B793F705080145E38A07C4ED
:1045000097C501009385052D17C501001305C5B09A
:1045100097A00100E780C00217C50100130505D56B
:1045200097A00100E780C001294597A00100E7801E
:1045300000069307A0F817070020230BF7BA970788
:10454000002083D7E7B917070020A303F7BAA18398
:1045500017070020230FF7B8854717070020A30A85
:10456000F7B897070020239D07B697400000E78023
:10457000802D170500201305A5B791459750000021
:10458000E78080FB13450408E1B6411122C497C5BA
:1045900001009385E51F2A8417C501001305C5A7EF
:1045A00006C697A00100E780A0F94C4017C501009E
:1045B0001305453A97A00100E78080F8294597A0A8
:1045C0000100E780C0FC034704009307F00F631F5E
:1045D000F70297C501009385A51B17C501001305B8
:1045E000A5A397A00100E780A0F54C4017C50100E6
:1045F0001305453797A00100E78080F42244B240BC
:104600002945410117A30100670063F8B240224425
:1046100041018280B1C1411122C417C501001305B7
:10462000A59F2E8497C501009385851106C697A086
:104630000100E780E0F0A28517C501001305C53D24
:1046400097A00100E780C0EF2244B2402945410114
:1046500017A301006700A3F38280411122C426C280
:104660002E84AA8497C501009385450E17C50100C5
:104670001305859A06C697A00100E78060EC17C570
:1046800001001305253A97A00100E78060EB29455A
:1046900097A00100E780A0EF97C501009385050B67
:1046A000970700202398979817C501001305C59612
:1046B000854497070020239D879697070020239A1B
:1046C0009796971700202394870297A00100E78010
:1046D00020E79715002083D5850117C50100130534
:1046E000E53497A00100E780A0E5294597A00100E7
:1046F000E780E0E997170020238897EE97200000D5
:10470000E78080B7228597500000E78040B80545D4
:1047100097500000E78040EB97F7FF1F938707C68D
:10472000DC4703D70700C167FD176312F702224475
:10473000B7E70400B240924403A3870517F5FF1FB3
:104740000345450E1306000A854541010283B24028
:104750002244924441018280011122CC37E40400BA
:104760005C5C06CE354697C501009385251417D5A8
:104770000100130525CE829711E917C50100130525
:10478000658F97A00100E78080F301A097F7FF1FD6
:104790009387070A3EC4B7F50700856793870780AC
:1047A000814617F6FF1F13062608E10519453EC688
:1047B00097E0FF1FE78080FF7C44194697F5FF1FB5
:1047C0009385850617050020130505898297340017
:1047D00017F6FF1F1306460597C501009385055F71
:1047E00017C501001305056097600000E780603B76
:1047F0002A841DCD97C501009385C5FC17C501000E
:104800001305858197A00100E78080D3A28517C595
:1048100001001305A50A97A00100E78060D2294591
:1048200097A00100E780A0D6F24062440561828033
:1048300097E00000E780C09D17C50100130505FF44
:1048400097500000E780A02F97A00000E78000F2BB
:1048500097500100E780805617F5FF1F130585AEBE
:1048600097500100E780203F17C50100130505FDA3
:1048700097500100E78000572A8497600000E78086
:10488000E09597000100E780602E97800100E780A7
:1048900080C797700000E78020EE97600000E780F7
:1048A000E00B97300100E780C0EF97C501009385CA
:1048B00065F117B501001305257619C897A0010009
:1048C000E78000C8A28517C5010013056501A1B7DF
:1048D00097A00100E780C0C617C501001305850237
:1048E00097A00100E780C0C5294597A00100E78097
:1048F00000CA97300100E780A0CB97F00000E78066
:1049000060EA55C985453705040097200000E78017
:10491000003397C501009385E5EA17B5010013053B
:10492000A56F97A00100E780A0C117C5010013057E
:10493000E5FE97A00100E780A0C0294597A00100EF
:10494000E780E0C497F7FF1F9387079383D707009B
:1049500017170020231DF7D88547171700202305B8
:10496000F7C897200000E78000B097200000E7809C
:10497000A09017150020035585D797500000E780B9
:104980000091054597500000E78000C497C50100DD
:10499000938545E317B501001305056897A001004D
:1049A000E78000BA17C50100130585F997A001003B
:1049B000E78000B9ADB597C501009385A5E017B5AF
:1049C00001001305656597A00100E78060B717C572
:1049D00001001305A50697A00100E78060B62945F0
:1049E00097A00100E780A0BA014569BF411122C428
:1049F00037E404008327041A06C682979750000004
:104A0000E780A08C8327040817F5FFFF1305656274
:104A1000829797F7FF1F2387A7E017F5FF1F13055E
:104A2000E59597400000E780A0142244B240410180
:104A300017030000670083D2B7E70400FC47117139
:104A4000A2DDCAD986DFA6DBCED72E8432892E8698
:104A5000AA8517F5FF1F1305A569829717F7FF1F92
:104A60001307076983470700930680029387E707C8
:104A700093F7F70FE3ECF610BA898A0717B701002E
:104A80001307C762BA979C43BA9782878D4797C529
:104A90000100938565D517B501001305E557630F30
:104AA000F40097A00100E780A0A917C50100130535
:104AB000659297A00100E780A0A8BDA497A001007F
:104AC000E78000A817C501001305459297A00100D3
:104AD000E78000A7294597A00100E78040AB930736
:104AE00020F8114697F5FF1F938585604A8517F7D3
:104AF000FF1F230FF75E97F7FF1FA38C075E97F04A
:104B0000FFFFE780603B2A841DC997C5010093859C
:104B1000A5CD17B501001305255097A00100E7802A
:104B200020A2A28517C501001305059097A00100DA
:104B3000E78000A1294597A00100E78040A597C51F
:104B40000100938565CA17B501001305E54C97A0D0
:104B50000100E780E09E17C501001305258E97A090
:104B60000100E780E09D294597A00100E78020A291
:104B70004165930730FA054697F5FF1F9385455722
:104B80007D1517F7FF1F2305F75697F0FFFFE78006
:104B9000A0322A841DC997C501009385E5C417B5C5
:104BA00001001305654797A00100E7806099A28581
:104BB00017C501001305458797A00100E7804098BD
:104BC000294597A00100E780809CB7E70400BC4F0F
:104BD0000566130606C8A14517F5FF1F034585C4E2
:104BE0008297FE506E54DE544E59BE591161828038
:104BF00091476303F40297C501009385E5BE17B59D
:104C000001001305654197A00100E780609317C577
:104C100001001305E58571BDB7E70400FC4F914520
:104C200017F5FF1F034505C0829797C501009385BF
:104C3000A5BB17B501001305253E97A00100E7802D
:104C4000209017C501001305658497A00100E78037
:104C5000208F294597A00100E780609397400000CE
:104C6000E78060BE914535A485476303F40297C58C
:104C70000100938565B717B501001305E53997A0C5
:104C80000100E780E08B17C501001305A58115B56C
:104C900097F7FF1F2390273DB7E704000566BC4F39
:104CA000130606C8C1450DBF8D476303F40297C5BF
:104CB0000100938565B317B501001305E53597A08D
:104CC0000100E780E08717B501001305657FD5B3C4
:104CD000930740F8114697F5FF1F938565414A8574
:104CE00017F7FF1F2306F74097F7FF1FA38307401F
:104CF00097F0FFFFE780401C2A84E30405EE97C588
:104D00000100938565AE17B501001305E53097A046
:104D10000100E780E082A28517B501001305C57088
:104D200097A00100E780C081294597A00100E78096
:104D3000008645BD9147E31CF4F6B7E70400FC4F3D
:104D40009305000217F5FF1F0345C5AD829797C570
:104D50000100938565A917B501001305E52B979010
:104D60000100E780E07D17B501001305E576F1BD90
:104D7000894763E3870297C501009385E5A617B5C8
:104D800001001305652997900100E780607B17B546
:104D900001001305A57531BB97F4FF1F83C464356B
:104DA00097F7FF1F83C7D73497C501009385C5A325
:104DB000A20417B5010013052526DD8C979001008C
:104DC000E7800078A28517B50100130565739790F9
:104DD0000100E780E076C204294597900100E78052
:104DE000007BC1849305D4FF93960401C1824A8657
:104DF00093F5F50F17F5FF1F1305B52F972000004A
:104E0000E780A0E7E35F90DC930750F817F7FF1FF8
:104E10002300F72E83C73900228697F5FF1F93855D
:104E2000252D85074A8517F7FF1FA304F72C97F058
:104E3000FFFFE78060082A84E30505DA97C50100D3
:104E40009385859A17B501001305051D97900100FC
:104E5000E780006FA28517C501001305E5BAC9B543
:104E6000894763E3870297C501009385E59717B5E6
:104E700001001305651A97900100E780606C17B573
:104E800001001305A56935B197400000E780A09B9C
:104E9000A28517F5FF1F1305A52597400000E780A1
:104EA000A06981B38D476303F40297C50100938520
:104EB000A59317B501001305251697900100E7800B
:104EC000206817B5010013052567E5B6B76602002F
:104ED0000146B7750200054597E0FF1FE780008D8A
:104EE000930760F817F7FF1F2304F72097F7FF1FBA
:104EF000A38107209307000617F7FF1F230CF71E57
:104F0000894717F7FF1FA307F71E97F7FF1F238493
:104F1000071E97F7FF1FA380071EC14717F7FF1F44
:104F2000230CF71C930720F917F7FF1FA306F71CA4
:104F3000314697F7FF1FA382A71C97F5FF1F9385A4
:104F4000251B4A8597F7FF1F2389071A97F0FFFF54
:104F5000E78080F62A84E30605C897C5010093859B
:104F6000A58817B501001305250B97900100E78070
:104F7000205DA28517B501001305855D55B3B147C6
:104F80006303F40297C501009385058617B50100F8
:104F90001305850897900100E780805A17B5010036
:104FA0001305C55C39B6B7E70400FC4F9305000450
:104FB00017F5FF1F03450587829797400000E7809C
:104FC0008088B145F9B5914763E3870297C5010031
:104FD0009385858117B5010013050504979001009D
:104FE000E780005617B501001305055AD9B497F4A8
:104FF000FF1F83C4241097F7FF1F83C7970FA204D6
:10500000DD8C8E04B77702006D14BE942286A685CF
:1050100017B501001305855897900100E7804052AD
:10502000B7E70400FC47228697F5FF1F9385950C90
:105030002800829793160401C1823000A685094595
:1050400097D0FF1FE78080762A8409C917B5010031
:105050001305855697900100E7806066930770F806
:10506000194697F5FF1F9385A5084A8517F7FF1F77
:105070002300F70897F7FF1FA38E870697F0FFFF1F
:10508000E78080E32A84E30E05B497B50100938599
:10509000A57517B50100130525F897900100E78065
:1050A000204AA28517B501001305055295B9994705
:1050B000630BF41297B501009385057317B50100D2
:1050C000130585F597900100E780804717B501002B
:1050D00013050551F9BA914763E3870297B50100BB
:1050E0009385857017B50100130505F397900100AE
:1050F000E780004517B50100130505505DBA97F428
:10510000FF1F83C424FF97F7FF1F83C797FEA204E6
:10511000DD8C8E04B77702006D14BE942286A685BE
:1051200017B501001305854E97900100E7804041B7
:10513000B7E70400FC47228697F5FF1F938595FB90
:105140002800829793160401C1823000A6850D4580
:1051500097D0FF1FE78080652A8409C917B5010031
:105160001305854C97900100E7806055930780F800
:10517000194697F5FF1F9385A5F74A8517F7FF1F77
:105180002308F7F697F7FF1FA38687F697F0FFFF30
:10519000E78080D22A84E30605A497B501009385B1
:1051A000A56417B50100130525E797900100E78076
:1051B0002039A28517B501001305454895B69947D2
:1051C0006303F40297B501009385056217B50100EA
:1051D000130585E497900100E780803617B501003C
:1051E00013054547F9B0B7E70400FC4F93050004E9
:1051F00017E5FF1F03450563829797300000E7809E
:105200008064994579B18D476303F40297B5010035
:105210009385855D17B50100130505E097900100A2
:10522000E780003217B501001305454459B017B5A2
:1052300001001305A54497900100E780404813053D
:10524000C01297D0FF1FE780C00F014597E0FFFF16
:10525000E78040E10D4597100000E780009F294559
:1052600097D0FF1FE780E00D97D0FF1FE78040FE3B
:105270008DBA99476303F40297B501009385C5562B
:1052800017B50100130545D997900100E780402B21
:1052900017B501001305453F29B817F7FF1F03474E
:1052A00077E597F7FF1F83C7E7E422075D8F9166D5
:1052B000BA96C2061166C1821306F6EF8D47636582
:1052C000D60297E7FF1F9387670B9C4B17F6FF1FCC
:1052D000034636E29386C7002DC203D6070069CA8B
:1052E0008907E39CD7FE89471307A0F8114697F575
:1052F000FF1F9385E5DF4A8597F6FF1F238AE6DEC9
:1053000017F7FF1FA307F7DE97F0FFFFE780C0BA8C
:105310002A84E308058C97B501009385E54C17B501
:105320000100130565CF97900100E7806021A285F9
:1053300017B5010013058536E5B203D60700630EE5
:10534000E60A8907E39BF6FE8D4779BF9147630420
:10535000F40297B501009385254917B5010013059F
:10536000A5CB97900100E780A01D17B5010013059C
:1053700065346FF00FF4B7E70400FC4F93050008A5
:1053800017E5FF1F0345054A8297C9B897B5010085
:105390009385854517B50100130505C89790010051
:1053A000E780001A17B50100130545326FF06FF062
:1053B0002390E70017E5FF1F130545FC9720010028
:1053C000E780804497B501009385054217B5010039
:1053D000130585C497900100E780801617B501007A
:1053E0001305C52F97900100E780801529459790F8
:1053F0000100E780C0198147C5BD2390070017E56C
:10540000FF1F1305A5F797200100E780E03F97B540
:1054100001009385653D17B501001305E5BF979021
:105420000100E780E01117B501001305A52C5DBF51
:10543000411122C406C6834705002A849DC797B53B
:1054400001009385253617B501001305E5BC97903B
:105450000100E780E00E4C4017B50100130505611F
:1054600097900100E780C00DE1A05841B707CF0039
:105470009387777D631DF70697B501009385853285
:1054800017B50100130545B997900100E780400B5F
:105490001C448356E4008355C40003C6070017B5B7
:1054A00001001305255E97900100E78060092945FA
:1054B00097900100E780A00D0357E40097070020B4
:1054C00083D7E7226309F7008355C400084497E0B7
:1054D000FFFFE780E0CD0356E4008355C400084495
:1054E0002244B240410117F3FFFF67002355B7077D
:1054F000CC009387777D6315F70497B501009385FA
:10550000652A17B50100130525B197900100E780C2
:1055100020031C448356E4008355C40003C60700DF
:1055200017B501001305055697900100E78040016B
:105530002244B24029454101179301006700230529
:10554000B707CE009387777D6304F70297B5010014
:105550009385452517B50100130505AC979001000B
:10556000E78000FE4C4017B501001305E546CDBDB0
:10557000B240224441018280B7E70400FC47411158
:105580002E8606C622C426C24AC02E842A89AA852F
:1055900017F5FF1F1305C5B5829797B501009385D1
:1055A000652617B50100130525A797900100E78030
:1055B00020F997F5FF1F83C5A5B317B501001305A3
:1055C00065CC97900100E780A0F7294597900100EE
:1055D000E780E0FB97F4FF1F938484B183C7040046
:1055E00041479387070693F7F70F636AF75C17B78E
:1055F00001001307E7B58A07BA979C43BA978287D9
:105600009D476307F40297B501009385A51F17B561
:105610000100130565A097900100E78060F217B5BF
:1056200001001305A5C697900100E78060F1ADACBD
:1056300097F7FF1F83C7D7ABDDCB17F7FF1F0347D4
:1056400057AB97F7FF1F83C7C7AA22075D8F97F74E
:10565000FF1F83C727AAC2075D8F97F7FF1F83C766
:1056600077A9E207D98F17F7FF1F2321F7A683C772
:10567000640097B501009385E51817B5010013057F
:10568000A59917F7FF1F2302F7A497900100E78061
:1056900020EB97F7FF1F938767A38C4317F6FF1F35
:1056A0000346A6A217B50100130505C09790010097
:1056B000E78000E9294597900100E78040ED97F7E2
:1056C000FF1FA38707A22244B240924402499307D6
:1056D00000F817F7FF1F230DF7A09D4517F5FF1FD3
:1056E000130505A14101174300006700E3E497603B
:1056F0000000E780609597F7FF1F238CA79E9357C4
:10570000850017F7FF1FA306F79E935705012A840C
:1057100017F7FF1F2300F79E93578501014517F7E1
:10572000FF1FA309F79C97600000E780A09297F7FE
:10573000FF1F2382A79C97B501009385A50C17B581
:1057400001001305658D97900100E78060DF17F673
:10575000FF1F0346469AA28517B50100130545B6FB
:10576000B1B7CD476303F40297B50100938585096E
:1057700017B501001305458A97900100E78040DCCA
:1057800017B50100130545B579BD37E404007C4425
:10579000414697F5FF1F9385B59517F5FF1F130534
:1057A0002593829717F5FF1F130585929710000028
:1057B000E78080C497100000E78000AC97F7FF1FD8
:1057C00083C7279417F7FF1F03479793A207032365
:1057D0008405D98F17F7FF1F2318F78E1306000AC9
:1057E00089452244B2409244024917E5FF1F034510
:1057F0006503410102838D476303F40297B50100FD
:105800009385450017B501001305058197900100A8
:10581000E78000D317B501001305C5BB29B517F400
:10582000FF1F0344048D97F7FF1F83C7778C97B53D
:105830000100938525FD220417A501001305C57DF0
:105840005D8C97900100E780A0CFA28517B501007D
:10585000130505AA97900100E78080CE294597900F
:105860000100E780C0D20D4697F5FF1F938545885C
:10587000228597E0FFFFE7802064AA8421C197B5C5
:105880000100938525F817A501001305E578979089
:105890000100E780E0CAA68517B50100130585A6BB
:1058A00097900100E780C0C92244B2409244024967
:1058B0002945410117930100670063CD97E7FF1F5A
:1058C000239A8778B7E70400116603A387051306B8
:1058D00006E8914539B78D476303F40297B5010097
:1058E000938545F217A501001305057397900100F4
:1058F000E78000C517B50100130585BC2DB317E47B
:10590000FF1F0344047F97E7FF1F83C7777E97B588
:105910000100938525EF220417A501001305C56F2B
:105920005D8C97900100E780A0C1A28517B50100AA
:105930001305859E97900100E78080C029459790C8
:105940000100E780C0C40D4697E5FF1F9385457AA7
:10595000228597E0FFFFE7802056AA841DC197B5F6
:105960000100938525EA17A501001305E56A9790C4
:105970000100E780E0BCA68517B501001305059B73
:1059800005B797E7FF1F2399876AB7E704001166F9
:1059900003A38705130606E89305000299B5894716
:1059A00063E3870297B501009385C5E517A501005C
:1059B0001305856697900100E78080B817B5010050
:1059C0001305C5B28DB197E4FF1F83C4847297E7B6
:1059D000FF1F83C7F77197B501009385A5E2A20465
:1059E00017A5010013054563DD8C97900100E78042
:1059F00020B5A68517B501001305C5949790010041
:105A0000E78000B4294597900100E78040B82286DE
:105A100097E5FF1F9385C56D268597E0FFFFE7801B
:105A2000A0492A84630E051A97B50100938585DD88
:105A300017A501001305455E97900100E78040B06F
:105A4000A28517B501001305259199BD854763F916
:105A50008718834519002244B24092440249B33565
:105A6000B00097E7FF1F2381B76017B5010013054A
:105A7000E58F410117930100670083ACA2852244A2
:105A8000B24092444A850249410117030000670071
:105A9000032299476303F40297B50100938585D6E5
:105AA00017A501001305455797900100E78040A90D
:105AB00017B50100130545BDBDB617E4FF1F03442C
:105AC000446397E7FF1F83C7B76297B501009385CB
:105AD00065D3220417A50100130505545D8C97902A
:105AE0000100E780E0A5A28517B5010013058589AF
:105AF00097900100E780C0A4294597900100E780B6
:105B000000A9194697E5FF1F9385855E228597E0DA
:105B1000FFFFE780603AAA841DC197B50100938515
:105B200065CE17A501001305254F97900100E7806A
:105B300020A1A68517B501001305C58595B397E784
:105B4000FF1F239F8758B7E70400116603A387054B
:105B5000130606E89305000869B1854797B501006B
:105B6000938545CA17A501001305054B630BF40087
:105B700097900100E780C09C17B501001305C5820E
:105B80005DB497900100E780A09B17B50100130555
:105B9000258397900100E780A09A294597900100FE
:105BA000E780E09E2244B2409244024997E7FF1FFB
:105BB000239C07504101175300006700633997B5D4
:105BC0000100938525C417A501001305E5449790AE
:105BD0000100E780E09617B50100130525AFA1B4D9
:105BE000B24022449244024941018280411106C6DA
:105BF00022C497E0FFFFE780202C9377F50FA1C325
:105C00002A8497B50100938565C117A50100130586
:105C1000A54097900100E780A0929375F40F17B507
:105C20000100130565DE97900100E7806091224432
:105C3000B240294541011793010067004395B240E6
:105C4000224441018280411122C491462A8417E6F0
:105C5000FF1F130626589D652D4506C697D0FF1FCA
:105C6000E780C0B4B7F7070003C70701A547631370
:105C7000F70001A09306001001469D65254597D0C9
:105C8000FF1FE780A0B297E7FF1F238587542244B8
:105C9000B240914617E6FF1F1306C6539D6529457E
:105CA000410117D3FF1F670063B05171CAD137E9B3
:105CB00004008327C904A2D52E8686D7A6D32E84B6
:105CC000AA8517E5FF1F1305A542829797E7FF1FD7
:105CD00083C707421307700A6387E710636CF700F6
:105CE0001307600A6384E704BE502E549E540E5975
:105CF0006D6182801307800A6388E7161307900A94
:105D0000E394E7FE8D476309F41C97B50100938582
:105D1000E5E217A501001305253097900100E78003
:105D2000208217B501001305A5DE25A08D47630C61
:105D3000F40297B50100938565E017A501001305EE
:105D4000A52D97800100E780A07F17B501001305FE
:105D500065D597800100E780A07E294597900100D6
:105D6000E780E08251B7854717B50100130545D597
:105D700017E7FF1F230AF72E97900100E780209472
:105D8000B7750200B76602000146054597D0FF1FB0
:105D9000E780C0A1930760F817E7FF1F230AF734D5
:105DA00097E7FF1FA38707349307002617E7FF1F16
:105DB0002322F734E5779387072117E7FF1F231D79
:105DC000F732B14597E7FF1F2389073297E7FF1F97
:105DD000A385A73217E5FF1F130585319730000013
:105DE000E780807511B7914763E3870297B501009B
:105DF0009385C5D417A501001305052297800100DE
:105E0000E780007417B50100130585CD99B797E4B5
:105E1000FF1F83C4242E97E7FF1F83C7972DA2047B
:105E2000DD8C8327C9046D14228697E5FF1F9385B7
:105E3000752C280082978E0493160401B775020012
:105E4000C1823000A695094597D0FF1FE7800096D4
:105E5000930770F817E7FF1F230CF728994597E77A
:105E6000FF1FA389A728BDB7914763E3870297B5B2
:105E700001009385A5CC17A501001305E5199780AE
:105E80000100E780E06B17B501001305E5C6D1B549
:105E900097E4FF1F83C4042697E7FF1F83C7772576
:105EA000A204DD8C8327C9046D14228697E5FF1FA9
:105EB00093855524280082978E0493160401B775A4
:105EC0000200C1823000A6950D4597D0FF1FE780E4
:105ED000E08D930780F8BDBF17B50100130585C499
:105EE00097800100E780A07D1305C01297C0FF1FB7
:105EF000E7802045014597D0FFFFE780A0160D45BC
:105F000097000000E78060D4294597C0FF1FE78015
:105F1000404397C0FF1FE780A033F9B341114AC047
:105F200097F6FF1F83D6A67C328917D6FF1F03562C
:105F3000064722C426C206C62A84AE849700000003
:105F4000E780C05F35C12DC0994763FF9704834741
:105F5000140003470400A207D98F13978700A18379
:105F6000D98FC2073167C1831307C755639EE70204
:105F700097D7FF1F83D7A742A301F400A183230271
:105F8000F40097F7FF1F83D7877691C7A302F40029
:105F9000A1832303F400A68517B50100130505BEF0
:105FA00097800100E780C05997F7FF1F83C7C76339
:105FB000B9CF97D5FF1F83D5853E17B501001305CF
:105FC000A5BD97800100E780A0572686A28517D53A
:105FD000FF1F0355C53C97000000E78060C16301C7
:105FE000090497E7FF1F83C7E71F9DCB95C897E775
:105FF000FF1F83C767078DE722852244B24002490D
:10600000A68592444101173300006700E35217B59B
:106010000100130565B997800100E780406AC1B7A8
:10602000B240224492440249410182808347550094
:106030008345450017B50100130505B3A207DD8DA3
:10604000178301006700C34F17B501001305C5B0E2
:10605000178301006700A3668D4763FBB70A011130
:1060600026CA06CE22CC0344350097E4FF1F83C422
:10607000741797B501009385E5B3B337800017E730
:10608000FF1FA301F71609C497B50100938545B317
:1060900017B50100130545B397800100E780404A1A
:1060A00097E7FF1F83C717146386970097000000C8
:1060B000E780802697E7FF1F83C7D7128DC78547E4
:1060C0002306F100B7E7040083A747177000854552
:1060D00013055030829717B501001305E5AF97807F
:1060E0000100E780C05D9967938757EE2316F100A2
:1060F000680085479145A30781002307F100973089
:106100000000E7806043F2406244D244056182802F
:106110008280894763F7B708011122CC06CE26CAD0
:106120008344250085472A84639DF404914763F5E1
:10613000B704034545008347340022055D8D97D79A
:10614000FF1F239EA72497000000E780004899675F
:10615000938767EE2314F1008347340023059100F1
:10616000A305F10083474400954528002306F1006C
:1061700097300000E780403CF2406244D244056121
:106180008280FDF89967938767EE2314F10097D713
:10619000FF1F83D7C720A305F10023050100A183BA
:1061A000E1B782800111996722CCD51717F4FF1F40
:1061B000130484432314F1008347040026CA97F490
:1061C000FF1F9384C4522305F10083D704002800E5
:1061D0009545A305F100A18306CE2306F100973073
:1061E0000000E780603503D604008345040017B53E
:1061F00001001305E59F97800100E7806034F240BD
:106200006244D244056182809D677971D917231653
:10621000F10097F7FF1F83C7273D06D62307F1003C
:10622000A9C3B7E70400FC47414697E5FF1F9385E4
:1062300025EA1305F10082976800CD4597300000EC
:10624000E780802F97F5FF1F83C5053A17B501003A
:106250001305059D97800100E780802EB2504561AF
:106260008280B7E70400BC47414681451305F10031
:106270008297D9B7B76702045D71938757AA3EC06A
:106280008567938707102312F10097F7FF1F938705
:10629000A73583C70700A2C4A30301002303F100AD
:1062A00097F7FF1F9387A74483D7070037E40400BD
:1062B00086C62314F10097D7FF1F9387470E83D715
:1062C0000700414668002315F1007C4497E5FF1F55
:1062D000938505E08297F1450A8597000000E780E5
:1062E000E021231EA1007C448A850810794682970C
:1062F0003C441305E103094681458297101093053C
:106300000002014597D0FFFFE780003EB6402644DB
:1063100061618280B7C7A55A01119387C7333EC414
:1063200097E7FF1F83C717EC3EC6B7F7070003C701
:10633000070106CE22CCA5476313F70001A0116424
:10634000930504F0930600100146254597C0FF1FF2
:10635000E780C0453000930504F0A146294597C069
:10636000FF1FE780A04497E5FF1F83C5B5E717B57A
:1063700001001305A59B97800100E780601CF24097
:1063800062440561828001119165A14630009385C8
:1063900005F02D4506CE97C0FF1FE780204122471C
:1063A000B7C7A55A9387C7336314F702B24517B529
:1063B00001001305E58AB335B00097E7FF1FA383FB
:1063C000B7E297800100E780A017F2400561828064
:1063D000814517B501001305E58A97E7FF1FA383E1
:1063E00007E097800100E780A01597000000E78094
:1063F000A0F2E1BFB7C7A55A79719387F7353EC6BA
:10640000B7E70400FC47AA8506D622D4414608080F
:106410008297B7F7070003C70701A5476313F70083
:1064200001A01164930504E8930600100146254578
:1064300097C0FF1FE78080377000930504E8D146BE
:10644000294597C0FF1FE780603617B50100130587
:10645000A59197800100E7808026B25022544561C3
:10646000828079719165D1467000938505E82D454C
:1064700006D697C0FF1FE78060333247B7C7A55ADB
:106480009387F73517B501001305C5876310F70229
:10649000B7E70400FC4717E5FF1F130565C3414636
:1064A0000C08829717B501001305C583978001007A
:1064B000E780E020B25045618280B7F7070003C74C
:1064C0000701A5476313F70001A0916541119306E9
:1064D00000100146938505E8254506C697C0FF1FB5
:1064E000E780C02CB24017A501001305A575410136
:1064F000178301006700A31CC16769768146FD17F9
:1065000005061397060141836364B7003E858280C8
:106510003307D50003470700B98F214713F8170049
:10652000858363050800B18FC207C1837D17137788
:10653000F70F6DF78506F1B741C5A547054763F22B
:10654000B70883471500034705003168A207D98FB4
:1065500013978700A183D98FC207C1831308C85539
:10656000054763900707411106C622C426C20344AB
:106570002500914763F087049307540063ECF5020C
:10658000A301C50021822302C5009304340091C6F3
:10659000A302D500A1822303D5002A84A6859700F3
:1065A0000000E780A0F526942300A4002181A30029
:1065B000A4000147B240224492443A8541018280BE
:1065C00005473A858280B7C7A55A01119387E734FA
:1065D0003EC42AC6B7F7070003C7070106CE22CC80
:1065E00026CAA5476313F70001A091642A84938506
:1065F00004EE930600100146254597C0FF1FE78073
:10660000E01A3000A146938504EE294597C0FF1F8C
:10661000E780C019A28517A501001305257397808F
:106620000100E780E0F197000000E780E0C4F2405D
:106630006244D2440561828001119165A146300017
:10664000938505EE2D4506CE97C0FF1FE780001607
:106650002247B7C7A55A9387E7346318F702B245B4
:1066600017A501001305056497D7FF1F2399B7D21B
:10667000C205C18197800100E78080EC970000008F
:10668000E78080BFF24005618280D147D14517A5E0
:1066900001001305256317D7FF1F2312F7D097803A
:1066A0000100E780E0E917D5FF1F035545CF9700AC
:1066B0000000E78080F1F9B721C1411126C206C66A
:1066C00022C4AE848DC52A8497200000E78000BCD8
:1066D00097E7FF1F83C707B199CB22852244B240B9
:1066E000A68592444101173300006700E3E4B240FD
:1066F0002244924441018280828079714AD006D638
:1067000022D426D24ECE93F715002E899DCBAD67AD
:10671000371700409387A7AA1CC3B7E70400BC4FF4
:1067200013060019854517D5FF1F034525C7829716
:1067300013451900B250225492540259F24945614E
:10674000828093F725006388071E2D4697A50100D8
:1067500093858565480097800100E78000D397F610
:10676000FF1F83C6A6F8139706014183954763F977
:10677000E70C014417F5FF1F130545E71306300525
:1067800013085004930810041303B004130E90056B
:106790009307640063F4F6043A84FD5997F4FF1FED
:1067A00083C4C4E497F7FF1F83C757E4A204DD8CBA
:1067B000AD679387B755638CF41463E3970AA967B1
:1067C0009387A755638FF414A28517F5FF1F130550
:1067D000E5E197000000E78060EE39A2B30785008D
:1067E00083C50700639AC50483C517006396050532
:1067F00083C527006392150583C53700639EC502D4
:1068000083C54700639A650283C757006396C70331
:10681000A2890DE897F5FF1F83C545EDB385354186
:10682000C20517F5FF1F130565DCC1814E95970062
:106830000000E780A0E8E9A005044204418089BF88
:106840003A84FD598547E3EB87F445C8854517F53C
:10685000FF1F1305A5D997000000E78020E671A867
:10686000B1679387C7556380F404B5679387D7559D
:10687000E39CF4F4A28517F5FF1F130525D7973085
:106880000000E78060CB89476300F4069305E4FFCE
:10689000C205C18117F5FF1F130565D597200000BC
:1068A000E780C09E91A00546A28517F5FF1F13053E
:1068B000E5D397F0FFFFE780A06697F7FF1F83C738
:1068C000A7D29DE397E7FF1F83C7C79191CF4800E9
:1068D00097800100E78060E793150501C1814800BA
:1068E00097300000E78040C5A68517A50100130575
:1068F000A54997800100E780A0C4FD57E39CF9F00B
:1069000097F7FF1F238407DE1345290025B5A285CD
:1069100017F5FF1F130585CD97F0FFFFE780407146
:10692000E1B7A28517F5FF1F130545CC97F0FFFFD0
:10693000E780C07155BF93F745000145E38C07DE42
:1069400017A501001305854597800100E78020D732
:1069500097300000E78040CD13454900E1BB41116D
:1069600022C437E404005C5C06C6354697A50100E6
:106970009385C5F317B501001305C5AD829711E9DD
:1069800017A501001305054397800100E78020D378
:1069900001A08327041C82972A84054597C0000024
:1069A000E780608697600100E780800B97600100B8
:1069B000E78080E097B00000E780E0972285B24052
:1069C0002244410182801567B717004013075755CD
:1069D00098C3D8439D66558FD8C3D843FD76758F2D
:1069E000D8C3D8431367F70FD8C335671307C7CC8D
:1069F00098C382804111054506C622C426C297C0AD
:106A0000FFFFE78000501305800497B0FF1FE78069
:106A1000006A757585457D1597C0FFFFE780A03931
:106A20007D7585451305F53697C0FFFFE780004368
:106A3000371400408327840A8D451305002093E70F
:106A400007202324F40A97C0FFFFE780C036B7E48D
:106A5000040097C0FFFFE780207CC85897800100A2
:106A6000E780E0C517B501001305C59E97800100BA
:106A7000E780E0C48327840C8545414593E70708F8
:106A80002324F40C97C0FFFFE780403D8D4513059C
:106A9000000897C0FFFFE780603C97C0FFFFE780DA
:106AA0004069014597C0FFFFE780406C854505457B
:106AB000894717F7FF1F230DF7C297C0FFFFE78035
:106AC000806C37070004B7E700E023A0E71097D0F9
:106AD000FFFFE780C0FF97D0FFFFE780801397009C
:106AE0000000E78000E897000000E780008A970038
:106AF0000000E780A0B497E0FFFFE78060EF970019
:106B00000000E780601097000000E780600B83A71B
:106B1000040817050000130585BE829797D7FF1F4D
:106B2000238EA786BC4C1306006485458297970088
:106B30000000E78080E997C0FF1FE780608B014578
:106B40008280B7F7070003C70701A547AE86631623
:106B5000F7009397450191C301A0AA8501462545F9
:106B600017C3FF1F670083C44111B2862E86AA8512
:106B70002D4506C697C0FF1FE78040C3B2400145C0
:106B8000410182809307000463E8C7021D71A2CC13
:106B90002A84080886CE32C697800100E780E08EFE
:106BA000B2461008A285294597C0FF1FE78000C0A4
:106BB000F6406644256182803955828041110D6519
:106BC0008D4506C697C0FFFFE780E01EB71700405F
:106BD0008D6623A6D70A17F5FF1F1305A5B11387E6
:106BE000C70A9387870A1CC15CC5856689675CC92B
:106BF00058C114C518C9B7E70400B24003A3871EE3
:106C00004101028397F7FF1F83C747B099EF4111F6
:106C100006C697100000E7808061B240854717F7ED
:106C2000FF1F2305F7AE41018280828011C589C50F
:106C300017C3FFFF6700C3578280411126C2AE848D
:106C40008D4522C406C62A8497C0FFFFE780002135
:106C5000B717004099C803A5C70C418D23A6A70C00
:106C6000B240224492444101828003A5870C418DA9
:106C700023A4A70CF5B78347050003471500A20717
:106C8000D98FC2076177C18713072720639AE7006E
:106C9000834525003705040017030000670023FA29
:106CA000828017F6FF1F1306A6A68147B28613033C
:106CB000F00FA9483308F6000348080013F7F70F50
:106CC0006307A80C630668008507E39517FF29474B
:106CD000B387E6002380A70097F7FF1F938707A4D9
:106CE0005DA8411113D765001347170006C693F638
:106CF0003500058B954791CA054699476387C600BD
:106D000009469D476383C600A14713F64500333605
:106D1000C00093F68503050685C2A145638BB604C2
:106D2000E145638AB604930580026388B60493053F
:106D300080036393B600914697F5FF1F2385F5C442
:106D400097F5FF1F2380C5C497F5FF1FA38CD5C2FD
:106D5000BE8517A501001305650F97700100E78038
:106D6000207EB240854717F7FF1FA30EF7C04101F1
:106D700082808546D1B78946C1B78D4675BF17A5B4
:106D800001001305250F177301006700637B17F7D8
:106D9000FF1F1307A798BA972380B700E147E302C4
:106DA000F5F493077002E30CF5FC82802A872380B8
:106DB0000500814717F5FF1F130585951308F00F90
:106DC0002946B306F50083C606006396E60297F6E9
:106DD000FF1F9386A694B69783C7070005452380B7
:106DE000F5009947636EF7029D4763FDE700E147B1
:106DF000630DF7008280638506018507E393C7FC76
:106E00000145C5B7238005008280B737004003C71E
:106E1000370083C7050093F70704D98F2380F50057
:106E20008280797126D24AD097F4FF1F83C484C729
:106E300017F9FF1F130949C606D622D44ECE52CCED
:106E400056CA5AC8B307990083C7070093F7F70FCC
:106E5000A5C79387140093F7F70F0D476361F70CED
:106E600017F7FF1F2300F7C497F7FF1F938747C348
:106E7000A69783C707001307100293F7F703638FE2
:106E8000E7286363F70A054463808720E389076E78
:106E900009476389E71413070002E38EE758B7E751
:106EA00000E03707400023A0E71801000100CA9462
:106EB0002380040023A0E710B787004003C76700C2
:106EC000058BE30F077897F6FF1F83C6C6BD0547FE
:106ED000E39AE67629472381E70209472383E702FD
:106EE0002385E70297F7FF1FA38007AA97F7FF1FE5
:106EF000A38B07BAB7870040A381070017F7FF1FCE
:106F0000A30607A805472383E700B25022549254F2
:106F10000259F249624AD24A424B4561828097F750
:106F2000FF1F238107B889B7130730026386E70A7A
:106F300063E6E71413074002638AE70813070003B8
:106F4000E39FE7F497F7FF1F938747B5A69703C71B
:106F50000700A1471377F70FE31AF71C17EAFF1F83
:106F6000130A8A7C83476A0097F6FF1F2384F6A0E2
:106F700097E7FF1F83C7B77B91C7FD5797F6FF1FA2
:106F8000238AF69E97E5FF1F83C5157A97F7FF1FA3
:106F9000A382B79E97E7FF1F83C7077993F9070876
:106FA0009306000493F707066393D7529307A0094B
:106FB000638DF51A63EAB7169307F005638AF54EF9
:106FC000930750096388F52E014479ABFD5717F7F5
:106FD000FF1F2300F79AE1B5FD5717F7FF1F23099D
:106FE000F79875BD17A50100130545FA97700100C4
:106FF000E780E06C97F7FF1F938747AAA69703C423
:107000000700814917FAFF1F130A8A8A1374F40FC5
:1070100097AA0100938A0AF863C7890429459770E3
:107020000100E780C056854717F7FF1FA300F788C8
:1070300017F7FF1F230D878617F7FF1F2306F79407
:1070400037E700E0B70640002320D7180100010011
:10705000378600408347A60293F7370F2305F602D1
:107060002320D7102DBDB3073A0183C507005685ED
:10707000850997700100E780A04C79BF854717F715
:10708000FF1F2305F78221BD17A50100130505F099
:1070900097700100E780A06297F7FF1F938707A012
:1070A000A69703C40700814917EAFF1F130A0A7451
:1070B0001374F40F97AA0100938ACAED63C589047B
:1070C000294597700100E780804C854717E7FF1F2F
:1070D000A30CF77017E7FF1F2309877017F7FF1F2F
:1070E0002304F78A37E700E0B70640002320D718CB
:1070F00001000100378600408347660293F7370F8F
:107100002303F602B1BFB3073A0183C507005685D2
:10711000850997700100E780A0424DB7854717E7C2
:10712000FF1F2303F76CA5BB9307400A638DF5345B
:107130009307200B6388F5369307100AE396F5E86A
:1071400083072A00014463D1074297E7FF1F83C7E3
:10715000D75D93F63700638E061A0546638EC62206
:1071600009466399C61A1D4775A217E5FF1F034517
:10717000C55BC94717EAFF1F034A3A5B97E5FF1F44
:1071800083C5C55A17E4FF1F0344545A6319F51009
:10719000CD476316FA1093077008639CF502130736
:1071A000300FB7170E006308E4001307900DB7B750
:1071B00004006314E40817E7FF1F2323F77CBE8550
:1071C00017A50100130585DD97700100E7804037A2
:1071D000E5BB93078008639DF50033048040B777D3
:1071E00046001374F40F938787CDB3D78702E1B7B6
:1071F00093079008639AF5003304804091671374F5
:10720000F40F9387C766D5B79307A008639BF50073
:1072100033048040B7173D001374F40F9387079031
:10722000E9B79307B008639AF5003304804091678B
:107230001374F40F938797D04DBF93F5F5078D47DF
:10724000639BF50033048040B7975B001374F40F21
:10725000938707D859BF8947639BF5003304804063
:10726000B7770B001374F40F9387071BBDBF8547D7
:10727000639AF50033048040DD671374F40F93873D
:1072800067E3A5B789E9330480408D671374F40F71
:10729000938777DC99BFF1679387072029BF970011
:1072A0000000E78040A0A285528597000000E7809B
:1072B000809F19BB9305610017E5FF1F0345E54655
:1072C00017E4FF1F0344744697000000E78040AEB8
:1072D00093057100228597000000E78060AD3C00B7
:1072E00017E7FF1F2328F77A834761002304F10083
:1072F00083477100A304F100894717E7FF1F230BA1
:10730000F7668357810017E7FF1F231FF7400944E3
:10731000A1AC154793F64700B336D00093F7870327
:10732000850685C32146638BC7066146638AC70607
:10733000130680026388C706130680036393C700A1
:10734000914717E6FF1F230FD66297E6FF1FA38B17
:10735000F66297E7FF1F2388E76217E7FF1F0347DF
:10736000E73C9376070497E7FF1F83C7373C8DEE12
:107370001377770C93067008630CD7021377F7071F
:107380008D46631ED70AB307F040B7955B0093F7AD
:10739000F70F938505D881A81947ADBF854755B725
:1073A000894745B78D4771BF930670086311D702AF
:1073B0001307300FB7150E006389E7021307900D0E
:1073C000B7B504006383E7021307700845BF93064F
:1073D000800C6311D702B307F040B775460093F7EE
:1073E000F70F938585CDB3D5F50297E7FF1F23A946
:1073F000B758F9B39306900C631AD700B307F0405F
:10740000916593F7F70F9385C566F1BF9306A00CBE
:10741000631BD700B307F040B7153D0093F7F70F94
:1074200093850590C9B79306B00CE319D7F4B30759
:10743000F040916593F7F70F938595D06DB7894626
:10744000631BD700B307F040B7750B0093F7F70F36
:107450009385051B49BF8546631AD700B307F040E3
:10746000DD6593F7F70F938565E3B5BF09EBB307C8
:10747000F0408D6593F7F70F938575DCADB7F16537
:10748000938505209DB783472A00C18B99C78547FF
:1074900017E7FF1F2303F74E05BE97E7FF1F238E55
:1074A000074C1DB6854717E7FF1FA30EF74C29BEF3
:1074B0003C0017E7FF1F232FF75C094793070003E2
:1074C0002314F10097E6FF1F2386E64A2DBD639A39
:1074D0000758A94763ECB74417A70100130747945F
:1074E0008A05BA959C41BA97828717E4FF1F034427
:1074F000D423094A630C440F636C8A0885476309E7
:10750000F40A9307F00F17E7FF1F0347A74663F638
:10751000E70017E7FF1F230FF74417EAFF1F034A8F
:107520006A45930700041374FA0F63F447011304C8
:10753000000497E7FF1F9387E75583AA0700228679
:1075400017E5FF1F1305451ED685330A8A40A29A08
:1075500097700100E78060F397E7FF1F238C474196
:1075600097E7FF1F23A8575397E7FF1F83C797404D
:107570001547639AE762B7E700E03707400023A0AA
:10758000E71801000100B7860040238086028DA520
:107590008D47630CF40A9947E315F4F697A70100A9
:1075A0009387878E17E7FF1F2326F74EA947A1BFB2
:1075B00017E7FF1F0347274F97E7FF1F9387873D75
:1075C000494697A50100938525956306870097A5F1
:1075D0000100938565903E8597700100E780E0EAA1
:1075E00017E7FF1F2328A74AC94731BF97E6FF1FA8
:1075F00083C6664B054797E7FF1F9387A7396394B8
:10760000E6023E851306700297A501009385458E1C
:1076100097700100E78060E717E7FF1F232CA7465C
:1076200093077002CDB53E851306300497A501007F
:107630009385458697700100E78020E517E7FF1FD7
:10764000232AA744930730047DBD97E5FF1F83C518
:10765000C50D17A501001305A59597700100E780DA
:1076600020EE854A17EBFF1F034BEB4397E5FF1F07
:1076700083C5A50B17A501001305859363185B0B44
:1076800097700100E780C0EB97E7FF1F83C7E7090A
:10769000B5CBE368F4E617A401001304248C638CD3
:1076A000670117A401001304E48B6386470117A444
:1076B00001001304A48C228597700100E780E00884
:1076C0001375F50F93071500860717E7FF1F2303B0
:1076D000F72C8D4717E7FF1FA30EF72A97E7FF1F29
:1076E0009387472B0147BE861376F70F890763659B
:1076F000A60297E7FF1F23AFD73897E7FF1F83C77F
:10770000672911B5979701009387477E17E7FF1FF9
:107710002322F7389147C5BB3306E4000346060031
:10772000A380070005072380C7007DBF9770010075
:10773000E78000E197E7FF1F83C727FFE1D7E362F8
:10774000F4DC179401001304647E638C57011794D2
:1077500001001304247E638647011794010013047B
:10776000E47E228597700100E78020FE1375F50FF7
:1077700093071500860717E7FF1F230DF7208D4796
:1077800017E7FF1FA308F72097E7FF1F93878720BE
:107790000147BE861376F70F8907E37CA6F433060C
:1077A000E40003460600A380070005072380C70006
:1077B000D5B797E5FF1F83C545F71795010013055A
:1077C000E57F97700100E780A0D797E7FF1F83C789
:1077D000371C93E7470017E7FF1FA30BF71A8347F0
:1077E0002A0017E7FF1FA303F71A6FF0EFFD1795A5
:1077F00001001305E57D97700100E78040EC97E7F5
:10780000FF1F9387A71883C7070017E7FF1F230DE4
:10781000F7F017E4FF1F0344E41533348000A9B3E5
:10782000179501001305057C97700100E78020E99A
:1078300097E7FF1F83C7D71593E7070117E7FF1FD8
:10784000A308F71483472A0017E7FF1F2300F71444
:107850006FF08FF7179501001305057A97700100F7
:10786000E780E0E503470A007D8B51EFB7870040D2
:1078700003C767021377C70B136727002383E70249
:1078800003C7A7021377C70B136727002385E702F7
:1078900003C7E7021377C70B136727002387E702A5
:1078A00003C727031377C70B136727002389E70252
:1078B000854717E7FF1F2309F7F217E7FF1F230785
:1078C000F7FE17E7FF1F2305F70A17E7FF1F23023D
:1078D000F70A97E7FF1FA38907F097E7FF1FA38722
:1078E00007FC97E7FF1FA385070897E7FF1FA38201
:1078F000070897E7FF1FA389070897E7FF1FA384DF
:10790000071A6FF06FEC89476312F70297E7FF1FC2
:1079100083C7C7E19146638CD70863E0F604638EA2
:10792000E70C6369F70A05476380E70EFD5717E721
:10793000FF1FA301F70437074000B7E700E023A0CB
:10794000E71801000100B78600401306F0FC238110
:10795000C60223A0E7106FF08FD4130720086382BC
:10796000E7086362F70213071008E391E7FC378723
:1079700000408347670293F7C70B93E72700230371
:10798000F7026FF06FE4130730086389E70213070B
:107990004008E39DE7F8378700408347270393F7C4
:1079A000C70B93E727002309F7026FF0EFE1378752
:1079B00000408347270393F73707F5B73787004021
:1079C0008347E70293F7C70B93E727002307F702E4
:1079D0006FF08FDF378700408347E70293F7370761
:1079E000F5B7378700408347A70293F7C70B93E7A4
:1079F00027002305F7026FF02FDD3787004083470C
:107A0000A70293F73707F5B7378700408347670228
:107A100093F73707ADB7179501001305E55E97702B
:107A20000100E780C0C997E7FF1F238F07CED5B3BA
:107A3000179501001305455E97700100E78020C887
:107A400097E7FF1F239207CE97E7FF1F938787F2E1
:107A500003C40700894763F3870009441374F40FD4
:107A600021B613070002E393E7EC6399090A638FD9
:107A7000F500930720026381F508179501001305AF
:107A8000255D97700100E780A0AB4DB5179501000B
:107A90001305455997700100E78060C20144179BA8
:107AA0000100130B6B59A14AB3078A0083C5070075
:107AB0005A85050497700100E78080A8E31654FFFB
:107AC00017950100130505BC97700100E78020BFE2
:107AD00017E4FF1F034484C511E497E7FF1F2388C1
:107AE00007C259B48947E313F4E4854717E7FF1F3A
:107AF000230FF7C06FF04FCD17E6FF1F0346F6C206
:107B000097E5FF1F83C565C217950100130545530F
:107B100097700100E780C0A26FF00FCB638FF50470
:107B200093071002E39BF5F497E5FF1F83C505C09B
:107B3000179501001305C55297700100E78040A01A
:107B400097E7FF1F23A847F597E7FF1F938747E3B2
:107B5000944383D7470017E7FF1F0347C7E217E6A1
:107B6000FF1F2323D6BC1D4497E6FF1F2390F6BCBE
:107B700097E7FF1F238DE7BAC5BA97E5FF1F83C5B7
:107B8000E5BA179501001305254F97700100E780AE
:107B9000209B97E7FF1F238C07B697E7FF1F2395CE
:107BA00007B86FF0CFF62547E387E79C1947639145
:107BB000E702B786004023808602B7E700E0370778
:107BC000400023A0E71801000100130600FC41B3A8
:107BD0001307100A6391E702B786004023808602EC
:107BE000B7E700E03707400023A0E71801000100D5
:107BF000130680FCA9BB1307A009E38FE7FC13075A
:107C0000400AE38BE7FC13072002E386E79605476B
:107C1000E383E796B7E700E03707400023A0E718C3
:107C2000E391099601000100B78600402380860297
:107C3000130620FC29BB17E7FF1F0347B7D36308D0
:107C4000F71E63E7E7029547630EF70E994763084F
:107C5000F704B786004023800602B7E700E0370745
:107C6000400023A0E718010001001306A0FCC5B1E5
:107C70009307F005630AF700930750096306F700BE
:107C800093071002E317F7FCB7E700E0370740005F
:107C900023A0E71801000100B786004051BF97E913
:107CA000FF1F83C929CD93070004CE8A63F43701EF
:107CB000930A000497E7FF1F9387C7DD03AA070015
:107CC00013F4FA0F2286D28517E5FF1F1305C5A509
:107CD00097600100E780607BB3878940529417E783
:107CE000FF1F2309F7C897E7FF1F23A587DA638ED5
:107CF0000902B787004023805703B7E600E0370644
:107D0000400023A0C6180100010003C72702134743
:107D100007042381E70203C727021377C70F2381D4
:107D2000E70223A0C6106FF08F97B786004023802C
:107D30000602B7E700E03707400023A0E71801007C
:107D40000100FDB5378700408347370097E6FF1FE6
:107D500083C6D6C393F70708D58FA301F700B706EC
:107D60004000B7E700E023A0D71801000100130688
:107D7000A0FC2301C70223A0D7106FF04F9297E712
:107D8000FF1F9387A7D1A69783C7070093F7F70F25
:107D9000D9CF97E7FF1F83C707D1D1EB17E7FF1FA5
:107DA000034757BD930700026313F70897E7FF1FC8
:107DB0009387879703AB070097EAFF1F83CA0A9749
:107DC00017EAFF1F034A9A9697E9FF1F83C929966E
:107DD000D2875687CE865A8697E5FF1F83C525939F
:107DE000179501001305C52A97600100E7804075CB
:107DF00097E7FF1F23A667B997E7FF1F238457B9AB
:107E000097E7FF1FA38047B997E7FF1F238D37B779
:107E100097E7FF1FA38C878EB7E700E03707400086
:107E200023A0E71801000100B7860040D1B3B7E7EF
:107E300000E03707400023A0E71801000100B786E3
:107E4000004025B529472381E70209472383E7023C
:107E50002385E7022387E7022389E7026FF08F88F3
:107E600003C76700118B6302078A83C75700918B92
:107E7000B5CF17E7FF1F034707C385476313F7060F
:107E800097E7FF1FA381E7B097E7FF1F238E0794B3
:107E900097E7FF1F238C07A097E7FF1F238A07ACF4
:107EA00097E7FF1F238707AC97E7FF1FA38E079273
:107EB00097E7FF1FA38C079E97E7FF1FA38A07AAD8
:107EC00097E7FF1FA38707AA97E7FF1FA38E07AABD
:107ED00097E7FF1FA38907BCB787004011476FF0E2
:107EE0008F8217E7FF1FA303F78279BF854717E744
:107EF000FF1F230BF78E17E7FF1F2309F79A17E7DA
:107F0000FF1F2307F7A617E7FF1F2304F7A669BF84
:107F1000854717E7FF1F2309F78C17E7FF1F230784
:107F2000F79817E7FF1F2305F7A417E7FF1F2302A2
:107F3000F7A417E7FF1FA309078A17E7FF1FA30787
:107F4000079617E7FF1FA30507A297E7FF1FA38266
:107F500007A28280411106C697000000E78080FBDF
:107F6000B787004023800700130740FC2386E70003
:107F70001307C004A386E70017D7FF1F1307C77AAC
:107F80002398E70017D7FF1F1307077E239AE70000
:107F900017E7FF1F13078789239CE70017E7FF1FD9
:107FA00013070795239EE70029472381E702094726
:107FB0002383E7022385E7022387E7022389E70279
:107FC000A3810700930600F8A380D70093069002D0
:107FD0002380D700FD562383D7002381E700B7060F
:107FE000400037E700E02320D71003C717001367CE
:107FF0001700A380E700B24097E7FF1F2398079878
:1080000041018280411106C697000000E78080F0A0
:10801000B787004023800700130700FC2386E70092
:108020003147A386E70017D7FF1F1307E76F239891
:10803000E70017D7FF1F13072773239AE70017D707
:10804000FF1F1307A77E239CE70029472381E70230
:1080500009472383E7022385E702A38107009306EC
:1080600000F8A380D700930690022380D700FD5626
:108070002383D7002381E700B706400037E700E0FD
:108080002320D71003C7170013671700A380E7004A
:10809000B24097E7FF1F239B078E41018280B7877D
:1080A00003009387074017E7FF1F232BF78C8547B3
:1080B00017E7FF1F2318F78CA14717E7FF1F2304BB
:1080C000F78C97E7FF1FA380078C97E7FF1F238D8F
:1080D000078A97D7FF1F238C076297D7FF1FA387B5
:1080E0000762814717D5FF1F13058562FD5517D617
:1080F000FF1F1306A6622947B306F5002380B600CA
:10810000B306F600238006008507E397E7FE97E7AE
:10811000FF1F2383079897E7FF1FA38F079697E713
:10812000FF1F238C079697E7FF1FA386078497E717
:10813000FF1FA384078497E7FF1F238F078297E71A
:10814000FF1F238A078297E7FF1F2389078297E78C
:10815000FF1FA383078297E7FF1F2380078297E70C
:10816000FF1FA38C0792828017E7FF1F0347A79387
:1081700085476316F700170300006700E3E817035D
:108180000000670063DD411122C406C617E7FF1F28
:108190000347679185472E8613F4F50FAA85631769
:1081A000F70417D5FF1F1305656C97600100E78082
:1081B000C02D97D7FF1F238B076EB78700402384FE
:1081C0008702B7E600E03706400023A0C61801008A
:1081D000010003C7A7021377C70F2385E702B24048
:1081E000224423A0C61001454101828017D5FF1FFC
:1081F0001305855B97600100E780202997D7FF1F53
:108200002384075EB787004023828702B7E600E039
:108210003706400023A0C6180100010003C767020B
:108220001377C70F2383E7025DBF411106C697008E
:108230000000E78000E7B24041011703000067003B
:10824000E3F2411106C697F0FFFFE780C0BD97D764
:10825000FF1F83C7775995C797D5FF1F83C5E5587B
:1082600089C917D5FF1F1305655897F0FFFFE780F1
:10827000209C97D7FF1FA389075697D7FF1F2385F9
:108280000770B2404101828041C9D9C597D7FF1F0D
:1082900083C7C76FD1C3011122CC4AC84EC656C28C
:1082A0005AC006CE26CA52C42E89AA890144930A0E
:1082B0000004371B030063772403B3078940C20718
:1082C000C183BE8463F4FA0093040004C204C18035
:1082D000130A1BD497D7FF1F83C707519DE37D1A4D
:1082E000631C0A00F2406244D2444249B249224A25
:1082F000924A024B0561828097F0FFFFE780A0B2AF
:10830000D1BF338589002694A685420497000000DA
:10831000E780A0E7418045B7828097D7FF1F93870A
:10832000277C18429C4383D645000345070083C53C
:10833000C700035646006396A50083D5E700638D0A
:10834000D502011106CE2386A7002397D700B705D3
:10835000CF00DC4B9385757D05077D162EC223006B
:1083600001003AC42316C1002317D10099C30A851E
:108370008297F240056182808280DC4DDC4B81CFA8
:10838000B7E70400904503A38705914517D5FF1F64
:1083900003454575028382806D713C083EC6B70770
:1083A000E500232291103EC8AA843C08328523268A
:1083B00011103ECA23248110232021112E899730C9
:1083C0000000E78040622A84979501009385C5CF1D
:1083D00017850100130545C497600100E78040162A
:1083E000A285179501001305A5DE97600100E780BF
:1083F0002015294597600100E7806019B705CB007B
:108400009385757D680097100000E780606BA285FA
:10841000680097300000E780604F01478146700098
:10842000CA85268597200000E780E08E05CD2A8446
:1084300097950100938545C9178501001305C5BDB2
:1084400097600100E780C00FA28517950100130512
:10845000E5D897600100E780A00E294597600100EC
:10846000E780E0128320C11003248110832441108F
:10847000032901105161828097D7FF1F93874766B8
:1084800018429C43797122D406D60348070083C85A
:1084900007012A8483D645000355460063960801E8
:1084A00083D82701638DD802238807010507239904
:1084B000D7003708CC00DC4B1308787D3ACC130783
:1084C000F5FF42CA23080100231EE100231FD1004B
:1084D00099C7080832C62EC482973246A245228523
:1084E00097000000E78080EBB25022544561828003
:1084F0006D713C083EC0B707E5003EC23C083EC473
:108500002326111023248110232291102317010008
:108510002318010023190100231A0100231B010065
:1085200097B7FF1F83D707EA99E3C167FD172316A3
:10853000F10097B7FF1F83D707E991EB97D7FF1F8C
:108540009387075A9C439C43DC4783D7070017B4A3
:10855000FF1F130424E7584C2317F10083574400EE
:10856000484B2318F10031E1979501009385C5BC74
:1085700017850100130545AA97600100E78040FCBC
:1085800017950100130585BC97600100E78040FB4B
:10859000294597600100E78080FF8320C1100324F4
:1085A0008110832441105161828097B7FF1F83C7D8
:1085B000D7E189EBB7E70400BC5782975C4C23AA4C
:1085C0000700E1BFFD1797B6FF1FA380F6E0035633
:1085D0000701834704014C470A85230BF1009730BC
:1085E0000000E780C02F97D7FF1F9387674F9C43FA
:1085F0000147814688430A866C0097100000E78097
:108600008071AA8429C1979501009385E5B21785E9
:108610000100130565A097600100E78060F2A68560
:1086200017950100130545B397600100E78040F1FD
:10863000294597600100E78080F5584CB7E70400B2
:10864000BC57484B9DBF97B7FF1F83C717D8F5D7B7
:10865000B7E70400BC4F1044854517D5FF1F0345FD
:10866000654882971DBF5C4EDC4BB9CFB1CD41113F
:1086700022C4178501001305259A2E8497950100C1
:108680009385C5A906C697600100E78060EBA285C7
:1086900017950100130505AF97600100E78040EAD8
:1086A000294597600100E78080EEB7E70400224487
:1086B000B24003A3870517D5FF1F0345A542130644
:1086C00040069145410102838280411122C417B4C2
:1086D000FF1F1304E4CC1C4C06C689C7DC4399C3B6
:1086E0004C488297584CB7E70400BC57484B8297D8
:1086F0005C4CB240224423AA07004101828017B794
:10870000FF1F1307E7CB834707009306F00B85078E
:1087100093F7F70F63E9F60097B6FF1F2382F6CAB7
:10872000034507008280930700F8FDB78357450093
:108730006386071001114AC817B9FF1F130989C8BA
:1087400052C4032AC90106CE22CC03274A0126CAF5
:108750004EC656C2F15735E31307D00DFD57636E71
:10876000C704B7E9040083A709072A841305860014
:1087700042054181B284AE8A8297232AAA0003254A
:10878000C9015C49A9E7979501009385259717854D
:1087900001001305658897600100E78060DA17958E
:1087A0000100130565A697600100E78060D929459F
:1087B00097600100E780A0DDDD57F2406244D244BB
:1087C0004249B249224A924A3E8505618280938796
:1087D0004400B705CF002319F5009385757D310559
:1087E00097100000E780C02D0325C9018345640070
:1087F000310597300000E78060110325C901268606
:10880000D685310597300000E780600D7146A2855E
:108810004A8597600100E78040C7504419CA83A782
:108820008905854517D5FF1F0345C52B82978147CD
:1088300069B797000000E780E0CBD5BFFD573E85C4
:108840008280411126C297B4FF1F9384A4B7D84CED
:1088500022C437E404003C54484B06C68297DC4CE3
:108860000323C4052244B240924423AA070017D52B
:10887000FF1F03452527854541010283411126C27B
:1088800097D4FF1F9384C4259C4006C622C44AC0C7
:10889000D5C3DC43C5C35CC12300B5002A849795CA
:1088A00001009385E580177501001305E576976053
:1088B0000100E780E0C8294597600100E78020CDEE
:1088C0009C4023A4070023A2070097B7FF1F9387AC
:1088D00027ADDC4FDC4B91C7295597000000E7809E
:1088E00000DF97B7FF1F9387E7ADDC4FDC4B89C7ED
:1088F00097000000E78020F537E904008327C905C9
:10890000894517D5FF1F0345E51D82978327C905B4
:10891000914517D5FF1F0345E51C82979C4003A393
:1089200047016309030022852244B2409244024970
:1089300041010283B24022449244024941018280B3
:108940000111328506CE22CC26CA2E849730000033
:10895000E7806009AA84978501009385A57817753B
:1089600001001305656B97600100E78060BD030798
:1089700084000356640083554400A68617950100C1
:108980001305458297600100E78080BB2945976009
:108990000100E780C0BF97B7FF1F83C7C7A0639DD3
:1089A0009700014597000000E78060D281450A8565
:1089B00097000000E780C0ECF2406244D2440561B9
:1089C00082806D712324811023261110232291109F
:1089D00093F745002E84638707143C083EC0B70711
:1089E000E5003EC23C083EC42317010023180100E5
:1089F00023190100231A0100231B010097B7FF1F51
:108A000083D7079A99E3C167FD172316F10097B73B
:108A1000FF1F83D7079991EB97D7FF1F9387470CC9
:108A20009C439C43DC4783D7070017B7FF1F1307FE
:108A300027972317F100544F835747002318F1005D
:108A4000DC4AA1E7978501009385056E1775010043
:108A50001305855C97600100E78080AE17850100F3
:108A60001305C56E97600100E78080AD29459760CA
:108A70000100E780C0B1134544008320C1100324E6
:108A80008110832441105161828097B7FF1F83C7F3
:108A900097912555D9C3FD1717B6FF1FA305F6906B
:108AA00003D6060183470701CC460A85230BF10054
:108AB00097300000E780A0E297D7FF1F9387470217
:108AC0009C4317B7FF1F1307A78D97860100938656
:108AD000E66A88430A866C0097100000E780A023AE
:108AE000AA8451D997850100938505641775010003
:108AF0001305855297600100E78080A4A68517853D
:108B000001001305656597600100E78060A32945B2
:108B100097600100E780A0A7268597000000E78006
:108B200000BB91BF93F725009DC7B7E70400BC4782
:108B30004146814528088297255597000000E78027
:108B400000B928089305F00F97000000E78040D394
:108B5000134524001DB793F71500014599DF9700D1
:108B60000000E78020991345140001BF5C4D4111BE
:108B700006C688C317D7FF1F2324F7F6B7E70400FC
:108B800083A70708170500001305E5E38297B240A5
:108B900097D7FF1F2388A7F4014541018280011167
:108BA0003335A000A307A100B7E7040083A7471748
:108BB00006CE1306F1008545130550308297F2402A
:108BC000056182808280411122C406C697D7FF1FAB
:108BD00083C7C7F2014489EF97B7FF1F83C7976028
:108BE000054499E717D4FF1F034404A0134414005D
:108BF000228597000000E780C0FA17850100130561
:108C0000656C09E4178501001305C56C2244B24068
:108C10004101176301006700A392797122D4A30F69
:108C2000010037E404008327841726D24AD006D6F1
:108C3000AA842E89130550309305F10132C682971C
:108C400032468347F10193150601C18185CB014569
:108C50002EC697000000E780C0F483274417B24572
:108C60004A8626858297054597000000E78060F3D5
:108C7000B25022549254025945618280832744178E
:108C80004A8626858297EDB741119397050122C444
:108C900006C626C2C1872E8463D40702B7E4040047
:108CA000FC5417A5FF1F0345E574829719C1BC54F6
:108CB00082972165218DB2402244924441018280F5
:108CC00093F715008DC7B7E7040083A7471A17A6C7
:108CD000FF1F1306267197D5FF1F938565E117A522
:108CE000FF1F03452571829713451400E9B793F7D9
:108CF000250099CFB7E70400BC4F130600648945EF
:108D000017A5FF1F0345056F82971345240065B71C
:108D100093F785009DC7B7E7040003A8871A1307D8
:108D2000401F97A7FF1F83C7E76C814613064006C5
:108D3000994517D5FF1F0355A5DC029813458400FC
:108D40009DBF93F745000145BDD7B7E4040083A755
:108D5000041817D5FF1F0355A5DA8297BC4C1306DC
:108D60000064914517A5FF1F0345C5688297134509
:108D7000440091B797D7FF1F83D787D86398A7027E
:108D800017D7FF1F231FB7D617D7FF1F231CC7D620
:108D900017D7FF1F2319D7D62E8617850100130575
:108DA000A558BE8517530100670083791785010018
:108DB00013050559176301006700639003574500C9
:108DC00097D7FF1F83D7C7D3631AF704C167411131
:108DD000F91722C417D7FF1F2324F7D237E4040062
:108DE00097D7FF1F23A007D297D7FF1FA38807D0CD
:108DF0007C4C06C6894517A5FF1F0345A55F8297D2
:108E00007C4C914517A5FF1F0345C55E8297224400
:108E1000B240410117030000670023DB1785010002
:108E20001305055217630100670063897D15954797
:108E300063E2A71C17870100130787460A053A95C6
:108E40001C41011122CC06CEBA972E848287178549
:108E500001001305654F97600100E7804086A1A2DD
:108E600003C7250099476311F7022E85970000007C
:108E7000E78000F583456400178501001305C54DA3
:108E800097500100E780C06B97B7FF1F238C073412
:108E9000178501001305054E7DBF03C725009547C3
:108EA0006319F702C16717D7FF1F035767C5F91783
:108EB00003D5A5006309F702B7E7040083A7C71726
:108EC0008297178501001305E54B97500100E78055
:108ED000007F854717B7FF1F2306F730178501006E
:108EE0001305C54C8DBF97D7FF1F239BA7C083D702
:108EF000E50097D6FF1F2396F6C083D7050197D6C6
:108F0000FF1F2391F6C083D7250197D6FF1F239C0F
:108F1000F6BE97D7FF1FA38307BE631BE502B7E723
:108F20000400BC4F096613060690A14517A5FF1F54
:108F30000345454C82970356E4008355A4001785EA
:108F400001001305654597500100E780605F51B748
:108F50009307700F2316F100B7E7040083A7870D6E
:108F600017A6FF1F034606496C0082974DF98547F7
:108F700017D7FF1FA304F7B85DB7178501001305C6
:108F8000A543D1BD83C5250091476392F50217859E
:108F900001001305E54397500100E78040729700F8
:108FA0000000E78080C2F2406244056182809947F8
:108FB0006392F502228597000000E78060E0834518
:108FC0006400178501001305253997500100E780DB
:108FD0002057D1BF9547639AF50083471400E1F30A
:108FE0001785010013050541BDB51785010013055F
:108FF000E540E1BF82806D7123248110232611108A
:1090000023229110328401CD8947630AF50283201F
:10901000C11003248110832441105161828017857F
:1090200001001305653EAE8497500100E78020697A
:10903000A285268597C0FFFFE7804054C9BFB7E7E8
:109040000400FC4728008297178501001305853C22
:1090500097500100E780A0668347810039C4130759
:10906000000B6380E7021387A7051377F70F8D4680
:1090700063EDE602A285280097D0FFFFE78020C3BA
:1090800079B78547E3F587F88345910017750100A7
:109090001305C52DB335B00097B7FF1F2386B7FC66
:1090A00097500100E780C0499DB703479100A20790
:1090B000D98F35671307D7556385E7086368F702CB
:1090C0002D671307B7556387E70631671307C75541
:1090D000638AE70429671307A7556394E702A2850B
:1090E000280097D0FFFFE78060F615B73967930631
:1090F000E765638ED71263E9F6001307E7556381CE
:10910000E712A28528003DB73D679306F7556387B0
:10911000D7121307F766E396E7FE97D0FFFFE780C5
:10912000E00EF5B50146A285280097D0FFFFE78045
:1091300020DFF1BDA285280097D0FFFFE78040EF38
:10914000F9B58947E3F587EC7914420441803C0086
:109150008144294783C627008504C204C1806386F1
:10916000E6008507E3E884FEA28497D7FF1F83D734
:10917000A7A1639097069307000863E0970637E47A
:1091800004005C5C26869305A10017D5FF1F13051C
:10919000A59782978547631EF5007C5C829797D7D9
:1091A000FF1F9387A79E9C431D8D9307F002E3F05A
:1091B000A7E6B7E70400FC4726869305A10017D56C
:1091C000FF1F13056594829797D7FF1F239E979AD9
:1091D00029A093070008E3FE97FCB7E70400FC5FB3
:1091E000829797D7FF1F23A3A79AA6851305A100EF
:1091F00097A0FFFFE780C0FBB7170300938717D442
:10920000B7360040FD17E38407E003C75600137725
:1092100007046DDB03C7B6001377F70F65F7C5BB0F
:10922000A285280097D0FFFFE78040E3CDB3A28559
:10923000280097D0FFFFE78000EED1BB97D0FFFF5B
:10924000E78080F6E9B3411122C417A4FF1F13047D
:10925000A41BAA8617860100130606062285C145AF
:1092600006C697500100E780C0460357440097A701
:10927000FF1F9387671A2393E70003576400239423
:10928000E700B240224441018280411106C69700A6
:109290000000E78080FBB7E7040083A7871417A6C8
:1092A000FF1F13066616D54501458297B2404D460D
:1092B00097A5FF1F938545161305703041011703CD
:1092C00000006700C39561712324811A37E404000C
:1092D000832704082326111A2322911A2320211BF5
:1092E000232E3119170500001305459A829717A9F7
:1092F000FF1F13092910994785442300A900231C47
:10930000F10097850100938525FF930740061775A7
:109310000100130565D0231CF1082308910097C9AB
:10932000FF1F9389C93C97500100E780602183D5D6
:10933000090017850100130525FB97500100E78000
:109340002020294597500100E780602403D50900BB
:10935000856997000000E78040EF832744171008D5
:1093600085451305503082978327441717A6FF1FA2
:109370001306860ACD45130570308297832744175C
:1093800017A6FF1F13064607B545130560308297E1
:1093900083274417300889451305103182978327A6
:1093A00044173009894513052031829783274415D6
:1093B000938509C80D45829783274415938509C86D
:1093C00011458297A305910023069100230891007F
:1093D00002CD230C01008327841630099145130523
:1093E00070408297832784161306B10085451305C4
:1093F000004082978327841670008545130510402E
:10940000829783278416300885451305204082976C
:1094100083278416100885451305504082978327BB
:1094200004157D558297832744137D5582977D557A
:1094300097A0FFFFE78020248327440C829797A002
:10944000FFFFE780C0FD8327841417A6FF1F1306C4
:10945000A6FBD5450145829789471306700F8145C4
:1094600028092306F1009790FFFFE78000C78D478A
:109470001306000881452808230CF1089790FFFF88
:10948000E780A0C59147230CF100977701009387EF
:1094900027AA984383C747003AC8230AF10097D008
:1094A000FFFFE78060DD70008545054597A0FFFF61
:1094B000E780802330099305700F094597A0FFFFCF
:1094C000E78080223008930500080D4597A0FFFF34
:1094D000E780802110089545114597A0FFFFE780A0
:1094E000A020C16717C7FF1F13078761F9171CC3A7
:1094F0002322070017A5FF1F130585EF97A0FFFF85
:10950000E780601D8327C41D17C5FF1F1305C55DB8
:1095100082973C4803450900854582978320C11AFC
:109520000324811A8324411A0329011A8329C119AA
:109530005D618280C16717C8FF1F0358685CF91717
:109540006301F8083DCDB5CD011126CAB7E404008A
:1095500083A7841222CC2E862315B10006CE2A843E
:1095600001478146ED45428582972AC611ED178550
:109570000100130565D997500100E7804014F240BF
:109580006244D24405618280FC440356A100A28556
:1095900082972C0017C5FF1F0355855697A0FFFF24
:1095A000E780202069DD17850100130525D7975036
:1095B0000100E780C01083A7C412ED452800829700
:1095C0007DBF8280411106C61DC9854717A7FF1FB1
:1095D000A309F7E2354697A5FF1F9385E5E113053B
:1095E000603097A7FF1F238F07E097F0FFFFE7800A
:1095F0000063B240410117F3FFFF6700035D97A7C7
:10960000FF1FA38007E0F9B7C16717C5FF1F035508
:10961000254FF9176307F500B7E7040003A3C71741
:1096200002838280854717C7FF1F2309F74C014536
:1096300017F3FFFF6700E3561793FFFFE70243A509
:109640002A8408452E89B28919C900C197150000DE
:109650009385A586610597300100E78080018144EC
:109660007D5A97100000E780E03963C7A404814465
:1096700097100000E780003A63C8A40497C7FF1F53
:10968000938707519C43DC47B307F9409187230236
:10969000F400638309048327C900B307F440958766
:1096A000A302F4001C4C89C79C4799C3228582976A
:1096B0001793FFFF670003A15C4413971400850410
:1096C000BA972390470171BF1C4813971400850473
:1096D000BA972390070069BF832789000547B3071E
:1096E000F4409587A302F40083570400638EE702D9
:1096F0008DC309476384E7040D47E395E7FA97872D
:1097000001009387E7231CCC9787010093874724A8
:1097100011A897870100938727EA1CCC978701003F
:10972000938787EA5CC8BDBF978701009387C7D539
:109730001CCC97870100938727D6EDB79787010048
:109740009387C7241CCC9787010093872725D9BF0F
:1097500095E51793FFFFE7024395004618448347BA
:10976000940075839D8B6317F70097100000E780C6
:1097700060B448C41793FFFF670063958280179316
:10978000FFFFE702E39013893500C16442094111EC
:10979000AA890144F11413590901054A2EC69710EC
:1097A0000000E7802026B2456348A400014541013E
:1097B0001793FFFF6700039183A709001317140095
:1097C000BA9783D707006388B700639497006374E0
:1097D0002A010504E1B70545D9BF1793FFFFE7024A
:1097E000438AAA892E89328BB6843A8ABE8A97A088
:1097F0000000E78020FB71C9268597200000E780E4
:1098000020098D4763E7A7007D551793FFFF670089
:10981000C38A83DB440097100000E780A0242A84D9
:1098200097100000E780402593077400314433050A
:10983000850263CDA70297100000E780A022971051
:109840000000E78020222A8497100000E780C022D1
:109850009307740031443305850263C3A70497104E
:109860000000E78020209307450029A897100000FA
:10987000E7808020330585021307F0179307C01790
:10988000E35FA7FA2D55E3C277F963040B02D6868E
:109890005286A6854A8597200100E78020BAB5B791
:1098A00097100000E780401D330585029307C5FF30
:1098B000D1BF832749001385C90083D527009700AE
:1098C0000000E78000EC61F581B769553DBF97C79F
:1098D000FF1F2391A72C97C7FF1F9387672B9043E8
:1098E00081470C463307F500420741836393B70075
:1098F00082805446139847008507C2962390E6005D
:10990000D5B797C7FF1F9387A7289C4303C5870038
:10991000828017C5FF1F0355E52782801783FFFF4D
:10992000E702A378C1671387D7FF630BE502636A79
:10993000A700F1176300F50201451783FFFF6700D9
:1099400003791387E7FF6302E502FD171D8D1335C9
:109950001500E5B797500000E780C0267D15C5BF0C
:1099600097500000E78040FBD5BF97500000E7808C
:1099700060F9EDB71783FFFFE70223734111AA8453
:1099800001442EC697100000E780C008B245634826
:10999000A400014541011783FFFF670043739C4802
:1099A000131514003E9583570500E385B7FE0504A3
:1099B000C9BF03485500814693F7F60F63E50701D9
:1099C00081473E858280584593975600BA9703D7C2
:1099D00027006316B70003D70700E304C7FE850618
:1099E000E1BF8346450001479377F70F63E4D70053
:1099F000814711A81C45131657000507B29703D6D7
:109A00000700E313B6FE3E8582801783FFFFE7025F
:109A1000236893170501C18797CAFF1F938A4A17C6
:109A2000635BF00883A70A00C0479C470357040004
:109A3000198D420541816368F50001442285178331
:109A4000FFFF6700236812052A94CDBFDC471394FB
:109A50004900014A3E94834744006341FA02014AA7
:109A6000834754006349FA028509C20993D9090161
:109A700083A70A009847E3EBE9FCC1B71C4413191C
:109A80005A00A6853E994A8597000000E780C0EEFF
:109A900005E1050AC9B75C4413195A00A6853E9929
:109AA0004A8597000000E78020ED19E1050A4DBFC7
:109AB000E30C09FA61B7AA8481495DBF1783FFFFF0
:109AC000E702A35E1C452A8481E79307C5001CC5F5
:109AD0001C44231204001CC09307F00F63EDB70071
:109AE00093F5F50F228597200000E78020E2178389
:109AF000FFFF6700C35D93940501C167C18063F9EF
:109B0000F500A685228597200000E78040E5C5B7CF
:109B1000C18193F5F50F228597200000E78000DFD3
:109B2000A685228597200000E78040E0C9B797C747
:109B3000FF1F9387E705884382801C4599C797C715
:109B4000FF1F23A7A704014582807D55828097C708
:109B5000FF1F9387E70398438347450048479207D1
:109B60003E9582801783FFFFE70223546171004511
:109B70001C183EC6B70780013EC81C183ECA835752
:109B8000440002CE02D002CC231EF10083478400A1
:109B90002A8902D22301F1023C083ED402D6970062
:109BA0000000E78000FB835705002316F102975061
:109BB0000000E78060C42307A1025C4003556400F5
:109BC000F18313F717008347F10252055181F99B86
:109BD000D98FA307F10297100100E780807539CD76
:109BE000AA840355050097A00000E78080BC83D7B6
:109BF00004002AD26800231CF10083D72400231D0F
:109C0000F1001C4803D647008C4397200000E780F2
:109C100000CD8347B400CA8617860100130646802C
:109C20008117A305F4006C00481097200100E7801D
:109C3000E0805D611783FFFF670063492155D5BF51
:109C40001C45B1CF03C5A700894613576500630BB8
:109C5000D7028D46630ED70285466300D7021307ED
:109C600040063305E50203C7B700418B15CB83C718
:109C7000B700BD8B3355F54082801375F50313078C
:109C8000803EC5B709671375F50313070771D1BF88
:109C9000372709001375F5031307077CD9B701456A
:109CA00082801783FFFFE702434003A98500630C0E
:109CB00009048347B900AE8493F7070E85C30345B3
:109CC0009900930520030D810505B305B50288446D
:109CD000610597300100E780E0A935A02E85970047
:109CE0000000E78020F62A8419CD97000000E78065
:109CF000605C8325C900B307B54063FA87002E94E2
:109D0000B305A440E9F51783FFFF6700433C854591
:109D10007DBF1783FFFFE70243392A8403D505007F
:109D2000011132C636C43AC22EC002CA02CC02CEDB
:109D300097A00000E780E0A782452ACA22852ECCA2
:109D400097000000E780E0E003570500231EE100D4
:109D500097500000E78040AAA24632469247230F60
:109D6000A10036874C08B286228501469700000084
:109D7000E780E0A605611783FFFF6700433517837F
:109D8000FFFFE702833261711C183EC6B7078001EE
:109D90003EC81C183ECA3C0800453ED4AA8402CCEA
:109DA00002CE02D002D202D697000000E78060DA2D
:109DB0008357050035592316F10297500000E780BC
:109DC000A0A32307A10209C48357440081EB2159B2
:109DD0004A855D611783FFFF6700632F03556400A9
:109DE0005205518197100100E780A0542A8965D15E
:109DF0008347B40093F7070E99C713058401973082
:109E00000100E780609983574400231EF1008347D7
:109E100084002301F1025C4003550900D98313F744
:109E2000070883471102231CA10093F7F707D98F76
:109E3000A300F10283572900231DF1005C40F18348
:109E400013F717008347F102F99BD98FA307F1029B
:109E500097A00000E780E0952AD235D98347940087
:109E60006800139757008347B400FD8BD98FA30573
:109E7000F4001C4803D647008C4397200000E7807D
:109E800000A6A687177701001307875974000546B7
:109E90004C10268597000000E78060942A890DD930
:109EA0008347B400A685FD8BA305F400970000004E
:109EB000E78060DF31BF1783FFFFE702031F8324C2
:109EC00085FE2A844111268597000000E78080D70F
:109ED000834734FF93F7070E8DCB2AC6268597005C
:109EE0000000E78060C809CD834734FFB245FD8B91
:109EF000A309F4FE91C5228597300100E780808791
:109F000041011783FFFF6700831C7DD98327C4FFAE
:109F10002685829775F5834734FF93F7070E91C71F
:109F2000228597300100E7802087032584FE970073
:109F30000000E78000E5E9B71783FFFFE702E313BE
:109F40009C4141112A8903C7070089472E849356F3
:109F500067006380F6040D466388C6049307F00724
:109F60006304F7022E8597200000E780C0A7AA842B
:109F70008149C16B130C490097C7FF1F938747C1E5
:109F80009C43984763E4E90441011783FFFF67009E
:109F9000831203D745008547E3F8E7FE2E85972017
:109FA0000000E780A0A9E1B703D74500E3FEE7FC86
:109FB0002E8597200000E78000A3AA8422859720A1
:109FC0000000E78060A4C204C98C5DB7DC4703557C
:109FD000A900139A49003E9A93170501C187635D52
:109FE000F00083570A006397A70263E7740383278F
:109FF000CA00034D5A002DA0A1672167A98F13073E
:10A00000F7EFE374F7FE6397090097000000E7801D
:10A01000209161FD85098DB783278A00034D4A0091
:10A02000835DA90003576900216A138BC7003AC6F4
:10A03000814A33CA4D01631E5D0197C7FF1F938795
:10A04000A7B59C43E1DBA28662868145268582977F
:10A05000D1B7A1679387F7EF930C4BFF63F24703E8
:10A06000B2455A8597F0FFFFE780A0710DC1032725
:10A070008B00104709CE10436382C4023107D5BF5D
:10A08000EE85668597000000E780008F71F9938662
:10A090001A0093FAF60F130B0B0271BF835644009C
:10A0A0005C43E3E9F6F622853AC697100000E780A4
:10A0B000807DA1679387D7042A8A035D44003247D5
:10A0C00063E897008347D90093E707F8A306F900F0
:10A0D0001C4766852286E2858297C1670844FD1782
:10A0E000337AFA00529508C02312A40125B797C706
:10A0F000FF1F9387E7A99843814715C314478147FA
:10A1000063FFD500939745004C47BE9519C903C717
:10A11000550081476375E600DC451606B2973E851B
:10A12000828003C745008147E37BE6FE16069C4517
:10A13000F5B71783FFFFE702A3F5AA892E8A8144AA
:10A1400097CAFF1F938ACAA483A70A00984763E6A9
:10A15000E4001783FFFF6700E3F6DC471394440035
:10A1600001493E9413BB140083474400634BF9003C
:10A17000014913BB140083475400634FF900850461
:10A18000E1B70844931759005287DA860146A28541
:10A190003E9582990509C9BF4844931759005287D3
:10A1A000DA860546A2853E9582990509E9B71783A7
:10A1B000FFFFE70283EF814517F5FFFF1305054811
:10A1C00097C7FF1F2398079C97000000E780A0F621
:10A1D0001783FFFF6700A3EF97C7FF1F9387479B76
:10A1E0009C4395C31783FFFFE70223EC814517F5D6
:10A1F000FFFF1305A54497000000E780C0F3178315
:10A20000FFFF6700C3EC82801783FFFFE70243E88C
:10A2100037E404008327841241112315E100AE893D
:10A220003289368A3A8681460147ED45AA8482976B
:10A230002AC621C90356A100D28597400100E780B4
:10A24000C0248327C413CE8526858297058905C936
:10A250008327440D2314210101462C002685829773
:10A260002A8401C9B7E7040083A7C712ED45280077
:10A270008297228541011783FFFF6700A3E44944C9
:10A28000D5B76554FDB75C41FD175CC1828017836B
:10A29000FFFFE70283E1B7E70400FC5F8297954781
:10A2A0003305F50281450D811783FFFF670023E227
:10A2B0001783FFFFE70263DFB7E70400FC5F8297C5
:10A2C00095473305F5020D811783FFFF670023E0F3
:10A2D0001783FFFFE70263DDB7E7040083A7870B5F
:10A2E0000355050082971783FFFF670043DE17833E
:10A2F000FFFFE70283DB035505003287AE86179622
:10A30000FF1F0356861797C5FF1F93852589970062
:10A310000000E780A0EF1783FFFF670043DB178390
:10A32000FFFFE70283D8B7E7040083A7C717829728
:10A330001783FFFF6700A3D91783FFFFE702E3D668
:10A34000B7E7040083A7871397C5FF1F938505858B
:10A35000829701451783FFFF670063D71783FFFFCD
:10A36000E702A3D4B7E7040083A7C71F8145179569
:10A37000FF1F0355850C82971783FFFF670023D5C6
:10A380001783FFFFE70263D2B7E7040083A78713B1
:10A3900097C5FF1F93858581829701451783FFFF2E
:10A3A0006700E3D21783FFFFE70223D0B7E704007B
:10A3B00083A7C71F81451795FF1F0355050E829779
:10A3C0001783FFFF6700A3D01783FFFFE702E3CDEA
:10A3D0002E8597800000E780E0AF97800000E7803F
:10A3E000E0EC1783FFFF670083CE1783FFFFE702D0
:10A3F000C3CB97800000E780E0F61783FFFF67007C
:10A4000003CD5C49E1175CC95CC583572501A107F1
:10A410002319F50083570501A1072318F500828051
:10A42000F1473305F50297B7FF1F9387277A9C43BF
:10A430003E9582808D476315F60803D74600854711
:10A4400063F0E7081783FFFFE70223C636853684EB
:10A450002E8997100000E780005929C983574400CE
:10A4600093140501C18063E39704228597100000CF
:10A47000E7806057FD14231294009307A002630045
:10A48000F5029307B0026307F50293079002631F7A
:10A49000F500228597000100E780C08501A80146EC
:10A4A000CA85228597A00000E78060B01783FFFF70
:10A4B0006700E3C1228597100000E780C003FDB765
:10A4C000828097B6FF1F9386A6709C42014599CF64
:10A4D0009843D44217B6FF1F232CE66E6396D7002D
:10A4E00097B6FF1F23A8E66E1385C7FE82801783E9
:10A4F000FFFFE70283BB97000000E780A04B714499
:10A5000033058502914597900000E78020E911E529
:10A5100065551783FFFF670083BB97B7FF1F23A510
:10A52000A76A97000000E780E0483305850291455F
:10A5300097900000E78080E661DD97B7FF1F23A7B3
:10A54000A76897000000E780E04697B7FF1F2397B2
:10A55000A76697000000E780E04597B7FF1F2390AC
:10A56000A766977701009387E7F017B7FF1F232BA4
:10A57000F76497070000938707E917B7FF1F2321A8
:10A58000F764014579B71783FFFFE70203B2AA8595
:10A5900017B5FF1F1305856297100000E780C05BA9
:10A5A0001783FFFF6700A3B21783FFFFE702E3AF44
:10A5B00097000000E78060FD97100000E780405B97
:10A5C00097B7FF1F9387C7609C4391CF1387C7FE40
:10A5D00019CB83D5C7FF17B5FF1F1305E55F97207C
:10A5E0000100E78020191783FFFF670043AE178340
:10A5F000FFFFE70283AB97000000E780C0EC09CDC6
:10A60000834785002A8493F7070499EB0355E500F7
:10A6100097000000E78080F91783FFFF670023ABF6
:10A620008347C5009304450117B9FF1F1309495A11
:10A6300085E3832709005CC997B7FF1F23AA9758B2
:10A6400083274900F1FB97B7FF1F23A59758E9B768
:10A65000FD172306F500610597800000E780C0D64E
:10A660008307840063CB07048347840093E707F8DC
:10A670002304F400B7E704009C5F82974205A947D2
:10A6800041813375F5028347840093F707FCC98F36
:10A690002304F4008347D4003E951C402318A400F3
:10A6A00089CF984319CB8347C40050408145850723
:10A6B0003305F502420541810297832709005CC8F2
:10A6C00097B7FF1F23A697508327490089E797B7BD
:10A6D000FF1F23A197508347C4009DDF83550401CA
:10A6E00017B5FF1F1305454F97200100E78080082D
:10A6F00025B71783FFFFE702439B97B7FF1F938799
:10A70000E7729C4701448583858B85E3AE84B285DF
:10A710003A8697100000E780804B2A8419C597106D
:10A720000000E780C041829408CC22851783FFFF98
:10A730006700E3991783FFFFE702839541112E8994
:10A7400032C6AA8997000000E780C031324713065D
:10A750000502CA86970500009385C5CC17B5FF1F73
:10A760001305C54597000000E780E0F82A8425C955
:10A770009304C50097000000E780E0411946AA85D0
:10A78000268597100000E78080158545268597105F
:10A790000000E780601117750100130565CB4E9529
:10A7A00083450500268597100000E78020165C4849
:10A7B00031468145A1075CC85CC483572401E11779
:10A7C0002319F40083570401E1172318F4001C4CEB
:10A7D0003E859780FFFFE7804090A30425012285F6
:10A7E00041011783FFFF6700E38D1783FFFFE70237
:10A7F000C38B4111AA842EC632C497100000E78093
:10A800006036004DB2452246834784000CC050C0DC
:10A8100093F7F70393E707042304F40023180400D5
:10A82000268597100000E780803183479400A94671
:10A830002317A40013D7370005073307D7029D8BD2
:10A8400085072306F400A306E40083C70401D84863
:10A850008507230FF7FE17B7FF1F13076737584306
:10A86000232A04009307440129E317B7FF1F23237A
:10A87000F73617B7FF1F232DF73417B4FF1F130444
:10A88000A435228597200100E78000E11C44858BD8
:10A890005D8D19E58145228597200100E78080EDD7
:10A8A00041011783FFFF670083821CC317B7FF1F97
:10A8B0002322F732D9B71773FFFFE702037F97050B
:10A8C0000000938565B7014597000000E78000B060
:10A8D00001451773FFFF6700837F1773FFFFE702D0
:10A8E000C37C97000000E78080B01773FFFF67000C
:10A8F000037E8347C500A5E31773FFFFE702E37AF2
:10A900002A840355E50097000000E78000C821C1B4
:10A910008347840093F7F7FB2304F4001C4091C79E
:10A92000DC4381C74C400145829797000000E780D7
:10A9300080B917B5FF1F1305252A97200100E7806E
:10A94000A0E50355E40097000000E78020C61773D8
:10A95000FFFF6700C37782801773FFFFE702E3748E
:10A9600097B7FF1F9387C72697050000938565C893
:10A9700017B5FF1F1305452623A0070023A20700D4
:10A9800097200100E780E0CE1773FFFF6700237474
:10A990001C4D91CFDC4381CF1773FFFFE702E370BB
:10A9A0008345070082971773FFFF67004372828019
:10A9B00097B7FF1F938787249C4303C507008280B6
:10A9C00097B7FF1F938787239C4303C51700828097
:10A9D00097B7FF1F938787229C4303C52700828078
:10A9E00097B7FF1F938787219C4303C54700828049
:10A9F00097B7FF1F938787209C4303C5370082804A
:10AA000097B7FF1F9387871F9C4303C5570082801A
:10AA100097B7FF1F9387871E9C4303C567008280FB
:10AA200097B7FF1F9387871D9C4303C577008280DC
:10AA300097B7FF1F9387871C9C4303C587008280BD
:10AA400097B7FF1F9387871B9C4303C5970082809E
:10AA500097B7FF1F9387871A9C4303C5A70082807F
:10AA600097B7FF1F938787199C4303C5B70011E170
:10AA70001D45828097B7FF1F938747189C4303C5E6
:10AA8000C700828097B7FF1F938747179C4303C572
:10AA9000D700828097B7FF1F938747169C4303C553
:10AAA000E700828097B7FF1F938747159C4303D524
:10AAB0000701828097B7FF1F938747149C4303C504
:10AAC0002701828097B7FF1F938747139C4303D5C5
:10AAD0004701828097B7FF1F938747129C4303D596
:10AAE0006701828097B7FF1F938747119C4303D567
:10AAF0008701828097B7FF1F938747109C4303C548
:10AB0000A701828097B7FF1F9387470F9C4303C518
:10AB1000B701828097B7FF1F9387470E9C4303C5F9
:10AB2000C701828097B7FF1F9387470D9C4303C5DA
:10AB3000D701828097B7FF1F9387470C9C438857A4
:10AB4000828097B7FF1F9387670B9C4303D5C7028B
:10AB5000828097B7FF1F9387670A9C4303D5E7025C
:10AB600019E11305800C828097B7FF1F93870709AF
:10AB70009C4303C50703828097B7FF1F938707088D
:10AB80009C43C85B828097B7FF1F9387A7068843C3
:10AB9000828097B7FF1F938727068843828019E139
:10ABA0007D558280F5DE984265DFFDD917B7FF1F1E
:10ABB0001307C7271847AA877155058B631D0724FC
:10ABC00003C507001547E37DA7FC03C7370013053E
:10ABD000F0057D171377F70FE364E5FC03C3570017
:10ABE000E30003FC83C86700E38C08FA03C777001F
:10ABF000494579171377F70FE364E5FA03C7A70010
:10AC000011481305F7FF1375F50FE36BA8F803CE92
:10AC100097000D481305FEFF1375F50FE362A8F8C2
:10AC200003C8B7006309080065181378F80F130507
:10AC3000600DE36705F703C5C700794879151375FB
:10AC4000F50FE36FA8F403C8D7000D457D181378FE
:10AC5000F80FE36705F503D80701930E4017511865
:10AC6000420813580801E3ED0EF303C8E7007D180E
:10AC70001378F80FE36605F303C827017D181378EE
:10AC8000F80FE36F05F103C88700C54E75181378F8
:10AC9000F80FE3E70EF103D86701856E938EBEE0EF
:10ACA0006D18420813580801E3EC0EEF03D8470172
:10ACB0006D18420813580801E3E40EEF03D887012A
:10ACC0007918420813580801E36C05ED03C8A70181
:10ACD0007D181378F80FE36505ED03C5B7011D482E
:10ACE0007D151375F50FE36DA8EA03C5D70171480B
:10ACF00079151375F50FE365A8EA03D5E701130885
:10AD0000E00F7D1542054181E36CA8E803C5070209
:10AD1000494879151375F50FE364A8E8C85301C9CC
:10AD200037C834005915130858BFE36BA8E603A8C9
:10AD3000870237C53400130555BF5918E36205E78C
:10AD400017B5FF1F232AC5EA03C6050117B5FF1F64
:10AD50002326F5EA0545E375C5E403D82501D04966
:10AD600033760603E31E06E203C61501E30A06E294
:10AD700017B6FF1F2320B6E883C527000146638767
:10AD8000A50003C61700F1453306B60283C70703C3
:10AD90009305C00272971A071307C70516031A977F
:10ADA00096084697B387B70241553E9732974207B8
:10ADB00041836362E8061773FFFFE702032F3685BE
:10ADC00097800000E780A06897000100E780204896
:10ADD0002A8497A00000E780805A2A9497F0000008
:10ADE000E78060262A9497900000E780A0812A944B
:10ADF00097F0FFFFE780E06F2A9497400000E7801C
:10AE000060932A9497700000E780A09C22951773A6
:10AE1000FFFF6700C32B82801773FFFFE702E32861
:10AE20004111A307A10097A00000E780A0C59305EA
:10AE3000F100170500001305E5B597F0FFFFE78067
:10AE4000802F014541011773FFFF670043281773E7
:10AE5000FFFFE702032317B4FF1F130424FD032899
:10AE6000840079599368180097B4FF1F23A414FD38
:10AE70001378180063100802BA84BE89368B328AB0
:10AE80002E89AA8A97F0FFFFE780E0A77D15269517
:10AE900019E531594A851773FFFF6700032297F0C0
:10AEA000FFFFE78040A67D152695A167E353F5FED9
:10AEB00097B7FF1F9387872E98433E8C814B01CB1A
:10AEC000014597F00000E7802044933B15004A8538
:10AED000DA865686D28597900000E780C04D2A8991
:10AEE00011CD1C44F99B17B7FF1F2325F7F48327C7
:10AEF0000C00CDD3E3800BFA829769BF268597B704
:10AF0000FF1F23A707F297F0FFFFE780809C4146D1
:10AF1000CE8517B5FF1F1305E5FA97300100E780CE
:10AF2000C05697D00000E78040990325040B97D0C6
:10AF30000000E780009D054597D00000E78000A451
:10AF4000054597000000E78060EDA9B797B7FF1FA0
:10AF50009387C7ED9C47858BEDC71773FFFFE7020B
:10AF6000C31417B5FF1F130525F497B7FF1F23AFB1
:10AF700007EA97B7FF1F23AD07EA97B7FF1F23AB79
:10AF800007EA97200100E780208197500000E780C2
:10AF9000E0F597100100E780A04C97100100E780D2
:10AFA000A05297B7FF1F9387E7E69C4391C70545DB
:10AFB00097800000E780402097B7FF1F938747CF17
:10AFC0009C4399C741657D1597700000E78040A2BA
:10AFD00097F00000E780E03D97D00000E780808F89
:10AFE00097B7FF1F938787F99C4313971701635601
:10AFF000070097F00000E78000AD97B7FF1F23A37D
:10B0000007EC97B7FF1F23A107EC97B7FF1F23AFEC
:10B0100007EA97B7FF1F23AD07EA97000000E78014
:10B02000008C97000000E780007297F0FFFFE78038
:10B03000401897F00000E78040D61773FFFF6700C5
:10B040000309828097B7FF1F938747DE884382807A
:10B050001773FFFFE702630597800000E7806075C4
:10B0600097800000E780C0771773FFFF6700230613
:10B070001773FFFFE702C3012A849304140201112E
:10B080002E85B289A685214636C63A8997300100B9
:10B09000E780403D0DE9B24638082686CE85130587
:10B0A000940497500000E780604121462C084A85AF
:10B0B00097300100E780003B1335150005611773D9
:10B0C000FFFF670023000145D5BF1773FFFFE702AD
:10B0D000C3FD9305450617B5FF1F130565B297100D
:10B0E0000100E78020691773FFFF670043FE1773B5
:10B0F000FFFFE70283FB41112EC697F0FFFFE780B9
:10B10000601BB24588C141011773FFFF670023FC34
:10B110001773FFFFE702C3F7AA842E84978000000D
:10B12000E780006CAA898545228597000000E780AA
:10B13000E07D83C7E4011389940899E3138904032C
:10B14000CE85228597000000E780407C214693054C
:10B150001902228597000000E780607897B7FF1FEB
:10B160009387C7CC8C43228597100000E780C0826C
:10B17000214693858402228597000000E78020768F
:10B180001773FFFF670003F41773FFFFE70263EF16
:10B19000397197F00000E780E0B49305400661E95B
:10B1A00097800000E78000606302051497B7FF1FD7
:10B1B00083C7C7A613B7170097B6FF1F2380E6A65D
:10B1C000014499CFC16417B9FF1F130929C6930918
:10B1D000400EFD1497000000E780C0866342A40A79
:10B1E00097F0FFFFE780000D4169B7290900096A60
:10B1F000FD7A2A8B81447D199389F97B130A0A71A0
:10B20000938A8AC797000000E780C08363D7A404AD
:10B210001304400EB387840217B7FF1F130707C13B
:10B220000324070B3E948357C4016382270B184005
:10B230003307EB4063EAE900834744008507B3879F
:10B240004703D6976365F70801468145094597F09E
:10B25000FFFFE780604EAA8B29E597400000E7805A
:10B26000808385476317F50689659385057117B552
:10B27000FF1F1305E59897100100E780A04F95A0E8
:10B28000B30734030327090BBA9703D7C701630831
:10B29000970003C75700A38207002382E700050435
:10B2A00015BF9305C500228597000000E78080E662
:10B2B0005E852286976501009385C51A97F0FFFF8A
:10B2C000E780E0525E8597100000E780608A850481
:10B2D00015BF97B7FF1F938767B59C478D83858BF5
:10B2E000C1F721611773FFFF670023DD0146854524
:10B2F000094502D002D202D402D697F0FFFFE780C0
:10B30000A043AA8479DD97F00000E780E09C1389D0
:10B31000C4002A8481454A8597000000E780005FC9
:10B320000C4041464A8597000000E780405B832936
:10B3300044006385090C4E8502D802DA02DC02DE85
:10B3400097300100E78060402ACE141005462C0893
:10B3500008184ECC97500000E780E00A1375F50FEF
:10B3600051ED8355840093E525004A859700000040
:10B37000E780E05E11460C104A8597000000E780E8
:10B3800000560146976501009385450E268597F086
:10B39000FFFFE780C045268597000000E780407DDD
:10B3A0005C40A1D3014685450D4597F0FFFFE7803E
:10B3B000A038AA841DD548401389C40097300100E5
:10B3C000E780A0382AC64A8597000000E780404CF5
:10B3D0003246636FC5004C404A8597000000E78005
:10B3E000005001468145268597F0FFFFE780204009
:10B3F000268597000000E780A077E5B58355840097
:10B40000ADB71773FFFFE70243CA97B7FF1F9387D4
:10B41000E7A19C471DC193E7870017A5FF1F1305F0
:10B42000257E17B7FF1F2327F7A097100100E7809D
:10B4300040321773FFFF670083C9DD9B17B7FF1FFB
:10B44000232AF79E97300000E780E0647DF117A57E
:10B45000FF1F1305E57A97100100E780E033D1BFA5
:10B460001773FFFFE702E3C14169AA892E8AB28AF6
:10B47000368BBA8B814417BCFF1F130C2C9B930C8B
:10B48000400E7D1997F0FFFFE780C05B63C4A40006
:10B4900001443DA03384940383270C0B3E948357CF
:10B4A000C401638627055A87D6865286CE85130542
:10B4B000040397000000E780E0BB01C923800B0074
:10B4C00022851773FFFF670043BF8347F40185C3DD
:10B4D0005A87D6865286CE851305940897000000B9
:10B4E000E78040B909C585472380FB00D1BF8504AB
:10B4F00051BF835745006380071E1773FFFFE702A4
:10B5000023B901112A8497000000E780C04D09C9C2
:10B5100085476309F50605611773FFFF670083BA66
:10B5200097E00000E780007C7DF5835744004947A1
:10B53000ED9BE392E7FEC145228597000000E7807E
:10B540004033AA84228597000000E780204F0357EC
:10B55000440002CE91472A89631AF700228597009A
:10B560000000E780A0513C082ACC3ECE97E00000C6
:10B57000E78080765C55C5D374084A86A685054564
:10B58000829751BF03574400D147E3F6E7F8032AF7
:10B590000400C169014997BAFF1F938A2A89130BD6
:10B5A000400EFD1997F0FFFFE780C049634FA90ED9
:10B5B0002285032A040097000000E780C042A145CD
:10B5C0002A89228597000000E780A02AAA84228584
:10B5D00097000000E780804A14402A86AA897808EC
:10B5E0002685CA8597000000E780C0E7AA8405D5B4
:10B5F00003C7F40189476315F7008347C10181DF61
:10B600005546D2851385640097300100E780E0E756
:10B61000014597800000E780C01901C583D7C401A8
:10B62000A5E797B7FF1F938767809C47935519003D
:10B63000858913D73700058B01CF8983858B639963
:10B64000B70001452EC697000000E780C0DBB24579
:10B650004E8597800000E780601F0346C1012A8461
:10B6600093751900268597900000E780E03935C171
:10B67000268597800000E780E018268511C00145E7
:10B6800097800000E780004C97300000E780A040E2
:10B690008547E312F5E883C754001307F00FE38CE6
:10B6A000E7E68507A382F400BDB5B304690383A769
:10B6B0000A0BBE9483D7C401638B37015546D285EC
:10B6C0001385640097300100E780C0D955DD050976
:10B6D000D1BD5DD86DB782801773FFFFE702439B32
:10B6E00097800000E780000C05C1C164014417A9E0
:10B6F000FF1F1309A9739309400EFD1497F0FFFF74
:10B70000E7804034634EA40017A5FF1F1305454F83
:10B7100097100100E780E0031773FFFF6700839A2B
:10B72000330534038327090B3E958357C50163888E
:10B7300097002312050097800000E780A00C050405
:10B7400075BF97A7FF1F9387676E9C478D83858B77
:10B750008DE31773FFFFE702439517A5FF1F13053E
:10B76000254A97100100E78020031773FFFF670049
:10B77000039682801773FFFFE7022393970500006B
:10B780009385C5A017A5FF1F1305854797100100D6
:10B79000E78020EE1773FFFF670063931773FFFFC7
:10B7A000E702A3908841B7E70400BC5B05054205AA
:10B7B0004181829709C585472300F5000505177368
:10B7C000FFFF6700C39083C7F5FF2E858507A38F12
:10B7D000F5FE828083C7F5FFFD1793F7F70FA38F60
:10B7E000F5FE99EF1773FFFFE702238CB7E704001C
:10B7F000BC571385F5FF82971773FFFF6700238DF2
:10B8000082801C41035745008D8FBA951CC12312BD
:10B81000B5003E85828093D78500A2051441DD8D59
:10B82000835745001387E6FF18C189072312F500E7
:10B8300013D685004111238FB6FEA38FC6FE4101AA
:10B84000828018419307F7FF1CC183574500850785
:10B850002312F500A30FB7FE8280835745008D8F1A
:10B860002312F5001C41BE950CC12E858280AA874B
:10B8700003D7470008410D8FAA952392E7008CC398
:10B880008280184108453305A740828083574500D0
:10B89000035765001D8F1C4108453385A7403305BC
:10B8A000A74082801773FFFFE702238041112EC655
:10B8B0002A8497000000E780A0FDB2456373B500BD
:10B8C00001A0835744000840BE952312B4003E9562
:10B8D00041011763FFFF6700837F1763FFFFE702E4
:10B8E000C37C41112E84B28532C697000000E780E8
:10B8F000A0FB3246A28597300100E78000B94101E4
:10B900001763FFFF6700A37C1763FFFFE702E3797C
:10B910002E84854597000000E78000F9230085000C
:10B920001763FFFF6700A37A1763FFFFE702E37760
:10B9300041112317B100894597000000E780C0F648
:10B940008347E1002300F5008347F100A300F500E1
:10B9500041011763FFFF670083771763FFFFE7026B
:10B96000C37493D78500A2054111DD8D2317B10063
:10B97000894597000000E78020F38347E10023001A
:10B98000F5008347F100A300F50041011763FFFFB5
:10B990006700E3731763FFFFE702237113978501C5
:10B9A00093D78501C166938606F0D98F13D785009A
:10B9B000758FD98FA2053707FF00F98D4111DD8DF5
:10B9C0002EC6914597000000E78000EE6C001146FE
:10B9D00097300100E78060AB41011763FFFF67000C
:10B9E000036F1763FFFFE702436C1C41854503C4E7
:10B9F000070097000000E78080E622851763FFFFBD
:10BA00006700E36C1763FFFFE702236A1C414111E3
:10BA1000894503C7070083C717002307E100A30771
:10BA2000F10097000000E78080E30355E100410149
:10BA30001763FFFF6700A3691763FFFFE702E36671
:10BA40001C414111894503C7070083C7170023071D
:10BA5000E100A307F10097000000E78040E0835772
:10BA6000E100410113D58700A2075D8D42054181A8
:10BA70001763FFFF6700A3651763FFFFE702E36239
:10BA80000C4141112A841146680097300100E7807B
:10BA9000C09F9145228597000000E78040DCB247B7
:10BAA000C166938606F01397870113D58701598DD8
:10BAB00013D78700758F598DA2073707FF00F98FBD
:10BAC0005D8D41011763FFFF670063601C45BE95F4
:10BAD0000CC18280AE87944391E6584101EF0CC1BE
:10BAE0005CC1828003C7570013671700A382E70079
:10BAF000B687D5B70CC3EDB7AA87084119CD184151
:10BB0000D44398C36313D500D8C32A87034657008C
:10BB10009376160081E6232007008280944381CA31
:10BB20008C4203A847008CC363930601CCC3799A67
:10BB300014C3A302C7003687D1BF1C45DC471D8D47
:10BB4000B777DBB6938777DB09853305F5024205C6
:10BB500041818280F147B385F50248452E95828068
:10BB60008347450085072302F50082801763FFFFA6
:10BB7000E702A3532A8409E41763FFFF67002355F4
:10BB800083474400F5DBFD1793F7F70F2302F4001A
:10BB9000E5F71C4403D7270005072391E700DC43A2
:10BBA00099C3228582974C4889CD83475400898B5D
:10BBB00099E71C4422859C479C439C478297232AF3
:10BBC00004000040232004007DB71763FFFFE70255
:10BBD000C34D8357250041112EC681EB01442285B8
:10BBE00041011763FFFF6700834E0357050081473C
:10BBF000F146E305F7FEB385D702404585072E944D
:10BC00008345440008C4F5F5B247AA8481E7232A96
:10BC1000040009A81C456C0022859C439C43829724
:10BC200048C84DDD85472312F400B24723200400A5
:10BC3000231804002319F4005C485CC483D7240053
:10BC4000FD172391F40061BF1763FFFFE702E3458F
:10BC500097A7FF1F9387C7FC88432326050023244B
:10BC60000500410597100100E78000B31763FFFF4F
:10BC70006700E3451763FFFFE702234317A4FF1F95
:10BC8000130404FA1C40411199CF9C472300B500CE
:10BC90002AC65CC197000000E78040FB1C40DC43E3
:10BCA00099C33245829741011763FFFF6700234222
:10BCB0000347450029E3584DAA877D551DCF1763DB
:10BCC000FFFFE702833E1CC3DC4797A6FF1F23A9A3
:10BCD000E6F4F156130507012390D70097050000FD
:10BCE0009385050297100100E780A098014517632E
:10BCF000FFFF6700C33D7D55828082801763FFFF91
:10BD0000E702A33A01116146814528009760FFFFD1
:10BD1000E780A03C97A7FF1F938787F09C432800EC
:10BD20009305F00FDC473EC697000000E780C0F4A3
:10BD300005611763FFFF6700833997A7FF1F93878C
:10BD400027EE9C43D847A1679387C702631EF70A73
:10BD5000397106DE22DC26DA80004AD84ED652D46B
:10BD600056D23285B28497000000E780C0C7AA8906
:10BD7000268597000000E78020C92318A4FC2685AB
:10BD800097000000E78040C82319A4FC268597008F
:10BD90000000E78060C783D744000A8A231AA4FC06
:10BDA000858393F7F70F230EF4FC8607BD0793F7FF
:10BDB000073F3301F1408A8A01498347C4FD636725
:10BDC000F902CE85130584FC232C54FD9700000056
:10BDD000E78080EA5281130104FCF2506254D2548D
:10BDE0004259B259225A925A21618280268597007F
:10BDF0000000E78060C193171900D69705092390CA
:10BE0000A7001379F90F55BF828097A7FF1F93876B
:10BE100027E19C43D847A1679387A702631AF70AD3
:10BE2000397106DE22DC26DA80004AD84ED652D49A
:10BE300056D23285B28497000000E780C0BAAA8942
:10BE4000268597000000E78020BCFD572318A4FC3E
:10BE500026852319F4FC97000000E780E0BA83D719
:10BE600044000A8A231AA4FC858393F7F70F230E54
:10BE7000F4FC8607BD0793F7073F3301F1408A8A38
:10BE800001498347C4FD6367F902CE85130584FC2D
:10BE9000232C54FD97000000E78000DE528113013F
:10BEA00004FCF2506254D2544259B259225A925A66
:10BEB00021618280268597000000E780E0B4931717
:10BEC0001900D69705092390A7001379F90F55BFDC
:10BED000828097A7FF1F9387A7D49C43D847A16769
:10BEE00089076310F70A397106DE22DC26DA800042
:10BEF0004AD84ED652D456D23285328997000000A5
:10BF0000E78060AEAA894A8597000000E780C0AF4D
:10BF1000835749000A8A2318A4FC858393F7F70FF7
:10BF2000230CF4FC8607BD0793F7073F3301F1406C
:10BF30008A8A8144834784FD63E7F402CE85130532
:10BF400084FC232A54FD97000000E780E0D2528150
:10BF5000130104FCF2506254D2544259B259225A8D
:10BF6000925A216182804A8597000000E780C0A92B
:10BF700093971400D69785042390A70093F4F40FA9
:10BF800055BF828097A7FF1F938787C99C43D847D7
:10BF9000A1679387E704631EF70A397106DE22DC86
:10BFA00026DA80004AD84ED652D456D23285B28490
:10BFB00097000000E78020A3AA892685970000004B
:10BFC000E78080A42318A4FC268597000000E78062
:10BFD000A0A3231AA4FC268597000000E780C0A236
:10BFE00083D744000A8A2319A4FC858393F7F70FAB
:10BFF000230EF4FC8607BD0793F7073F3301F1409A
:10C000008A8A01498347C4FD6367F902CE85130517
:10C0100084FC232C54FD97000000E780E0C552818A
:10C02000130104FCF2506254D2544259B259225ABC
:10C03000925A21618280268597000000E780C09C8B
:10C0400093171900D69705092390A7001379F90FC4
:10C0500055BF828097A7FF1F938787BC9C43D84713
:10C06000A1679387C704631AF70A397106DE22DCD9
:10C0700026DA80004AD84ED652D456D23285B284BF
:10C0800097000000E7802096AA8926859700000087
:10C09000E7808097FD572318A4FC2685231AF4FC1B
:10C0A00097000000E780409683D744000A8A23194E
:10C0B000A4FC858393F7F70F230EF4FC8607BD07D6
:10C0C00093F7073F3301F1408A8A01498347C4FD52
:10C0D0006367F902CE85130584FC232C54FD970079
:10C0E0000000E78060B95281130104FCF2506254F1
:10C0F000D2544259B259225A925A216182802685DD
:10C1000097000000E780409093171900D697050923
:10C110002390A7001379F90F55BF828097A7FF1FBF
:10C12000938707B09C43D847A167DD076317F704DF
:10C130001763FFFFE70263F7797132853284970056
:10C140000000E780408A2AC6228597000000E78029
:10C15000A08B2311A102228597000000E780A08810
:10C16000B2452300A102280897000000E780C0B074
:10C1700045611763FFFF670083F5828097A7FF1F64
:10C18000938707AA9C43D847A167938787046317BF
:10C19000F7041763FFFFE70243F1797132853284B8
:10C1A00097000000E78020842AC6228597000000BF
:10C1B000E78080852311A102228597000000E78097
:10C1C0008082B2452300A102280897000000E78082
:10C1D000A0AA45611763FFFF670063EF828097A7FE
:10C1E000FF1F9387E7A39C43D847A1679387A704C2
:10C1F0006312F7021763FFFFE70223EB0111280028
:10C20000814597000000E78020A705611763FFFFC5
:10C210006700E3EB828097A7FF1F938767A09C438B
:10C22000D847A167938757026319F7021763FFFF87
:10C23000E702A3E70111328597F0FFFFE780A07ABC
:10C240002308A1008145280097000000E780C0A2D4
:10C2500005611763FFFF670083E7828097A7FF1FD1
:10C260009387079C9C43D847A1679387E702631B8A
:10C27000F7041763FFFFE70243E3011132853284BD
:10C2800097F0FFFFE7804078AA84228597F0FFFFB0
:10C29000E7808077854709E9228597F0FFFFE780EF
:10C2A00080744205B337A00028008145231891000F
:10C2B0003ECA97000000E780209C05611763FFFFDE
:10C2C0006700E3E0828097A7FF1F938767959C43F1
:10C2D000D84799476313F7081763FFFFE702E3DCCA
:10C2E00079713285328497F0FFFFE780C06F2AC6EC
:10C2F000228597F0FFFFE78020712310A10222859D
:10C3000097F0FFFFE780206E2301A102228597F0BE
:10C31000FFFFE780406DA301A102228597F0FFFF98
:10C32000E780606C2302A102228597F0FFFFE7807F
:10C33000806B2313A102228597F0FFFFE780A06A9C
:10C34000B2452314A102280897000000E780C0929C
:10C3500045611763FFFF670083D7828097A7FF1FA0
:10C360009387078C9C43D847A1679387C7036313C0
:10C37000F7081763FFFFE70243D3797132853284F0
:10C3800097F0FFFFE78020662AC6228597F0FFFF1F
:10C39000E78080672310A102228597F0FFFFE780E6
:10C3A000A0662311A102228597F0FFFFE780A0631A
:10C3B0002302A102228597F0FFFFE780C062A3025B
:10C3C000A102228597F0FFFFE780E0612303A1022D
:10C3D000228597F0FFFFE7800061B245A303A10229
:10C3E000280897000000E780208945611763FFFF58
:10C3F0006700E3CD82801763FFFFE70203CB0111E3
:10C400002A8497F0FFFFE780005EAA84228597F0D8
:10C41000FFFFE780605F228597F0FFFFE780C05E47
:10C42000035744008D4763F7E700228597F0FFFF2D
:10C43000E780805D228597F0FFFFE780E05C2800C1
:10C44000A68597000000E780208305611763FFFF42
:10C450006700E3C79797FF1F9387877C9C43D84764
:10C46000A167FD07631FF7001763FFFFE702E3C340
:10C47000328597000000E78040F81763FFFF6700F0
:10C4800003C582809797FF1F938787799C43D8477E
:10C49000A167E5076315F7081763FFFFE702E3C02D
:10C4A00079713285328497F0FFFFE780C0532AC646
:10C4B000228597F0FFFFE7802055228597F0FFFF48
:10C4C000E78080542310A102228597F0FFFFE780C8
:10C4D000A053520551812311A1022285230201029A
:10C4E00097F0FFFFE7802050A302A102228597F07A
:10C4F000FFFFE780404F2303A102228597F0FFFF53
:10C50000E780604EB245A303A102280897F0FFFF21
:10C51000E780807645611763FFFF670043BB828039
:10C520009797FF1F9387C76F9C43D847A16793874F
:10C53000E703631FF7001763FFFFE70203B73285C6
:10C5400097000000E78060EB1763FFFF670023B8E8
:10C5500082809797FF1F9387A76C9C43D847A1675A
:10C5600093874704631EF7021763FFFFE702E3B3F5
:10C5700079713285328497F0FFFFE780C0462AC682
:10C58000228597F0FFFFE7802048B245280897F002
:10C59000FFFFE780606E45611763FFFF670023B30D
:10C5A00082809797FF1F9387A7679C43D847A1670F
:10C5B000938787026310F7041763FFFFE702E3AE78
:10C5C00079713285328497F0FFFFE780C0412AC637
:10C5D000228597F0FFFFE7800041B2452300A102CA
:10C5E000280897F0FFFFE780206945611763FFFF88
:10C5F0006700E3AD82801763FFFFE70203AB011121
:10C6000097F0FFFFE780203EAA85280097F0FFFF04
:10C61000E780806605611763FFFF670043AB97976C
:10C62000FF1F9387E75F9C43D847A167D107631F2C
:10C63000F7001763FFFFE70243A73285970000006A
:10C64000E780A0FB1763FFFF670063A882809797CE
:10C65000FF1F9387E75C9C43D847A167C507631F0B
:10C66000F7001763FFFFE70243A43285970000003D
:10C67000E780A0F81763FFFF670063A582809797A4
:10C68000FF1F9387E7599C43D847A167B907631FEA
:10C69000F7001763FFFFE70243A132859700000010
:10C6A000E780A0F51763FFFF670063A2828097977A
:10C6B000FF1F9387E7569C43D847A167AD07631FC9
:10C6C000F7001763FFFFE702439E328597000000E3
:10C6D000E780A0F21763FFFF6700639F8280979750
:10C6E000FF1F9387E7539C43D84789476318F70296
:10C6F0001763FFFFE702639B0111328532C897F091
:10C70000FFFFE780402EAA85280097F0FFFFE78013
:10C71000A05605611763FFFF6700639B82809797B0
:10C72000FF1F9387E74F9C43D847A1678D0763118D
:10C73000F7041763FFFFE702439701113285328444
:10C7400097F0FFFFE780202A13066100AA844C00BF
:10C75000228597300000E780C0232800A68597F047
:10C76000FFFFE780605105611763FFFF67002396B5
:10C7700082809797FF1F9387E74A9C4381CFDC43D2
:10C7800091CB1763FFFFE702439282971763FFFF86
:10C790006700E39382801763FFFFE70203917971DB
:10C7A0003C08AE843ED2A165B7070A002A843ED475
:10C7B00048103C08DD053ED636C432C63AC297D092
:10C7C000FFFFE780E02F12474810BA8597F0FFFF80
:10C7D000E780C01332464810B28597F0FFFFE7802C
:10C7E000E014A2464810B68597F0FFFFE7800012DC
:10C7F000501001478146A685228597D0FFFFE7802C
:10C80000805145611763FFFF6700638C1763FFFF6B
:10C81000E702A38901117C000329C501AE843ECA49
:10C82000A165B70707002A843ECC48087C00C505EF
:10C830003ECE97D0FFFFE780A0288345D900480867
:10C8400097F0FFFFE780800C500801478146A685DE
:10C85000228597D0FFFFE780004C05611763FFFF3B
:10C860006700E3861763FFFFE702238483C7950011
:10C8700093F7F707A384F50097000000E78040F9DD
:10C880001763FFFF6700A3841763FFFFE702E381DD
:10C8900079713C08AE843ED2A165B70709002A84AD
:10C8A0003ED448103C08938545043ED632C636C473
:10C8B00097D0FFFFE780C020A2464810B68597F0CA
:10C8C000FFFFE780A00432464810B28597F0FFFFD3
:10C8D000E780C005501001478146A685228597D084
:10C8E000FFFFE780404345611753FFFF6700237E4A
:10C8F0001753FFFFE702637B83C7950041112A842A
:10C9000093F7F707A384F50032852EC697F0FFFF53
:10C91000E780800F85672AC46370F5029770000076
:10C92000E78020E92246B24509ED1147814622857C
:10C9300097000000E78060E641011753FFFF6700A2
:10C94000037901478346F501DDB71753FFFFE7027F
:10C95000237401113C003ECAB7070A003ECC3C00DC
:10C960003ECE83C79500AA89328593F7F707A38443
:10C97000F5002E8497F0FFFFE78000098567637D4F
:10C98000F504A165AA8493858504480897D0FFFF24
:10C99000E7800013268597700000E78080E12A89F0
:10C9A00029E19145480897F0FFFFE78020F6A6852A
:10C9B000480897F0FFFFE78060F7CA85480897F0BE
:10C9C000FFFFE780A0F4014781465008A2854E850D
:10C9D00097D0FFFFE780203405611753FFFF670002
:10C9E000636E8145480897F0FFFFE78020F2034916
:10C9F000090275BF1753FFFFE702836979711C10A5
:10CA00003ECAB7070F003ECC404D1C10AA84AE8929
:10CA10004808994532C636893ECE97D0FFFFE78059
:10CA2000200A32464808B28597F0FFFFE78000EE03
:10CA3000630C0902A545480897F0FFFFE780C0E6B0
:10CA40002546CA8597200100E78020A450080147A9
:10CA50008146CE85268597D0FFFFE780C02B4561B4
:10CA60001753FFFF670003668355C402480897F019
:10CA7000FFFFE780A0EB0355E402814505C585472C
:10CA800085456301F502C167FD179305F00F630B40
:10CA9000F5007D1597700000E780208E9305150046
:10CAA00093F5F50F480897F0FFFFE78020E68345F0
:10CAB0000403480897F0FFFFE78040E5834514032F
:10CAC000480897F0FFFFE78060E483552403480897
:10CAD00097F0FFFFE78080E583554403480897F00F
:10CAE000FFFFE780A0E49DB71753FFFFE702E35B7A
:10CAF00083C795008146014693F7F707A384F500A5
:10CB000097000000E78040EF1753FFFF6700235CAA
:10CB10001753FFFFE702635979713E841C103ECA28
:10CB20002E89B7070F00A1653ECCFD051C10AA8415
:10CB3000480842C03AC23ECE36C432C697D0FFFF44
:10CB4000E78000F832464808B28597F0FFFFE7809B
:10CB5000E0DBA2464808B68597F0FFFFE78000DDDE
:10CB600012474808BA8597F0FFFFE78020DC0248AB
:10CB7000630C08029145480897F0FFFFE780C0D298
:10CB80001146A28597200100E780209050080147B8
:10CB90008146CA85268597D0FFFFE780C01745618B
:10CBA0001753FFFF6700A3528945480897F0FFFF1E
:10CBB000E78080CF834704002300F50083471400FB
:10CBC000A300F500E1B71753FFFFE702634C83C7EB
:10CBD000950001112A8A93F7F707A384F50032859F
:10CBE000AE8432C697F0FFFFE78000E232462A8922
:10CBF000328597F0FFFFE78000DF85676373F902F6
:10CC0000AA894A8597700000E780A0BA2A8419EDA6
:10CC1000114781464A86A685528597000000E78025
:10CC2000C0B705611753FFFF6700C3499387E9FF4A
:10CC300093F7F70F0547E366F7FE8347F50195EB9A
:10CC40008947E380F9FE8346F401528501474A860D
:10CC5000A68597000000E78040B4A167D90748087F
:10CC60003ECC230A010002CE97000000E780A0B06E
:10CC70004DBF639EE7008947639EF900930710202C
:10CC8000231FF50097700000E780C0B76DBF09470C
:10CC9000E39BE7FA8D47E398F9FA22859770000045
:10CCA000E78080DF9797FF1F9387C7169C4399E71C
:10CCB0009797FF1F9387C7FF9C4399C703D504002D
:10CCC00097800000E780A0CE231F040022855DBF6F
:10CCD0001753FFFFE702633D01113C003ECAB7074F
:10CCE0000B003ECC3C003ECE83C795002A8932859E
:10CCF00093F7F707A384F500AE8497F0FFFFE78072
:10CD0000A0D093170501C187635AF006A1652A8454
:10CD10009385E502480897D0FFFFE78060DAA28597
:10CD2000480897F0FFFFE78060C09797FF1F938741
:10CD300027F89C43A9EB01449375F40F480897F03A
:10CD4000FFFFE780A0BC9355844093F5F50F48089A
:10CD500097F0FFFFE78080BB9355044193F5F50FF3
:10CD6000480897F0FFFFE78060BA01478146500806
:10CD7000A6854A8597D0FFFFE780E0F90561175344
:10CD8000FFFF6700C334416585460546A2857D15D2
:10CD900097500000E78060BD59DD51059700010004
:10CDA000E780808F130440063344850271B7175320
:10CDB000FFFFE702832F0111B70706003EC683C7B6
:10CDC000950021642A8993F7F707A384F500AE84C0
:10CDD00028009305A4040AC40AC897D0FFFFE7807F
:10CDE00020CE300001478146A6854A8597D0FFFFB7
:10CDF000E78060F297E0FFFFE7808015130494045A
:10CE0000480822CC230A010002CE97000000E780E8
:10CE1000809605611753FFFF6700632B1753FFFFD1
:10CE2000E7020327C1642A8901449799FF1F938968
:10CE3000E9FF130A8002FD1497E0FFFFE78080C13D
:10CE40006347A40001451753FFFF6700A327B307FB
:10CE5000440303A7C90ABA9703D7070063069700DC
:10CE600083D72700638427010504F9B70545E1BF8F
:10CE70001753FFFFE702C3212A8A2E8999C123A0F5
:10CE8000050081498144979AFF1F938AEAD9614B33
:10CE900097E0FFFFE78040C263C7A4004E851753A9
:10CEA000FFFF670023223384640383A70A003E94B4
:10CEB0008357040099E7630409002320890085044F
:10CEC000C1BF4146D2851305440097100100E78099
:10CED000605975F5A289E5B71753FFFFE702431BB9
:10CEE00039717C083ED4B7070A003ED67C083ED88C
:10CEF00083C795002A8A328593F7F707A384F50044
:10CF00002E8932C697F0FFFFE78000B08567637314
:10CF1000F5083246AA84328597F0FFFFE780A0AC7F
:10CF20008547AA8963E8A706A1659385850428102B
:10CF300097D0FFFFE780C0B8268597700000E78094
:10CF400040872A8429ED9145281097F0FFFFE7805C
:10CF5000E09BA685281097F0FFFFE780209DCE85F7
:10CF6000281097F0FFFFE780609A01478146301054
:10CF7000CA85528597D0FFFFE780E0D9A1679387E4
:10CF8000770448183EDC230A010202DE97F0FFFF17
:10CF9000E780607E21611753FFFF6700A312814580
:10CFA000281097F0FFFFE7806096A685281097F07D
:10CFB000FFFFE780A0979797FF1F9387E71D9C438C
:10CFC00081CB22856389090097D00000E780402447
:10CFD0008345040271B797D00000E780C022CDBF1F
:10CFE0001753FFFFE702C30A83C795004111AA89BF
:10CFF00093F7F707A384F5003285AE84328A97F061
:10D00000FFFFE78060A08567637FF5022A8997604C
:10D010000000E780007A2A84914631C58347F501F4
:10D0200005476387E70291C70D476366F704AD467E
:10D030001DA89305050303250A004146971001002A
:10D04000E78040420DE941011753FFFF6700830766
:10D050009305950803250A00414697100100E780D3
:10D060006040814669F54A86A6854E859700000096
:10D07000E780C081C9BF83250A0013059408977013
:10D080000000E780A02919C1C146F1BF9797FF1F93
:10D09000938747D89C4399E79797FF1F938747C18A
:10D0A0009C4399C7228597800000E780208A69FD0C
:10D0B0008547A30FF400228597B00000E7806084C5
:10D0C000228597600000E780E0734E8581464A869E
:10D0D000A68597F0FFFFE780607BA16793875704E1
:10D0E00048003EC42302010002C697F0FFFFE7801C
:10D0F000806891BF1753FFFFE702A3F883C795002D
:10D100004111AA8993F7F707A384F50032852E8988
:10D11000B28A97F0FFFFE780208F85676374F50E72
:10D12000AA8497600000E780C0682A840DED416BF7
:10D13000014A979BFF1F938B6BCF130C400E7D1BF7
:10D1400019A833048A0383A70B0B3E948357C401A9
:10D1500063836705050A97E0FFFFE780A08EE3423F
:10D16000AAFE95460DA08357C501639697029305C5
:10D17000050303A50A00414697100100E780802EB1
:10D18000994611E181462686CA854E8597F0FFFFB4
:10D19000E780C06F85A883A50A0013050403977074
:10D1A0000000E780A017C14679FD2285231E940068
:10D1B00097A00000E780E074228597600000E78078
:10D1C00060649797FF1F938727FD9C43A9C32300A3
:10D1D0000402228597D00000E78040F04E8581460A
:10D1E0002686CA8597F0FFFFE780406AA16793878C
:10D1F000070448003EC42302010002C697F0FFFF67
:10D20000E780605741011753FFFF670003EB894731
:10D210002300F402E1B7397106DE22DC4AD880002F
:10D2200052D456D25AD026DA4ED65ECE2E8A3289C3
:10D230002A8B97D0FFFFE780E07D060571054199B5
:10D240008A8A3301A140232224FC231404FC97D0B2
:10D25000FFFFE780207C83479A000605350593F79A
:10D26000F7072315A4FCA304FA004A85232624FC0F
:10D2700097E0FFFFE780407993170501C18763407E
:10D28000F0025681130104FCF2506254D254425908
:10D29000B259225A925A025BF24B21618280AA84CF
:10D2A0004A8597E0FFFFE7802076AA894A8597E0C4
:10D2B000FFFFE7806075A1659385C5022A89130584
:10D2C00044FC97C0FFFFE780A07F268597C0FFFF43
:10D2D000E780E073854511C94A86CE8597C0FFFF78
:10D2E000E780606DAA8B21E98945130544FC97E02E
:10D2F000FFFFE780A061A685130544FC97E0FFFFD0
:10D30000E780C062CE85130544FC97E0FFFFE7800D
:10D31000E061CA85130544FC97E0FFFFE7800061E8
:10D3200001478146130644FCD2855A8597D0FFFFFA
:10D33000E780609EB9B78145130544FC97E0FFFF85
:10D34000E780C05CA685130544FC97E0FFFFE780FB
:10D35000E05DCE85130544FC97E0FFFFE780005DAC
:10D36000CA85130544FC97E0FFFFE780205C8144F9
:10D3700097D0FFFFE780006AE3D4A4FA83A70B01EC
:10D3800013971400BA9783D5070099C5130544FC79
:10D3900097E0FFFFE78080598504D9BF797106D6F1
:10D3A00022D44AD000184ECE52CC56CA26D25AC8E1
:10D3B000AE893289AA8A97D0FFFFE780A06506056B
:10D3C000690541990A8A3301A140232A24FC231CC0
:10D3D00004FC97D0FFFFE780E06383C79900060550
:10D3E0002D0593F7F707231DA4FCA384F9004A85B4
:10D3F000232E24FC97E0FFFFE780006193170501CF
:10D40000C187634FF0005281130104FDB2502254D2
:10D4100092540259F249624AD24A424B4561828093
:10D42000AA844A8597E0FFFFE780005EA1659385A7
:10D43000A5022A89130544FD97C0FFFFE7804068D5
:10D44000268597C0FFFFE780805C854509C9CA85AE
:10D4500097C0FFFFE78020592A8B29E189451305F2
:10D4600044FD97E0FFFFE780604AA685130544FD71
:10D4700097E0FFFFE780804BCA85130544FD97E0E6
:10D48000FFFFE780A04A01478146130644FDCE8591
:10D49000568597D0FFFFE7800088B5B78145130513
:10D4A00044FD97E0FFFFE7806046A685130544FD35
:10D4B00097E0FFFFE7808047CA85130544FD97E0AA
:10D4C000FFFFE780A046814497D0FFFFE7808054AC
:10D4D000E3DBA4FA83270B0113971400BA9783D5D3
:10D4E000070099C5130544FD97E0FFFFE78000445E
:10D4F0008504D9BF1753FFFFE70223BB83474500CD
:10D50000404DD5EFFD575DC48346940009476363E2
:10D51000D70A0346B400854663EEC6088306E400D6
:10D5200063CA06085C45F9562390D7009787FF1F0A
:10D5300083C7C76F99E3A304E4009787FF1F93870E
:10D5400027779C4381E78947A306F4009797FF1F3D
:10D55000938787C49C4381E789472306F400970596
:10D56000000093854506AA841305040197F0000086
:10D57000E7802010FD57231AF40281471CDC014884
:10D580009787FF1F23A0876A9787FF1F9387C76925
:10D59000232E040304C0804397D0FFFFE780C051CF
:10D5A00061463306C502814522859750FFFFE7801B
:10D5B000C0B281473E851753FFFF670043B1FD5757
:10D5C000D5BF1753FFFFE70243AE2A840355450238
:10D5D00097600000E780E01D19E5231E0400175343
:10D5E000FFFF6700C3AE8357E401F5DB930504FF3B
:10D5F000174501001305452197E00000E780E0147E
:10D60000F9BF1753FFFFE70243AA2E89A165411115
:10D610009385E5032A8436C432C6BE843AC297C0D5
:10D62000FFFFE780E04912472285BA8597E0FFFFB8
:10D63000E780C02D32462285B28597E0FFFFE78064
:10D64000E02EA2462285B68597E0FFFFE780002EF8
:10D65000630309029145228597E0FFFFE780C0241C
:10D660001146A68597100100E78020E2410117537B
:10D67000FFFF6700C3A58945228597E0FFFFE7808C
:10D68000A02283C704002300F50083C71400A30071
:10D69000F500E9BF1753FFFFE70223A183C79500F9
:10D6A000444D054793F7F707A384F5001C42411149
:10D6B00083C707006367F7062E842A89B1C003C7B2
:10D6C000D400630FF7021787FF1F1307675E184325
:10D6D00005C3A386F40097A00000E780404A83C7F3
:10D6E000D40099E741657D1597400000E780403000
:10D6F00083D72403918B89C797E00000E780C0138C
:10D700004A85A28597F0FFFFE7808010A167C107D7
:10D7100048003EC42302010002C697F0FFFFE780E5
:10D72000800541011753FFFF6700639A1753FFFFFE
:10D73000E702A39703D745008D47AA8441112E84A1
:10D7400032892E8563E3E70297E0FFFFE780C02B75
:10D75000AA8523000900268597C0FFFFE780A0283F
:10D7600041011753FFFF6700839697E0FFFFE780B3
:10D77000A0292AC6228597E0FFFFE780E028B2456E
:10D7800085472A862300F900268597C0FFFFE7809A
:10D790008022F9B7397106DE22DC26DA80004ED607
:10D7A00052D456D24AD85AD05ECEAE89B284AA8A12
:10D7B00097D0FFFFE7800025060513052502419954
:10D7C0000A8A3301A140232224FC231404FC97D0AD
:10D7D000FFFFE780202383C7990006054D0593F7D7
:10D7E000F7072315A4FCA384F9002685232624FC2F
:10D7F00097E0FFFFE780402193170501C187634051
:10D80000F0025281130104FCF2506254D254425986
:10D81000B259225A925A025BF24B21618280AA8B42
:10D8200003AB040097C0FFFFE780601E51E583D77C
:10D83000440001498544F11793B71700A301F4FC94
:10D84000834734FCA165C9C79385E504130544FCEF
:10D8500097C0FFFFE780C026A685130544FC97E02C
:10D86000FFFFE780A00ADE85130544FC97E0FFFF79
:10D87000E780C00B834734FC114691E30946DA8503
:10D88000130544FC97E0FFFFE78060058144630ACD
:10D890000900416B7D1B97D0FFFFE780A01663CC8A
:10D8A000A40201478146130644FCCE85568597C0E5
:10D8B000FFFFE7804046B1B7A685130634FC97000A
:10D8C0000000E780E0E6933415002A8986048DBFC6
:10D8D0009385C504A5BF8327C90013971400BA9781
:10D8E00083D5070063886501130544FC97E0FFFFBB
:10D8F000E780C003850445B71743FFFFE70263785D
:10D9000079711C103EC4B7070F003EC61C103EC8FC
:10D9100083C79500AA8A328593F7F707A384F50099
:10D92000AE89328497E0FFFFE780000E9317050170
:10D93000C187635AF0062A8A228597E0FFFFE780B5
:10D94000A00C2A895285032B040097C0FFFFE780B3
:10D95000000C39ED8357440081440544F11793B717
:10D960001700A303F10083457100DA872287CA8676
:10D970005286280097000000E780E0C801478146F2
:10D980003000CE85568597C0FFFFE780C038A1677D
:10D990009387D70348083ECC230A810026CE97F010
:10D9A000FFFFE78040DD45611743FFFF6700E3703D
:10D9B000A2851306710097000000E78060D7AA8453
:10D9C000094455D13544E30055FB4A8597F0FFFFE4
:10D9D000E78000450D4441D9014497D0FFFFE7801F
:10D9E0006002634DA400C16B0144FD1B97D0FFFF93
:10D9F000E7804001634EA4001544B5B7DC4413171B
:10DA00001400BA9783D70700638327030504F1B78F
:10DA1000D84493171400BA9703D70700631B770104
:10DA200023902701268597A00000E78080DB014432
:10DA30001DBF050465BF1743FFFFE702636583C78A
:10DA4000950041112A8A93F7F707A384F5003285E0
:10DA50002E89328497E0FFFFE78000FB93170501D2
:10DA6000C1876353F006AA89228597E0FFFFE7800C
:10DA7000A0F92311A1004E85832A040097C0FFFF5F
:10DA8000E780E0F839E58357440085440144F11705
:10DA900093B71700A300F1000348110003572100BA
:10DAA000D6875285CE862686CA8597F0FFFFE78007
:10DAB0006006A167F10748003EC42302910022C618
:10DAC00097F0FFFFE78020CB41011743FFFF67007E
:10DAD000635FA2851306110097000000E78040C530
:10DAE0002A84894455D98357210011678544BA9700
:10DAF000C2071167C1831307F7EFE36FF7F8978742
:10DB0000FF1F938727319C4381CB85451305210057
:10DB100097500000E78020758355210022858144BD
:10DB200097C0FFFFE78040E525D923100500228537
:10DB300097A00000E78040CD85B71743FFFFE702BD
:10DB4000435483C7950041112A8B93F7F707A384A9
:10DB5000F50032852E8A328497E0FFFFE780C0EA25
:10DB600093170501C1876351F006AA8A228597E0C1
:10DB7000FFFFE78060E92A895685832B040097C060
:10DB8000FFFFE780C0E831E5835744008144054446
:10DB9000F11793B71700A301F10003483100DE87A6
:10DBA0005A854A87D6862286D28597F0FFFFE7807E
:10DBB00060F6A167ED0748003EC42302810026C637
:10DBC00097F0FFFFE78020BB41011743FFFF67008D
:10DBD000C34EA2851306310097000000E78040B5D0
:10DBE000AA8409445DD99167CA97C2071167C183A6
:10DBF0001307F7EF0544E362F7FACA8597C0FFFF02
:10DC0000E78080D7014451F9814997D0FFFFE78031
:10DC100060E063DBA900984893971900BA9703D78F
:10DC2000070005EF2390270197D0FFFFE78080DEF4
:10DC30001544E384A9F6268597A00000E780C0BCC0
:10DC40009787FF1F9387071D9C430144B9D74A85D7
:10DC500097500000E780C05889B785097DB7174302
:10DC6000FFFFE702E34279713E847C083EC82E8ABA
:10DC7000B7071400A1653ECAE5057C08AA89080813
:10DC800036C4428932C6BA8AC6843ECC97C0FFFFEA
:10DC9000E78000E3CA85080897E0FFFFE78000C738
:10DCA00032460808B28597E0FFFFE78020C8A24609
:10DCB000630A09049D45080897E0FFFFE780C0BE9E
:10DCC0001D4681459740FFFFE780204163890A0890
:10DCD0009145080897E0FFFFE78000BD1146A68543
:10DCE00097000100E780607A100801478146D285DD
:10DCF0004E8597C0FFFFE780000245611743FFFF95
:10DD00006700433CB685080897E0FFFFE78000C244
:10DD10001C400808D8439355C701858912075183D1
:10DD2000B205D98D97E0FFFFE78040C01C4008088E
:10DD300083C5870097E0FFFFE78040BD1C400808CF
:10DD400083C5A70097E0FFFFE78040BC1C400808A0
:10DD500083C5970097E0FFFFE78040BB85BF8945FB
:10DD6000080897E0FFFFE78020B483C70400230082
:10DD7000F50083C71400A300F500BDB71743FFFFEC
:10DD8000E702033183C795004111AA8993F7F7078A
:10DD9000A384F5003285AE84328497E0FFFFE780EC
:10DDA000A0C693170501C187635DF0042A89032A81
:10DDB000040097C0FFFFE78080C519E9835744003E
:10DDC0000548F11793B71700A307F100814631A862
:10DDD0001306F100A28597000000E78060951DC53D
:10DDE0001C459DC783D6470001480347F1009307B0
:10DDF0008500D2884A86A6854E8597000000E78078
:10DE000040E641011743FFFF6700C32B09487DBF70
:10DE10001D486DBF1743FFFFE702832765715C084C
:10DE20003EC4B7077B013EC65C083EC883C7950069
:10DE30002A8A328593F7F707A384F500AE8997E025
:10DE4000FFFFE78040BA8357E100E1C7894528001A
:10DE500097C0FFFFE780C0C68145280097E0FFFF1D
:10DE6000E780C0AA97C0FFFFE780A0CC9787FF1F7D
:10DE7000938787329C431784FF1F034424DBAA84C3
:10DE80003334800099C3136424009787FF1F93875E
:10DE900027E29C4399C3136444009787FF1F93872D
:10DEA00067F79C4399C31364840083D5040028005A
:10DEB000014997E0FFFFE78060A783D52400280091
:10DEC00097E0FFFFE78080A683D54400280097E015
:10DED000FFFFE780A0A597D0FFFFE780A0AE9315D6
:10DEE0000501C181280097E0FFFFE78020A4A285FB
:10DEF000280097E0FFFFE78060A39C446360F9027D
:10DF0000014781463000CE85528597C0FFFFE780EC
:10DF100080E059611743FFFF6700C31ADC44131404
:10DF2000490028003E9497E0FFFFE7806096834712
:10DF300044000347540089070607BA978607E36A37
:10DF4000F5FC835524002800814A97E0FFFFE78015
:10DF5000E09D83454400280097E0FFFFE780009B99
:10DF600083455400280097E0FFFFE780209A83470D
:10DF7000440063C9FA00814A8347540063C1FA022E
:10DF80000509A5BF1C4413975A002800BA9783D5EA
:10DF90000700850A97E0FFFFE7804099C9BF032B80
:10DFA000C40093975A0028003E9B83552B00850A96
:10DFB00097E0FFFFE780809783550B00280097E0EC
:10DFC000FFFFE780A0964DBF1743FFFFE702E30D79
:10DFD0005C4993E717005CC997A00000E78020B672
:10DFE0001743FFFF6700A30E1743FFFFE702E30B92
:10DFF0002E84814597F0FFFFE780C0E705C5835772
:10E000000500FD172310F50009C4835725002310D0
:10E01000F40097000000E78060FB01451743FFFF15
:10E020006700E30A31457DD823100400C5BF1743BC
:10E03000FFFFE702E30583C7950041112A8A93F7A2
:10E04000F707A384F50032852E89328497E0FFFF1D
:10E05000E780809B93170501C1876356F006AA8964
:10E06000C145228597E0FFFFE780A0802A8B4E857F
:10E07000832A040097C0FFFFE780609931E9835746
:10E080004400231101000544F11793B71700A300C2
:10E09000F10081440348110003572100D6875285BF
:10E0A000CE862286CA8597F0FFFFE780A0A6A167EB
:10E0B0009387170248003EC42302810026C697E0DA
:10E0C000FFFFE780406B41011743FFFF670083FFBD
:10E0D00013061100A28597F0FFFFE7806065AA8410
:10E0E00009E523110100094475B7930521005A85FC
:10E0F00097000000E78080EF835721002A84D9DB56
:10E100009787FF1F938707D19C4381CB85451305D4
:10E11000210097500000E7800015835521002685D7
:10E12000314497C0FFFFE78020852DD523100500DF
:10E13000268597900000E780206D0144A1BF17431A
:10E14000FFFFE70283F641112E896C00AA8402C604
:10E1500097F0FFFFE78000D20DC1035705000507C8
:10E160002310E50097000000E78040E681473E85E8
:10E1700041011743FFFF670083F53247954765DB91
:10E18000CA85268597300000E780400DC147E340EF
:10E1900005FE3244854741462310F40083570900A9
:10E1A000A685130544002311F40097000100E780C1
:10E1B000C02D228545BF1743FFFFE70263ED83C7EC
:10E1C00095004111AA8A93F7F707A384F5003285D9
:10E1D000AE89328497E0FFFFE78000839317050143
:10E1E000C1876356F0062A8AC145228597D0FFFF72
:10E1F000E7802068AA845285032B040097C0FFFFA4
:10E20000E780E08031E98357440023110100854411
:10E21000F11793B71700A300F10001440348110060
:10E2200003572100DA875685D2862686CE8597F059
:10E23000FFFFE780208EA1679387070248003EC456
:10E240002302910022C697E0FFFFE780C052410100
:10E250001743FFFF670003E7A2851306110097F03D
:10E26000FFFFE780E04C2A8409E52311010089447F
:10E2700075B726859305210097000000E78060ECC4
:10E28000AA8449FD83552100228597B0FFFFE780CE
:10E29000A06E49F5014997C0FFFFE780A077635D55
:10E2A000A900184893171900BA9703D707000DEF74
:10E2B000035721002390E70097C0FFFFE780807598
:10E2C000630625039787FF1F9387C7B49C4399C7AD
:10E2D0000355210097500000E78080F02285979039
:10E2E0000000E78060521DBF050975B795443DB732
:10E2F00005C19307F00F630FF500C547630CF500E8
:10E300009307F5FF05453315F500420541818280ED
:10E310000145828041657D158280B9E91743FFFF81
:10E32000E702A3D803450603328497000000E78084
:10E3300060FC9305803EB305B502C205C18181CD65
:10E340000357E402854763F8E7001305040197E0EB
:10E350000000E78020428357E40241677D17638510
:10E36000E700FD172317F4021743FFFF670023D6CA
:10E3700082801743FFFFE702C3D0004283C79500A6
:10E38000444D0349140093F7F707A384F50083472E
:10E390000400220911673369F900A167B347F90046
:10E3A00041112A8BAE8A63ECE70E834724001307E2
:10E3B000C00EB91793F7F70F6373F71003473400D4
:10E3C000C14763EEE70E834744001307E00793C796
:10E3D00007086371F70C8349840083477400A2091E
:10E3E000B3E9F900856763F7F90A034A64008347D4
:10E3F00054004E85220A336AFA0097500000E780E5
:10E40000403B61C123962403834B3400137AFA0006
:10E41000239A3403238874032399440393890401C2
:10E42000631C090023A60402239804024E8597E08A
:10E430000000E78060363DA0034924004A8597002C
:10E440000000E78020EB2397A402834744004E8519
:10E45000A388F402E38D0BFCE30B09FC97E00000BA
:10E46000E780202F97900000E780007381460146E7
:10E47000D6855A8597E0FFFFE7800058A16793870C
:10E4800097033EC423020100480002C697E0FFFF45
:10E49000E780602E41011743FFFF670003C28544F8
:10E4A000A2862686D6855A8597E0FFFFE780C0546E
:10E4B000A167938797033EC423029100F1B7BD443F
:10E4C000C5B79144F1BF1743FFFFE70263BC0111D9
:10E4D0001C08404D3EC2B7070F003EC41C083EC694
:10E4E0002A89AE8997C0FFFFE780A0DA585C1C5CE0
:10E4F0006346B70E6394E50063E2A70E3385A74039
:10E50000B3B7A700B305B7401306803E81469D8D83
:10E5100097000100E78080B793140501C180A165D1
:10E520009385C503480097B0FFFFE7806059814598
:10E53000480097D0FFFFE780603D83550404480002
:10E5400097D0FFFFE780803E83552404480097D092
:10E55000FFFFE780A03D814589CCC167FD1793058A
:10E56000F00F6388F400268597500000E780E0E014
:10E57000AA85480097D0FFFFE7804039035544043F
:10E58000814501CDC167FD179305F00F6307F500C5
:10E5900097500000E78060DEAA85480097D0FFFF13
:10E5A000E780C03683456404480097D0FFFFE780CA
:10E5B000E03583457404480097D0FFFFE7800035BD
:10E5C000500001478146CE854A8597B0FFFFE7801E
:10E5D000807405611743FFFF6700C3AE814481B7B4
:10E5E0001743FFFFE70263AC83C7950093F7F70774
:10E5F000A384F50097000000E78020ED1743FFFF9C
:10E600006700E3AC1743FFFFE70283A883C79500C9
:10E610004111404D93F7F707A384F5002A8A32850C
:10E62000B284AE8997D0FFFFE780003E2A8B268513
:10E6300097D0FFFFE780403D2A89268597D0FFFFCE
:10E64000E780603A93170B0163CA0702E177CA9724
:10E65000C207C183116763E3E70293070910C2078A
:10E66000C1831307B00F637BF70093170901C187BC
:10E67000AA8A634AF000C54763FE57014101174368
:10E68000FFFF670023A497B0FFFFE780C028E317D0
:10E6900025FFD5B763080B0263060902814463892D
:10E6A0000A02B7077F0023106405231124057CC0EC
:10E6B000568597000000E780E0C39304803EB304D2
:10E6C000950239A0B7077F00232004047CC0814451
:10E6D0000355240497E00000E780A0A3A1C497C0DD
:10E6E000FFFFE78000BB269593D7F44133379500B1
:10E6F000AE97BA9708DC5CDCCE85528597000000A7
:10E70000E780A0DC99E023220404A1679387B70384
:10E7100048003EC42302010002C697E0FFFFE780E5
:10E720008005A9BF814701481CDC232E0403E9B7FB
:10E730001743FFFFE702639797C0FFFFE780C037EB
:10E74000E1473305F502914597500000E78000C589
:10E75000E55711C59777FF1F23A8A74C81473E8532
:10E760001743FFFF6700A39685471777FF1F230F07
:10E77000F74A82801743FFFFE70223939777FF1F33
:10E780009387474A80433DC0835704046390A7069C
:10E7900083572404639CB7043689B28497C0FFFF73
:10E7A000E78020AF5C5C63C3B7046395B7001C5C73
:10E7B00063EEA7028347640463F3F400A687230390
:10E7C000F4048347740463F39700A687A303F40457
:10E7D0008357440441677D176385E700850723124B
:10E7E000F4043C4481C7CA85268582971743FFFFFE
:10E7F0006700E38D9777FF1F9387C7429C430145CE
:10E8000099C303C5870082801743FFFFE702E389AE
:10E810000111B70707003EC683C79500584D0AC4CB
:10E8200093F7F7070AC8A384F5002A89AE8411CBB1
:10E830001C4283C707002304F70097900000E7807D
:10E840000034216493055402280097B0FFFFE7804D
:10E85000202797000000E78020FAAA85280097D09B
:10E86000FFFFE780A00A300001478146A6854A8560
:10E8700097B0FFFFE780204A13044402480822CCE7
:10E88000230A010002CE97E0FFFFE780C0EE05619A
:10E890001743FFFF6700A3831743FFFFE702E380EF
:10E8A00001117C003ECAB70707003ECC7C003ECE7B
:10E8B00083C795002E84AA8493F7F707A384F500F5
:10E8C000A16593855502480897B0FFFFE780401F78
:10E8D00097000000E78040F2AA85480897D0FFFF24
:10E8E000E780C002500801478146A285268597B07F
:10E8F000FFFFE780404205611733FFFF6700237D7C
:10E900009777FF1F938707329C43094599C303C537
:10E91000970082809777FF1F9387C7309C430945F4
:10E9200099C303C5D70082809777FF1F9387872FEE
:10E930009C43014599C303C5A70082801733FFFF9D
:10E94000E70203750111B70708003EC683C79500AB
:10E95000404D0AC493F7F7070AC8A384F5002A8933
:10E96000AE8429C41442854703C7060063E0E70A62
:10E9700083479400094681496380C702B307F74083
:10E98000A304E400B339F00083C716002305F400A4
:10E9900097900000E780A01E03572403058B19C73A
:10E9A0006386090097D00000E78000E921649305A1
:10E9B0008402280097B0FFFFE780801097000000D6
:10E9C000E78040F4AA85280097D0FFFFE78000F495
:10E9D00097000000E78080F5AA85280097D0FFFF08
:10E9E000E780C0F2014781463000A6854A8597B08E
:10E9F000FFFFE780403213047402480822CC230A48
:10EA0000010002CE97E0FFFFE780E0D605611733F3
:10EA1000FFFF6700236B1733FFFFE7020369011154
:10EA20007C003ECAB70708003ECC7C003ECE83C7C0
:10EA300095002E84AA8493F7F707A384F500A165B7
:10EA400093858502480897B0FFFFE780600797002D
:10EA50000000E78020EBAA85480897D0FFFFE780F9
:10EA6000E0EA97000000E78060ECAA85480897D0AC
:10EA7000FFFFE780A0E9500801478146A28526856F
:10EA800097B0FFFFE780202905611733FFFF67007C
:10EA900003649777FF1F9387E7189C43014599C349
:10EAA00003C5B70082801733FFFFE702036001113F
:10EAB000B70707003EC683C79500404D0AC493F7C9
:10EAC000F7070AC8A384F5002A89AE8405C81C424A
:10EAD000054783C707006368F7060347B400630F61
:10EAE000F700A305F40097900000E78040098347F2
:10EAF000B400B9CF97D0FFFFE78040BE21649305F3
:10EB0000B400280097B0FFFFE78080FB970000006B
:10EB1000E78060F8AA85280097D0FFFFE78000DF34
:10EB2000014781463000A6854A8597B0FFFFE78000
:10EB3000801E2904480822CC230A010002CE97E057
:10EB4000FFFFE78040C305611733FFFF67002358CD
:10EB500097D0FFFFE78020BF55B71733FFFFE702CD
:10EB6000C35401117C003ECAB70707003ECC7C00AD
:10EB70003ECE83C795002E84AA8493F7F707A3841B
:10EB8000F500A165AD05480897B0FFFFE78040F3A9
:10EB900097000000E78020F0AA85480897D0FFFF83
:10EBA000E780C0D6500801478146A285268597B0E8
:10EBB000FFFFE780401605611733FFFF6700235111
:10EBC0009777FF1F938707069C43094599C303C5A1
:10EBD000C70082801733FFFFE702234D01117C003D
:10EBE000AE843ECAA165B70707002A843ECCD10592
:10EBF0007C0048083ECE97B0FFFFE78060EC9700AE
:10EC00000000E78020FCAA85480897D0FFFFE78036
:10EC1000E0CF500801478146A685228597B0FFFFC7
:10EC2000E780600F05611733FFFF6700434A173322
:10EC3000FFFFE702834783C7950093F7F707A38495
:10EC4000F50097000000E78020F91733FFFF670009
:10EC500003481733FFFFE702A34383C79500032947
:10EC6000C501411193F7F707A384F5001C4283C93E
:10EC70000700854763E637079777FF1F9387C751DC
:10EC80009C432E84AA8485CF97000000E78080F300
:10EC900089476306F502630409028347C90063805C
:10ECA00037032306390197900000E78040ED835732
:10ECB0002903898B89C797D00000E780E0B72685B4
:10ECC000A28597000000E78020F1A167CD074800EA
:10ECD0003EC42302010002C697E0FFFFE780A0A91F
:10ECE00041011733FFFF6700E33D9777FF1F9387CD
:10ECF00067F39C431D4599C303C5E7008280173322
:10ED0000FFFFE702833A0111B70707003EC683C73A
:10ED10009500584D0AC493F7F7070AC8A384F50075
:10ED20002A89AE8415C71C4283C7070093968701C2
:10ED3000E18663C4060685466381D7068346E700FD
:10ED40006388F6002307F70097900000E78020E330
:10ED500021649305E400280097B0FFFFE78040D6C8
:10ED600097000000E780A0F8AA85280097D0FFFF51
:10ED7000E780C0B9014781463000A6854A8597B033
:10ED8000FFFFE78040F93504480822CC230A010040
:10ED900002CE97E0FFFFE780009E05611733FFFF7B
:10EDA0006700E3321733FFFFE702233001117C00D5
:10EDB0003ECAB70707003ECC7C003ECE83C7950015
:10EDC0002E84AA8493F7F707A384F500A165B905FB
:10EDD000480897B0FFFFE780A0CE97000000E780CB
:10EDE00000F1AA85480897D0FFFFE78020B25008BD
:10EDF00001478146A285268597B0FFFFE780A0F1F5
:10EE000005611733FFFF6700832C1733FFFFE7020D
:10EE10002328AA8401441779FF1F1309E9E0E14977
:10EE200097C0FFFFE78040C96344A400014519A8CB
:10EE300033053403832709003E95835725006397E4
:10EE4000970011051733FFFF6700C3270504C9BFEB
:10EE5000032E8500630A0E121773FF1F130383FB33
:10EE60000323030063150300294363900612032361
:10EE70004E01631503001D43639907101733FFFF0D
:10EE8000E7022320C689428A3E89BA8AB684328B39
:10EE9000AE8B2A84B5E103554E0019E501431A856E
:10EEA0001733FFFF67006321A167A98F116763FB19
:10EEB000E70097000000E78080F5814597F0FFFFAD
:10EEC000E780C0120844B70700E05841F98F1845A1
:10EED0005CC1B707001FF98F1CC55C4991C761056C
:10EEE00097E00000E780408BE38A09FA228597903B
:10EEF0000000E78060C65DB7328597C00000E780FC
:10EF000040430D4349DD1C44116703D54700A16709
:10EF1000A98F63FBE70097000000E78040EF814581
:10EF200097F0FFFFE780800C0323840093164B01CA
:10EF3000D1828347B300035663008588FD8BA30508
:10EF4000F300FD777D8E558EFD76FD16B204F18EB1
:10EF500083274301C58E231273012313D300230497
:10EF6000530123052301A3044301BDDF228597B08C
:10EF7000FFFFE78020CDAA850844B5D1610597D071
:10EF80000000E780207F8DB71D431A8582801733EC
:10EF9000FFFFE702E30F0569AA84AE89328A0144C4
:10EFA000FD5A7D1997C0FFFFE780C0A56347A40005
:10EFB00001451733FFFF6700E310D844931714008F
:10EFC000BA9703D70700631F3703239057016307DE
:10EFD0000A00268597900000E780A0809C449DC38E
:10EFE00083D76700B3F72701639E3701D2880148B2
:10EFF00081470147814601468145268597000000EB
:10F00000E78040E5050479BF1733FFFFE7024308B7
:10F0100079711C103EC4B7070F003EC61C103EC8D5
:10F0200083C79500AA8A328593F7F707A384F50072
:10F030002E89328497D0FFFFE780009D931705014A
:10F04000C187635AF006AA89228597D0FFFFE7801F
:10F05000A09B2A8A4E85032B040097B0FFFFE78010
:10F06000009B39ED8357440081440544F11793B761
:10F070001700A303F10083457100DA872287D28647
:10F080004E86280097E0FFFFE780E0570147814662
:10F090003000CA85568597B0FFFFE780C0C7A167DB
:10F0A0009387F70348083ECC230A810026CE97D0E9
:10F0B000FFFFE780406C45611733FFFF6700830067
:10F0C000A2851306710097E0FFFFE7806066AA84BF
:10F0D000094455D1528597E0FFFFE78060D40D4485
:10F0E00059D90546D285268597000000E78060EA59
:10F0F0002A8451B71733FFFFE70223FB835507002C
:10F100000346270041112A842E8532C62EC497E07B
:10F11000FFFFE780E0D001C93246A2452285970073
:10F120000000E78000E741011733FFFF670023FA83
:10F130001733FFFFE702E3F483C795004111AA8A62
:10F1400093F7F707A384F5003285AE89328497D010
:10F15000FFFFE780608B93170501C1876357F00AB3
:10F16000C1452A8A228597C0FFFFE78080702A8DDB
:10F17000228597D0FFFFE78020892A89228597D0B2
:10F18000FFFFE7804086930705F893F7F70F130713
:10F19000E007AA8B637BF706228597D0FFFFE78005
:10F1A00080842A8C228597D0FFFFE780C083AA8CB9
:10F1B0005285032B040097B0FFFFE780408539E9B3
:10F1C00083574400231101008144F11793B71700BE
:10F1D000A300F100054403471100835621009387E3
:10F1E00084005685DA8822885286CE8597F0FFFF04
:10F1F000E78020A7A167E90748003EC423028100F9
:10F2000026C697D0FFFFE780005741011733FFFF65
:10F210006700A3EA13061100A28597E0FFFFE780CD
:10F220002051AA8409E52311010009446DB7930513
:10F2300021006A8597F0FFFFE780A0F02A8441FD56
:10F24000835521009356C9001316490185486688E5
:10F25000E2875E87858A5182268597000000E780D5
:10F2600060BF2A848DBF1733FFFFE70283E183C7A6
:10F27000950041112A8B93F7F707A384F500328597
:10F28000AE89328497C0FFFFE780007893170501AD
:10F29000C1876352F00A2A8A228597C0FFFFE78060
:10F2A000A076AA8A228597C0FFFFE780E0752A89A9
:10F2B000228597C0FFFFE7800073930705F893F757
:10F2C000F70F1307E0072A8C6377F706228597C0AC
:10F2D000FFFFE7804071AA8C228597C0FFFFE7807F
:10F2E00080702A8D5285832B040097A0FFFFE78052
:10F2F000007239E58357440085440144F11793B700
:10F300001700A301F10003473100930784005A85D9
:10F31000DE882688D6865286CE8597F0FFFFE78066
:10F3200040948D4748003EC42302910022C697D0E6
:10F33000FFFFE780404441011733FFFF6700E3D739
:10F34000A2851306310097E0FFFFE780603E2A8424
:10F35000894455D99356C9001316490185486A88CE
:10F36000E6876287858A5182D68597000000E7800C
:10F3700060AEAA8449BF1733FFFFE70263D12A8931
:10F3800081440144617A916A177BFF1F130B8BA89C
:10F3900097B0FFFFE780006863C7A400228517339A
:10F3A000FFFF670023D28327090093991400CE97AB
:10F3B00003D50700330745014207418363645703C0
:10F3C00005C103270B0019C785453E8597400000FE
:10F3D000E78060E9832709000504CE9723900700A2
:10F3E00085047DB797000000E78060A283270900AD
:10F3F0000504CE972390070065D5814597F0FFFF60
:10F40000E780C0BEF1BF1733FFFFE70263C883C7C1
:10F41000950041112A8A93F7F707A384F5003285F6
:10F420002E89328497C0FFFFE780005E93170501A5
:10F43000C187635AF004AA89832A040097A0FFFFBA
:10F44000E780E05C31E58357440085440144F117CF
:10F4500093B71700A301F10003483100D687528506
:10F460000147CE862686CA8597D0FFFFE780806A4F
:10F47000A167F50748003EC42302910022C697D039
:10F48000FFFFE780402F41011733FFFF670083C371
:10F49000A2851306310097E0FFFFE78060292A84E8
:10F4A00089445DD99777FF1F9387C7969C4381CF87
:10F4B000044997B0FFFFE780E055AA85268597406D
:10F4C0000000E78040DA1305040197000000E780A0
:10F4D000C0EA228597800000E78000338144ADBFF9
:10F4E0001733FFFFE702E3B983C795004111AA8AEA
:10F4F00093F7F707A384F5003285AE893284231190
:10F50000010097C0FFFFE780205093170501C187D6
:10F510006354F0062A8AC145228597C0FFFFE78021
:10F520004035AA8B5285032B040097A0FFFFE7808C
:10F53000004E21E98357440085440144F11793B7F5
:10F540001700A300F1000348110003572100DA87D8
:10F550005685D2862686CE8597D0FFFFE780805BD2
:10F56000A1679387270248003EC42302910022C668
:10F5700097D0FFFFE780202041011733FFFF67008E
:10F58000C3B3A2851306110097E0FFFFE780401A7E
:10F590002A8489444DD99777FF1F9387A78798437B
:10F5A0003E8901CF044997B0FFFFE780A046AA85B6
:10F5B000268597400000E78000CB130504019700E3
:10F5C0000000E78080DB97B0FFFFE780A044954410
:10F5D0003DD9930521005E8597F0FFFFE78060B677
:10F5E000AA8435F11C480357210022852390E700A7
:10F5F00097800000E780402183270900A9D70355A1
:10F60000210097400000E780A0BD35BF1733FFFF02
:10F61000E70223A783C795004111AA8A93F7F7074A
:10F62000A384F5003285AE89328497C0FFFFE7805E
:10F63000A03D93170501C1876351F0062A8A2285F0
:10F6400097C0FFFFE780403C2A895285032B0400C6
:10F6500097A0FFFFE780A03B31E583574400854436
:10F660000144F11793B71700A301F10003483100DB
:10F67000DA8756854A87D2862686CE8597D0FFFFC1
:10F68000E7804049A167F90748003EC42302910082
:10F6900022C697D0FFFFE780000E41011733FFFF1E
:10F6A0006700A3A1A2851306310097E0FFFFE78062
:10F6B00020082A8489445DD99167CA97C2071167D7
:10F6C000C1831307F7EF8544E362F7FA9767FF1FDB
:10F6D000938747749843BE8B01CF044997B0FFFFCF
:10F6E000E7804033AA85268597400000E780A0B7D1
:10F6F0001305040197000000E78020C897B0FFFFC2
:10F70000E780403195443DD11C48228581442390B7
:10F71000270197800000E780200F83A70B00B9D74F
:10F720004A8597400000E780A0AB89B71733FFFFF9
:10F73000E702A3972A844105B28497000000E7807E
:10F74000C0C311C5228597800000E780E00B814689
:10F750000146A685228597800000E780C04E1C4C9C
:10F7600089C7DC4799C3228582971733FFFF67005B
:10F7700003969767FF1F9387E74A9C43014599C308
:10F780001385070182809767FF1F9387A7498843E6
:10F7900082801733FFFFE70243919317C600DD8D88
:10F7A000C2054111C1812A8432C697C0FFFFE7809C
:10F7B000E0173246228511829375F60F97C0FFFF3E
:10F7C000E780C01441011733FFFF670043901733F0
:10F7D000FFFFE702E38B79713C083ED2B7070C00CC
:10F7E0003ED43C083ED683C79500AE842A8993F761
:10F7F000F707A384F500A16593853504481097A009
:10F80000FFFFE780E02BC165FD150144176AFF1F6C
:10F81000130ACA61930A400EAE892E8B2EC697B08A
:10F82000FFFFE78020224205931704014181C18335
:10F83000B24563E9A702C167FD176387F500481069
:10F8400097C0FFFFE780800E501001478146A685D4
:10F850004A8597A0FFFFE780004C45611733FFFF03
:10F86000670043863307540383270A0BBA9703D6EE
:10F87000C701630A3601638A35014810970000000A
:10F88000E78060F1DA85050451BFB285EDBF17232B
:10F89000FFFFE702037F79717C083EC8B7071100BC
:10F8A0003ECA7C083ECC83C79500AA89328593F76F
:10F8B000F707A384F5002E8997C0FFFFE780C014E7
:10F8C00085676378F504A165AA848905080897A06F
:10F8D000FFFFE780E01E268597400000E78060ED8F
:10F8E000133415000A04A285080897C0FFFFE780BB
:10F8F000E001A685080897C0FFFFE780200325CC1C
:10F90000014781461008CA854E8597A0FFFFE78012
:10F91000804045611723FFFF6700237AB307540334
:10F920000327CA0ABA9703D70700631C970003D6B8
:10F93000270063806505080897000000E780A0E5C0
:10F94000DE8505042EC697B0FFFFE780A0104205B4
:10F95000931704014181C183B245E3E1A7FCC1676C
:10F96000FD17E38FF5F8080897C0FFFFE78000FC5C
:10F9700041BFB285F9B7C165FD150144176AFF1F84
:10F98000130ACA4A930A80022E8BAE8B65BF1723D7
:10F99000FFFFE70283711841834717008346070082
:10F9A000A207D58FD207D1832390F5008347270084
:10F9B000034717008D45A207D98F91832310F600C6
:10F9C00097C0FFFFE780A0E91723FFFF67002370C0
:10F9D0001723FFFFE702C36BC16401441769FF1FD0
:10F9E0001309C94493098002FD1497B0FFFFE78013
:10F9F00060066347A40001451723FFFF6700836C7F
:10FA0000330534038327C90A3E9583570500E385F0
:10FA100097FE0504D9BF1723FFFFE70263672A8A11
:10FA2000AE89B284B68A97400000E78080D819E595
:10FA300091473E851723FFFF6700C3682A894E85DB
:10FA400097C00000E780E08E2A84638E0A048D4709
:10FA50006DD103570500C547E31D47FD0347F90175
:10FA60008546AD47E317D7FC8347450081CF414624
:10FA7000A6855D0597F00000E780C09E814755D9B7
:10FA8000AD4745BF130965012302E500CA852685F8
:10FA900097100000E780606231C1A547E38B0AF848
:10FAA0002302040079B705C183570500E39247F9A3
:10FAB0004146A685190597F00000E780A09A814786
:10FAC0002DD99947BDB74E8597000000E78080F09B
:10FAD0002A84954739DD130955004DBF4146A68557
:10FAE00023104401231134011305190097F000007D
:10FAF000E780A099228597800000E780A0EA8147EF
:10FB00000DBF1723FFFFE702435A79717C003ECCFB
:10FB1000B7070A003ECE7C003ED083C79500B28472
:10FB20002E8493F7F707A384F5001306A1002A8912
:10FB30002C00268597000000E780A0E5A165280835
:10FB40008D0597A0FFFFE780A0F790408355A100A7
:10FB500003558100854697000000E78000ECAA84E9
:10FB6000AA85280897C0FFFFE78040DA0356A10066
:10FB700083558100280897000000E780C0C1300845
:10FB800001478146A2854A8597A0FFFFE780A0181C
:10FB9000854748103ED42302910202D697D0FFFF3A
:10FBA000E78060BD45611723FFFF670043521723BD
:10FBB000FFFFE702834F79717C003ECCB7070A0054
:10FBC0003ECE7C003ED083C79500B2842E8493F74E
:10FBD000F707A384F5001306A1002A892C002685C7
:10FBE00097000000E780E0DAA16528088D0597A05E
:10FBF000FFFFE780E0EC90408355A10003558100B2
:10FC0000814697000000E78040E1AA84AA85280881
:10FC100097C0FFFFE78080CF0356A1008355810086
:10FC2000280897000000E78000B7300801478146A8
:10FC3000A2854A8597A0FFFFE780E00D48102302C8
:10FC4000910202D402D697D0FFFFE780C0B245618F
:10FC50001723FFFF6700A3471723FFFFE702E344D3
:10FC600097000000E78060DB1723FFFF6700234653
:10FC70009767FF1F938747FB884382801723FFFF07
:10FC8000E702A342835725004111AE842A8423074B
:10FC9000B10017F5FFFF130525466C002316F10090
:10FCA00097A0FFFFE780204991C42285978000003C
:10FCB000E780E0D6FD572310F400130620028145AB
:10FCC000130554009720FFFFE780204141011723CF
:10FCD000FFFF6700C33F1723FFFFE702633B797114
:10FCE0007C003ECCB7070A003ECE7C003ED083C7E6
:10FCF0009500AA89AE8493F7F7073285A384F500AF
:10FD00001306A1002C0097000000E78080C803556F
:10FD10008100114497400000E780A0A915C5035554
:10FD2000A100014497B00000E780A06011CD035707
:10FD300005008357810045446318F7008545970007
:10FD40000000E780E0F301442169930539002808A9
:10FD500097A0FFFFE780C0D6A285280897C0FFFFC5
:10FD6000E780C0BA0356A100835581002808970098
:10FD70000000E78040A2300801478146A6854E85F5
:10FD800097A0FFFFE78020F948104AD423028102A0
:10FD900002D697D0FFFFE780009E45611723FFFF43
:10FDA000670043321723FFFFE702832E9767FF1F89
:10FDB000938747E72A8488432E8915C5035745034F
:10FDC0008357C4016311F702232605022318050295
:10FDD000410597D00000E780209C630609009780CA
:10FDE0000000E78060DB81449769FF1F9389090465
:10FDF000130A800297B0FFFFE780C0C563C4A40464
:10FE00009767FF1F9387C7EA9C4399C70355C401AF
:10FE100097200000E780C0BD630709002285978016
:10FE20000000E780C0A01306400E81452285972080
:10FE3000FFFFE780802AFD57231EF4001723FFFFF2
:10FE4000670043283385440383A7C90A3E950357B7
:10FE500005008357C4016317F700CA8597000000A7
:10FE6000E78000E2850479B71723FFFFE70243220A
:10FE700083C795004111AA8993F7F707A384F5007A
:10FE80003285AE8497C0FFFFE78000B8856763784E
:10FE9000F5042A8997400000E780A091014401CD34
:10FEA00083D704003144638827018545970000000B
:10FEB000E78080EF01444E85A2864A86A68597D0CA
:10FEC000FFFFE780A09CA1679387170448003EC40A
:10FED0002302810002C697D0FFFFE780C08941015D
:10FEE0001723FFFF6700031E1723FFFFE702431AD4
:10FEF0009767FF1F938707D3804329C4014597C0A5
:10FF00000000E780002181470148C1641CDC232EEA
:10FF10000403232004041769FF1F130929F1014476
:10FF20009309400EFD1497B0FFFFE780A0B1634F27
:10FF3000A400814517F5FFFF1305857F97A0FFFFFC
:10FF4000E780601F1723FFFF6700C31733053403E3
:10FF50008327090B3E958357C50163879700854525
:10FF600097000000E78040E4050475BF9357050142
:10FF700013D78700A380F50093170501C183A183E0
:10FF80002380E5002381F500A381A500828017234B
:10FF9000FFFFE70283112300050083C71500A300BC
:10FFA000F50083C725002301F50083C73500A301B1
:10FFB000F50083C745002302F50083C75500A3025F
:10FFC000F50083C7650093059500A303050023038F
:10FFD000F50023040500328597000000E78040F912
:10FFE0001723FFFF6700A30E1723FFFFE702430A53
:10FFF0004111E9540DCD85CD93F9C5FF2E842A8991
:020000040001F9
:10000000AA84338AA900B7EA040063189A020D880B
:10001000854411CCB7E704009C5F82972AC62286EC
:100020006C003305390197E00000E7800046268523
:1000300041011723FFFF6700E30883A78A039104A8
:10004000829793170501C183A183A38EF4FE935772
:100050000501238FF4FEA183238EA4FEA38FF4FE5B
:100060006DB763E6D5021723FFFFE7020304B287EB
:1000700041113686BE8536C697E00000E780E04035
:10008000B246410136851723FFFF670043048146CE
:1000900036858280838705001387F5003D05FD873F
:1000A00093F77708834607007D158606B58FA30072
:1000B000F5006307B7007D17834717009D83DDB701
:1000C00082801723FFFFE70243FEB7E7040083A700
:1000D000070932872A863A85829713351500172338
:1000E000FFFF6700C3FE15C181478DC11723FFFFC6
:1000F000E702A3FB414697E00000E780003985470F
:100100003E851723FFFF670083FC81473E85828081
:100110001DCD1723FFFFE70243F9414681452A849D
:100120009720FFFFE78060FB4146814513050403EC
:100130009720FFFFE78060FA0147C167232204048C
:1001400038C87CC805451723FFFF670043F8014501
:10015000828081473DCDB5CD1723FFFFE702E3F451
:10016000B2842E891306800581452A849720FFFFDB
:10017000E780A0F6CA8524C4268597000000E780A2
:10018000C0F64146814522859720FFFFE780E0F4D5
:100190003044A285228597000000E780C0F29304D6
:1001A0000401A285268597000000E780E0EEA68581
:1001B0001305040297000000E78000EE22859700F7
:1001C0000000E78020F585473E851723FFFF670085
:1001D00003F03E8582801723FFFFE70263EB4111A6
:1001E000E9540DCD85CD93F9C5FF2E842A89AA84C3
:1001F000338AA900B7EA0400639844030D88814458
:1002000011CCB7E704009C5F82972AC622866C0057
:100210003305390197E00000E7802027268541015A
:100220001723FFFF670003EA83A78A0391048297DD
:1002300093170501C183A183A38EF4FE9357050193
:10024000238FF4FEA183238EA4FEA38FF4FE6DB74B
:1002500065CD1723FFFFE702A3E3B28411E605454E
:100260001723FFFF670003E62A842E890145EDD995
:100270003C487848B3E6E700E5D69386F7FFB3B786
:10028000F6007D17032A4404BA9734C87CC8630576
:100290000A06C14913050A03B38949412295637DC2
:1002A0003601B2862E86A68597000000E780A0DB87
:1002B0007C40BE9464C065B7CE862E86CE859700FE
:1002C0000000E78040DAC114D2944E99232204043E
:1002D000A2879306040103C7070003C60703850727
:1002E000318FA38FE7FEE398F6FE3044A285228586
:1002F00097000000E78020DD2699C1493306994028
:1003000063EC9900A9DCA686A68513050403970073
:100310000000E78040D579BF8147B306F40033077A
:10032000F6000347070083C5060085072D8F23804D
:10033000E600E39437FF3044A28522859700000051
:10034000E78060D8C1145DBF014582800DC11723CD
:10035000FFFFE70283D51306800581459720FFFF45
:10036000E780A0D705451723FFFF670043D6014567
:100370008280814749C5C1C51723FFFFE702E3D249
:10038000FC4141462E84AA846399C7041386050163
:10039000A2878146C14503C7070003C50703850738
:1003A000298F3305D600034505008506298FA38FC5
:1003B000E7FEE392B6FE3044A28526859700000052
:1003C000E78060D0228597000000E78060F88547CD
:1003D0003E851723FFFF670083CF138507031D8E1C
:1003E000814522959720FFFFE78020CF7C401307AF
:1003F00000F813060402A2972388E70251BF3E8546
:1004000082801723FFFFE70243CA6D712E84B284F6
:10041000AA8590102800368997000000E780A0D3B5
:1004200009EDD55725A050400C402800970000004A
:10043000E78040E27DD5FD142104F5F42C004A85C7
:1004400097000000E78020F3814761DD3E85516120
:100450001723FFFF6700A3C71723FFFFE702E3C4CB
:1004600041112EC432C62C00054697000000E780DB
:1004700080F941011723FFFF670063C51723FFFFC2
:10048000E702A3C201112A842EC602C802CA02CC06
:1004900002CE97E00000E780402BB2462A86A28574
:1004A000080897000000E78060FB1375F50F0561F1
:1004B0001723FFFF6700A3C11723FFFFE702E3BE77
:1004C0007971B2872A8421462308B10013051101EE
:1004D000BE853AC436C697E00000E78000FBB2460E
:1004E00093059101368597000000E78060A822857A
:1004F000141035460C0897000000E78020F62A8487
:10050000224701E921460C103A8597E00000E78078
:10051000C0F7228545611723FFFF670043BB172300
:10052000FFFFE70283B87171AE84AA850A85328421
:1005300097000000E78060BB11C90A86A685228566
:1005400097000000E78020B8814711E1C5473E854C
:100550004D611723FFFF670083B71723FFFFE702F3
:10056000C3B11D712A8AB289BE84354685471305F9
:1005700011012E8CB68A3A8BC28C468D2308F1006D
:1005800097E00000E78060F010100C085285231FF0
:10059000010097000000E780C0F82A843DEDA147E4
:1005A0006313FD089307900591E0E5473546E28522
:1005B0001305110113990A012308F10013590901C8
:1005C00097E00000E78060EC1357890093978A005A
:1005D000D98F90080C085285231FF1009700000066
:1005E000E78020F42A8415E9A1E49387FA00918337
:1005F0001379F9003EC6631309004149668B8144B3
:10060000C14B854DB247639F970C6A868C0033853A
:100610005C0197E00000E78040E722852561172311
:10062000FFFF670043A993079004C9F0A547BDBF2A
:10063000834701050947C14B2308F1008347110592
:10064000A58FA308F10093872400814463E1FB0494
:10065000014714083386E6008C08B386E400BA9597
:10066000DA9683C6060083C505000507AD8E230014
:10067000D600E390E7FE4147639CE70490080C082E
:10068000528597000000E780C0E925D181A0B3061C
:100690009B00BA871008B305F60090083E9603C584
:1006A00006000346060085078506298E2380C500BF
:1006B000E39277FF998F90080C085285BE949700BB
:1006C0000000E78000E68947014749D12A84B1B795
:1006D00090083E96034606001408BE962380C60086
:1006E000850759BFB2478504638797148147180867
:1006F000B306F70098083E973386F90003470700D2
:10070000034606008507318F2380E600E39177FFDB
:1007100090080C08528597000000E78080E05DF5A6
:100720003546E285130511012308B10197E0000069
:10073000E780A0D513970401418393978400218318
:10074000D98F10180C085285231FF1009700000064
:10075000E78020DD25FD814710183387F9003E969C
:100760000347070003460600B306FB008507318FE9
:100770002380E600E39277FF65A81808B306F70028
:1007800098083E973386F9000347070003460600A2
:100790008507318F2380E600E3E127FFCA87639E48
:1007A000770990080C08528597000000E78060D711
:1007B00011FD81479800B306F700900818103E9786
:1007C0003E9603470700034606008507318F2380C6
:1007D000E600E39177FF3546E28513051101230812
:1007E000B10197E00000E78040CA139704014183FC
:1007F000939784002183D98F10180C085285231FEA
:10080000F10097000000E780C0D1E31105EC8147BB
:1008100010183387F9003E96034707000346060089
:10082000B306FB008507318F2380E600E3E227FF54
:10083000C109410BC1BB814785B79408BE9683C6E9
:10084000060018083E972300D700850789BF6380FC
:1008500006321723FFFFE702438259712A84BE89BB
:10086000B28B85473546130511022E8B468C428983
:10087000BA8A368A2300F10297E00000E780E0C0E0
:1008800010180C1022852317010297000000E78042
:1008900040C963180512A147631FFC069307900522
:1008A00063930900E5473546DA8513051102931471
:1008B0000A012300F102C18097E00000E780E0BC5C
:1008C00093178A0013D78400D98F90080C102285C3
:1008D0002317F10297000000E780A0C47DE1639236
:1008E00009049307FA00BD88918391E0C144C207CF
:1008F000C183DE8C814A3EC6414DB24763E2FA0EA7
:100900006286B3854B01881097E00000E78080B5D0
:100910004DC93D557DA093079004E39609F8A5477E
:1009200059B7834701050947C14C2300F1028347AA
:100930001105B3C7F900A300F1029387290081498B
:1009400063E1FC04814618103306D7008C08338716
:10095000D900B69556970347070083C5050085065D
:100960002D8F2300E600E390D7FE41476390E70612
:1009700090080C10228597000000E78080BA35D1DE
:1009800089A0B3863A01BA871010B305F600900823
:100990003E9603C506000346060085078506298E98
:1009A0002380C500E39297FF3387EC4090080C103A
:1009B0002285BA9997000000E780A0B689470147D1
:1009C00041D165611713FFFF6700E36E90083E9603
:1009D000034606001410BE962380C600850779B72B
:1009E000B247850A93990A01939D8A0093D9090118
:1009F0006391570F85473546DA85130511022300A9
:100A0000F10293D9890097E00000E78000A8B3EDD8
:100A10003D0190000C1022852317B10397000000C0
:100A2000E78020B059FD8147A68963EA97062686AC
:100A30000C084A8597E00000E78020A58147181040
:100A4000B306F700100898083E973E960347070044
:100A5000034606008507318F2380E600E3E197FE19
:100A6000639FA90590080C10228597000000E7807D
:100A700040AB21F981479810B306F7009008181889
:100A80003E973E9603470700034606008507318FD1
:100A90002380E600E391A7FF4109C10CB9BD180806
:100AA0009000B306F7003E963387FC00034707002B
:100AB000034606008507318F2380E600B5B7980806
:100AC0004E97034707001C10CE972380E700850947
:100AD00041BF85473546DA85130511022300F1022F
:100AE00093D9890097E00000E780209AB3ED3D019B
:100AF00090000C1022852317B10397000000E780B7
:100B000040A2E31005EC814718089000B306F700F7
:100B10003E963387FC00034707000346060085071F
:100B2000318F2380E600E391A7FF41460C084A85F8
:100B300097E00000E780609581471810B306F70042
:100B4000100898083E973E960347070003460600A4
:100B50008507318F2380E600E391A7FF90080C10F2
:100B6000228597000000E780C09B1DD599BD7D556B
:100B700082801713FFFFE702435301112A842E8559
:100B800093055100328902C002C202C402C6930416
:100B9000740097F0FFFFE780A03D1D46A685130572
:100BA000910097E00000E780408E10088A854A8512
:100BB00097000000E780E09619ED930714001808ED
:100BC00083C607000346070085070507B18EA38F7C
:100BD000D7FEE397F4FE05611713FFFF6700234F6D
:100BE0001713FFFFE702C34A2E848C414111AA89E3
:100BF000838715003289914463D30700A144975736
:100C0000FF1F938767599C43A1C7C1CA8D47231013
:100C1000F10083C725004A852301F10083C7350011
:100C2000A301F10083C745002302F10083C75500EB
:100C3000A302F10083C7650093059100A30301009F
:100C40002303F1002304010097F0FFFFE780403207
:100C50000C404A860A8597F0FFFFE780803303281F
:100C6000040083564400A6881D0881470147E51605
:100C700042868A854E8597000000E780408E2A894B
:100C800019E5A685228597B0FFFFE780E0C14A8578
:100C900041011713FFFF6700E3424A860A8597F078
:100CA000FFFFE780002F6DB71713FFFFE702433EFA
:100CB0002E848C414111AA89838715003289914481
:100CC00063D30700A1449757FF1F9387E74C9C43CA
:100CD000A1C7C1C68D472310F10083C725004A85EF
:100CE0002301F10083C73500A301F10083C745004C
:100CF0002302F10083C75500A302F10083C76500FA
:100D000093059100A30301002303F10023040100D4
:100D100097F0FFFFE780C0250C404A860A8597F0D0
:100D2000FFFFE780002783564400032804008A85DC
:100D3000858EC2061D08C1822312D400A688814771
:100D40000147E51642864E8597000000E78060B0B7
:100D500041011713FFFF6700E3364A860A8597F0C3
:100D6000FFFFE78000234DBF1713FFFFE702E333C8
:100D7000B335B000011185052A891315F6013365D5
:100D800015012308B1009305110136843AC632C01B
:100D90003EC442C297F0FFFFE780801DA247124881
:100DA000425593D68700230BF10093059101935789
:100DB0008800A30AD100A30BF100230C010197F0D6
:100DC000FFFFE780E01A3247024603280400B337EA
:100DD000E000835644009207914411C2A1444A8521
:100DE000A68842860C0897F0FFFFE78040772A89A3
:100DF00019E5A685228597B0FFFFE780E0AA4A851E
:100E000005611713FFFF6700832C1713FFFFE7022D
:100E1000232801113EC68647B335B0008505AA894F
:100E20001315F6015D8D2308B10093051101368479
:100E30003A89B28442C446C297F0FFFFE78040136C
:100E400022489248164593578800A30AF10093055B
:100E5000910193D78800230B0101A30BF100230C10
:100E6000110197F0FFFFE780A01032471040835632
:100E70004400B337E000920703280900914891C06D
:100E8000A1480C084E8597000000E780809CAA844A
:100E900001E9835544004A8597B0FFFFE780C0A071
:100EA000268505611713FFFF6700C321AA959307E5
:100EB000F00F171701001307A7986317B50013C5A4
:100EC000F7FF1375F50F828005058346F5FFB58F93
:100ED000BA9783C70700D5B7035745001441930756
:100EE000F00F171601001306A695369742074183A7
:100EF000139506014181631BE500AD8FB29703C5D1
:100F00000700130515F3133515008280850603C508
:100F1000F6FFA98FB29783C70700D9BF1713FFFF4A
:100F2000E702A318B28736842E86BA86AA853E8544
:100F3000BA8497F0FFFFE7806052634F0500228577
:100F400097E00000E78060802A86A686A285268535
:100F500097F0FFFFE78080501713FFFF670023170C
:100F60001713FFFFE702C3125D712A8BAE8A1715B4
:100F700001001305658A2C00B284368ABA893E893D
:100F800097F0FFFFE780C04F2A845DE134104146AF
:100F9000DA85280097F0FFFFE780404C2A8449E972
:100FA0008547A303F100A6C2930771002408BEC4BD
:100FB000A68685470D462C18281002DC02DED6C016
:100FC000BEC697F0FFFFE78000442A8435E18347DF
:100FD0007102A6860D4693F7F7072300FA00C14772
:100FE0003EDE2C188947281026DCA303F10097F079
:100FF000FFFFE78040412A8405ED4146A6854E85E6
:1010000097D00000E78060488D47A6860D462C18D3
:101010002810A303F10097F0FFFFE780C03E2A8469
:1010200001E94146A6854A8597D00000E780E04562
:10103000228561611713FFFF6700C3081713FFFFC5
:10104000E702A30697F70000938707EF984383C74B
:10105000470079712A89AE84170501001305457C84
:101060000C083AC42306F10097F0FFFFE7804041E7
:101070002A8405ED14104146CA85080897F0FFFF41
:10108000E780C03D2A8415E1140815462C0008109D
:1010900097F0FFFFE780803C2A8401E921462C0875
:1010A000268597D00000E780403E228545611713D2
:1010B000FFFF6700C3011713FFFFE70203FF97F766
:1010C0000000938767E79C477971AA842E841705EF
:1010D0000100130565750C083EC697F0FFFFE78019
:1010E000203A0DE914104146A685080897F0FFFF45
:1010F000E780C03605E1140811466C00081097F02F
:10110000FFFFE780A03519E58347F10193F7F70367
:101110002300F40045611713FFFF670043FB17131B
:10112000FFFFE70283F83688A14881470147E5467B
:1011300097F0FFFFE780A0421713FFFF670023F936
:101140001713FFFFE70263F63688A148814701477E
:10115000E54697F0FFFFE780C06F1713FFFF6700BA
:1011600003F71713FFFFE70243F401112A842E85CA
:101170000C0832C697F0FFFFE780803009ED324758
:10118000970601009386C6681008C145228597001E
:101190000000E780E0D805611713FFFF670023F325
:1011A0001713FFFFE70263F04111C1472EC032C49D
:1011B0008A8509463EC23EC697F0FFFFE780A0241D
:1011C00041011713FFFF670083F01713FFFFE702CA
:1011D000C3ED4111AE8613061009AA850A8502C027
:1011E00002C202C402C697F0FFFFE7802027410138
:1011F0001713FFFF6700A3ED1713FFFFE702E3EAF2
:101200003287970601009386A6622E869305000218
:1012100097000000E780C0D01713FFFF670023EBA3
:101220001713FFFFE70263E87971C1472ACC2ED07C
:1012300032D42C080D4628003ECE3ED23ED602C403
:1012400002C602C802CA97F0FFFFE780C01B4561D3
:101250001713FFFF6700A3E71713FFFFE702E3E49D
:101260000111AA842E84170501001305E55C8A8507
:1012700097F0FFFFE780C02015E514084146A685DA
:101280000A8597F0FFFFE780601D09ED8347E101C4
:101290000347F101A207D98FCA07C9836177D98FA4
:1012A0002310F40005611713FFFF670043E215CD1B
:1012B0001713FFFFE70263DF9757FF1F9387479BD3
:1012C00090439755FF1F9385E59A1755FF1F130508
:1012D000259697D00000E78000C51755FF1F13051E
:1012E00025951713FFFF670083DE1755FF1F1305B2
:1012F000259482808DCD1713FFFFE70203DB9757FC
:10130000FF1F9387E796944301112E840A86975511
:10131000FF1F9385259697D00000E78040C60A8579
:101320000294014505611713FFFF670043DA7D55FD
:1013300082801713FFFFE70243D797D00000E780B2
:1013400080D19757FF1F23A5A79217F5FFFF13051D
:10135000E5C997B00000E780C0741713FFFF67006E
:1013600003D71757FF1F1307E7929317150008437A
:101370003E95FD572310F50082801713FFFFE7020B
:10138000C3D22A84084009E51713FFFF670023D45E
:101390001C4158401CC06313E5005CC083475500E6
:1013A00023200500F99BA302F50097A0FFFFE7802B
:1013B000207CC9BF1713FFFFE70283CD9757FF1F9C
:1013C0009387478F98432A8411CB8347350093F73F
:1013D000070289C703550500894502971305440193
:1013E00097B00000E780403B835504000355E400BC
:1013F00097300000E780A00C485819C597A0FFFF60
:10140000E7800077232A0402130584039700000075
:10141000E780E0F68144B1499790FFFFE780C06D17
:1014200063CBA402834734002320040493F727FCF2
:10143000A301F40000489790FFFFE780E06C1316CB
:101440001500814522859710FFFFE78000C917131B
:10145000FFFF670023C7B387340303290403850410
:101460003E994A8597000000E78060F12304090057
:1014700065B78347350093F7070299E301458280FA
:101480008357E500E39CB7FEC167FD176316F600BE
:1014900005458280054599A81713FFFFE702E3C0C1
:1014A00093170601C187B2842A8401496359F00267
:1014B000835705009DCB01456367F6000345840013
:1014C0003E953325A6001375F50F0DA01C48131784
:1014D0001900BA9783D70700E38E97FA050997900A
:1014E000FFFFE7806062E343A9FE01451713FFFF9A
:1014F0006700E3BD1713FFFFE70283B9AE89AA8433
:101500009790FFFFE78000562A8497D0FFFFE7807F
:10151000A02EAA8601471306840197050000938533
:1015200085E41745FF1F130525779790FFFFE78098
:10153000801C2A8925C98C441304C50022859E0578
:1015400093F5050897A0FFFFE780403CCC408387D8
:101550007400E18163DD070493E50508228597A007
:10156000FFFFE780A03A0D4693854400228597A0AF
:10157000FFFFE780C03683D50400228597A0FFFFD8
:10158000E780E03D83D52400228597A0FFFFE78018
:10159000003D03D6490083A50900228597A0FFFFDF
:1015A000E780E0334A851713FFFF6700A3B193F587
:1015B000F5076DB71713FFFFE70223AF01112A8468
:1015C000328532C697A0FFFFE780E0279780FFFFB4
:1015D000E7806034835704001757FF1F1307078500
:1015E0003246231BF100930700F8A30DF1001C47BE
:1015F0001843231AA1008983858BB307F740B2856E
:1016000048083ECE231C0100230D01009700000076
:10161000E78080EE05611713FFFF670043AB1713E8
:10162000FFFFE702E3A6004101453DC49304C40067
:1016300026853289AE8997A0FFFFE780C0249545B3
:101640002A8A2685035B040197A0FFFFE7802021FB
:10165000268597A0FFFFE780603E8D45AA8A2685F4
:1016600097A0FFFFE780A01F268597A0FFFFE780D8
:10167000E03C5C48420A135A0A01D2975CC4231822
:101680006401814763983A0146054D81330625413F
:101690009337160013F5F70F1713FFFF670083A2A8
:1016A0001713FFFFE702E39D89692A8BAE8B328A0D
:1016B000B68A81440144314CFD199790FFFFE780C1
:1016C000A04363CDA4009790FFFFE780E045018D24
:1016D00033B5AA001713FFFF6700239E33898403E5
:1016E00083270B003E9963170A008347890085040E
:1016F0003E94E1B703560A00DE854A8533F6C900F9
:1017000097000000E780E0F16DD10545E1B71713C0
:10171000FFFFE702839901112A847C000355E5004D
:101720003ECAB70707003ECC7C003ECE97200000A3
:10173000E78020082A898545480897A0FFFFE780B1
:1017400020399945480897A0FFFFE780E015AA8453
:101750004A8597200000E780A0082380A4009747CF
:10176000FF1F9387A76C9C434166130606F0939670
:10177000870113D78701558F93D68700F18E558F38
:10178000A207B706FF00F58FD98F11462C001385ED
:1017900014003EC497D00000E78020CF5008A382F9
:1017A00004008945228597000000E780E0E019C920
:1017B000AA851305840397A0FFFFE780E0313C4032
:1017C00085073CC005611713FFFF6700439017139F
:1017D000FFFFE702838D9790FFFFE780E0342A84C4
:1017E00005049790FFFFE78020333305A402F147FB
:1017F00091453305F50297200000E78020BA11E5F6
:1018000065551713FFFF6700838C9747FF1F23ABB6
:10181000A7489790FFFFE78020312A84050497901E
:10182000FFFFE780602F3305A40289450605972056
:101830000000E780A0B669D59747FF1F23ACA744F7
:101840009790FFFFE780402E2A8405049790FFFFC2
:10185000E780802C3304A4029747FF1F239E874212
:101860009790FFFFE780402C2A849790FFFFE78046
:10187000A02A930714003385A7029747FF1F239ED2
:10188000A740970701009387E7BE1747FF1F23294B
:10189000F7400145BDB71703FFFFE702637FAA8446
:1018A0002E8901449749FF1F93894958130A8006DE
:1018B0009790FFFFE78040266347A4000145171378
:1018C000FFFF670023803305440383A709024A868C
:1018D000A6853E9597000000E780E0B919E1050470
:1018E000C1BF0545E9BF1703FFFFE7028379AA8A55
:1018F0002E8BB28B368C3A8A814401448149974CB5
:10190000FF1F938CAC52130D80069790FFFFE7806A
:10191000A02063C9A40011E085494E851703FFFF8D
:101920006700A3793389A40383A70C025E86D6855A
:101930003E994A8597000000E780E0B31DC197906B
:10194000FFFFE780601E0544636D4501D286628615
:10195000DA851305090397000000E780A0D411C1C0
:10196000854985045DB71703FFFFE7026372C16411
:1019700041112A8901449749FF1F9389294B130A72
:101980008006FD1436C632C42EC29790FFFFE78052
:10199000A01892452246B2466348A4000145410181
:1019A0001703FFFF670003723305440383A709028F
:1019B0003E9509C683473500C18B9DC791C68347B5
:1019C000350093F707028DC3630699008357E5003E
:1019D000639C27010357050001CB63E7E5008347BC
:1019E0008500BA97E3CDF5FA050469BF1703FFFF39
:1019F000E702036AC1642A8901449749FF1F93895A
:101A0000E942130A8006FD149790FFFFE780C0109B
:101A10006346A4001703FFFF6700C36A330544034E
:101A200083A709023E958357E500638A9700630404
:101A300099006396270197000000E780E09705046E
:101A4000E1B71703FFFFE702436389692A8AAE8A79
:101A5000328BB68B8144174CFF1F130C2C3D930C1B
:101A60008006314DFD199790FFFFE780E00A63C6BD
:101A7000A4001703FFFF67000364338994038327DF
:101A80000C028355CA015A863E994A859700000088
:101A9000E780609E31C1814D15A03384AD0383275B
:101AA000090303D60B00D68533F6C9003E94228580
:101AB00097000000E780E0B609E9850D9790FFFFE9
:101AC000E7808003E3CBADFC01A8228597000000EE
:101AD000E780E08A23040400850471B71703FFFF41
:101AE000E702235A4169AA8A014A174BFF1F130BC9
:101AF000EB337D19C14B054C9790FFFFE780C00188
:101B00006346AA001703FFFF6700235B9309800663
:101B1000B3073A0383290B02BE9983D7E900638E8A
:101B2000270163842A01639A570103A4890301E80A
:101B30004E8597000000E780C0BD050A75BF83573A
:101B40000401639977099304C400268597A0FFFFD9
:101B5000E78060D385452A8D2685835C040197A0A4
:101B6000FFFFE780C0CF268597A0FFFFE780A0E7B3
:101B700062056185635905048D45268597A0FFFFA1
:101B8000E780E0CD8945268597A0FFFFE78020CD3F
:101B90008945268597A0FFFFE78060CC854526858F
:101BA00097A0FFFFE780E0CC83470500094793F744
:101BB000F707639AE7009945268597A0FFFFE7801E
:101BC00040CBA30285014848337D2D0123189401A1
:101BD0006A9548C40040A1BF1703FFFFE702E34C2A
:101BE00037E404008327041D82979747FF1F83C7AC
:101BF000E7101725FF1F1305A58FA300F500832706
:101C0000441C82978327841C81461306F00F81456C
:101C1000014582971703FFFF6700634B1747FF1FBC
:101C20001307C7FD18439745FF1F83C5250D974729
:101C3000FF1F9387270B834687030346970363970A
:101C4000D5009747FF1F238BC70A828083C5870172
:101C50000347A7036317B6009747FF1F2380E70AD0
:101C6000828003C687016317C7009747FF1F23873A
:101C7000D708828083C68701130750026319D700F3
:101C8000930760021747FF1F230AF706828083C667
:101C90008701130660026315D60093077002DDB753
:101CA00083C7870155BF9747FF1F9387A703D44B6F
:101CB0000947638DE6081703FFFFE702033F174953
:101CC000FF1F130969FF3E8483470900918B9DCF55
:101CD000B7E4040083A7041D829783A7441C17451B
:101CE000FF1F1305E5FD829783A7841C81461746D5
:101CF000FF1F0346E6FE81450145829721C58347C4
:101D00000900ED9B1747FF1F2308F7FA83470400DC
:101D100093F7F70F85CB91471747FF1F232EF7FC4B
:101D200097000000E78080EB97000000E78040EF1D
:101D3000B7E70400BC4F414691451745FF1F0345D7
:101D4000E5FA82971703FFFF670063388280170365
:101D5000FFFFE70283358D4741116306F504C54750
:101D60006308F50285476310F5029747FF1F238933
:101D7000A7F8B7E70400BC4B930500101745FF1FF9
:101D80000345C5F6829741011703FFFF670023341F
:101D900085471747FF1F2305F7F6B7E70400BC4B3D
:101DA00093050020E1BF9747FF1F9387A7F3D44B0C
:101DB0001147638DE600B7E7040083A7071D8297EC
:101DC000B7E70400BC4B930500044DBF0549174716
:101DD000FF1F232327F383C7070032C62E8493F700
:101DE000F70FD5D3B7E4040083A7041D7D14137443
:101DF000F40F8297E37689FCB245994703C6150034
:101E0000E3F0C7FCFC4409061745FF1F130585EFE7
:101E10008297BC48930500081745FF1F034505ED51
:101E2000829779BF1703FFFFE70223281747FF1F99
:101E3000130747EB4047184B1C409746FF1F23A949
:101E4000F6EA6316E4001747FF1F2325F7EA130598
:101E500084FE9790FFFFE78000AA035564FF9780F8
:101E6000FFFFE780807297A0FFFFE78060D0170335
:101E7000FFFF6700C3251703FFFFE7020323974710
:101E8000FF1F938727E6D84BDC4789C797000000E0
:101E9000E78080F985471747FF1F232FF7E497470F
:101EA000FF1F9387A7D59C43930500021745FF1F8B
:101EB0000345C5E383C787031747FF1F2300F7E4E4
:101EC000B7E70400BC4B82971703FFFF670023208E
:101ED0009747FF1F23AAA7E082801703FFFFE702AF
:101EE000231B37E404007C4CA1451745FF1F034525
:101EF000E5DF82977C48A1451745FF1F034505DFB5
:101F00009744FF1F938404DE8297DC4489EB97009B
:101F10000000E78080D91703FFFF6700A31A03D5ED
:101F200067FF9780FFFFE7804066AA896DD1D84898
:101F300091476310F7027C4C91451745FF1F0345FD
:101F4000E5DA82977C4891451745FF1F034505DA7E
:101F5000829703A9490103D409018947B7E904001D
:101F60001747FF1F232AF7D883A7091D210442041E
:101F7000829783C784011715FF1F130565576119E1
:101F80001717FF1FA306F75683A7491C41808297A6
:101F90009747FF1F238607D683A7C91C814609469A
:101FA0009375F40F4A85829711E99747FF1F83C7FE
:101FB00067E589C79710FF1FE78060C0B7E7040097
:101FC000BC4F2146A1451745FF1F034525D28297E7
:101FD00099B71703FFFFE702430D93F7052001119F
:101FE0002E8481CF97000000E78020E9134504206C
:101FF00005611703FFFF6700830D93F70510A9CF55
:102000009744FF1F938404CEDC4897000000E780CC
:1020100020C11747FF1F130767BE184383C78401FA
:10202000034787036318F700DC4489C79700000063
:10203000E78080DF85471747FF1F232FF7CAB7E7E1
:102040000400BC4B930500021745FF1F034505CA5A
:1020500082971345041069BF93F70508BDC79747DA
:10206000FF1F83C737CAE91719469745FF1F938596
:1020700085C91305D10093F4F70F1749FF1F0349D2
:1020800069C897C00000E780404093970401C1836E
:102090001747FF1F130787C7231DF100231CF100FB
:1020A0009747FF1F938707C43ACE3ACAD8432306FF
:1020B000010009CBDC439315890154080D46E185E5
:1020C000680082971345040825B793F72500A5C338
:1020D0009747FF1F938707C1D84B89476306F702CD
:1020E0009747FF1F83C747BD13F7270011EF918B59
:1020F00099CFB7E70400BC4F1306000A894517457E
:10210000FF1F0345A5BE829713452400D5B5974709
:10211000FF1F9387A7AE9C4383C787031747FF1F03
:10212000230EF7BC97000000E78060DBF1BF93F758
:10213000050281CB97000000E78060DA13450402B6
:1021400045BD93F7850081CB97000000E780E0D282
:102150001345840071BD93F7150081CB97000000F3
:10216000E780A0B41345140061B593F7450081CB17
:1021700097000000E78060B31345440095BD93F7D6
:10218000050495C39747FF1F83C7C7B591CB970039
:102190000000E780A0A491471747FF1F232EF7B444
:1021A00013450404B1B593F705010145E38207E443
:1021B0009747FF1F938707B3D84B91476310F704E6
:1021C0009747FF1F938747AF9C4313D7270085830B
:1021D000D98F858B91E7B7E7040083A7071D829706
:1021E000B7E70400FC4F91451745FF1F034505B0B5
:1021F000829785471747FF1F2320F7B01345040137
:10220000C5BB9747FF1F238FA7BE82801703FFFF21
:10221000E702A3E99747FF1F23AC07AC9747FF1FCF
:1022200023AA07AC85471744FF1F1304249D1747B3
:10223000FF1F2323F7AC1C4083C787031747FF1FEB
:10224000230EF7AA9790FFFFE780409329C59717C1
:10225000FF1F23A3A72A1C40170500001305A5D7BD
:1022600083C787031747FF1F230AF7A81717FF1F06
:10227000A300F7289747FF1FA38607A6B7E7040028
:1022800083A7070882979747FF1F2381A7A61703F5
:10229000FFFF6700C3E3B7C7898E938767ED171702
:1022A000FF1F232BF72445BF1747FF1F034787A3B3
:1022B000795555E79747FF1F9387C7A203C71700B4
:1022C00005079746FF1FA38FE6A003C717008D469B
:1022D0003377D7029746FF1FA386E6A083C6170071
:1022E0001747FF1F13078791184393F6F60FA9EEC0
:1022F000834787031747FF1F2302F7A08547174728
:10230000FF1F2301F79E9747FF1F9387E79A9C4380
:102310000145998BA9E71703FFFFE70203D937E4CB
:1023200004007C48C1451745FF1F0345259C829743
:102330003C4885451745FF1F0345459B829701454E
:102340001703FFFF6700A3D883C71700854663956F
:10235000F6008347970379BF8347A70361BF828055
:102360009747FF1F83C70798A1CF1703FFFFE70217
:10237000C3D337E404009747FF1F238507967C48A3
:1023800085451745FF1F0345659682977C4C91450F
:102390001745FF1F0345859582977C489145174552
:1023A000FF1F0345A59482973C48C1451745FF1F71
:1023B0000345C593829701451703FFFF670023D1AB
:1023C000795582801703FFFFE70223CE2A84035545
:1023D00065FF9780FFFFE780401B9747FF1F9387AC
:1023E0006790D847BE841DEF9790FFFFE780807706
:1023F0009C48232004009DEB9747FF1F23AC878E4A
:102400009747FF1F23A6878EB7E70400BC4B89457B
:102410001745FF1F0345858D829701451703FFFF71
:102420006700E3CA630A8700184375BF80C39747F4
:10243000FF1F23A1878CC9BF7955CDB71703FFFFB5
:10244000E702A3C69747FF1F9387079C884323266D
:10245000050023240500510597A00000E780C03344
:102460001703FFFF6700A3C61703FFFFE702E3C3DD
:102470001744FF1F130444991C40411199CF9C47F6
:102480002302B5002AC61CC197000000E78040FB6C
:102490001C409C4B99C33245829741011703FFFFB3
:1024A0006700E3C21703FFFFE70223C04111444D59
:1024B000328532842EC69790FFFFE780C0522AC42F
:1024C00022859790FFFFE780205403A84400630C07
:1024D0000800B245835744001840224683D5450082
:1024E000AA862685029841011703FFFF670023BED5
:1024F0001703FFFFE70263BB404D1DC808C09705E7
:102500000000938565031305440197A00000E78050
:1025100040169747FF1F9387278F9C43014589E704
:102520009747FF1F23A2878E1703FFFF670023BA79
:102530007D55DDBF1703FFFFE70223B701116800D8
:102540009305F00F02C602C802CA02CC02CE970061
:102550000000E780A0F105611703FFFF670023B7C4
:102560009747FF1F9387478A9C43D847A1679D07DA
:102570006319F7021703FFFFE70223B30111328546
:102580009790FFFFE7802046230AA100814568005D
:1025900097000000E78080ED05611703FFFF6700EB
:1025A00003B382809747FF1F938707869C43D847D2
:1025B000A167938777036319F7021703FFFFE70209
:1025C000C3AE011132859790FFFFE780C041230A17
:1025D000A1008145680097000000E78020E90561BF
:1025E0001703FFFF6700A3AE82809747FF1F938703
:1025F000A7819C43D84795476316F7041703FFFF4D
:10260000E702A3AA0111328532849790FFFFE78089
:10261000803D230AA10022859790FFFFE780C03EFE
:1026200083574400231BA10081453ECC1C40680019
:102630003ECE97000000E78060E305611703FFFFCF
:102640006700E3A88280930785FF8DC38327C5FFBA
:1026500091CFDC4B81CF1703FFFFE70203A50325D2
:1026600085FF82971703FFFF670063A68280170329
:10267000FFFFE70283A32A8432859790FFFFE7805C
:102680008036BD4763EBA70018449377F5000345F8
:10269000B70041995D8DA305A7001703FFFF6700F1
:1026A00003A31703FFFFE70243A001117C003ECA0A
:1026B000B70707003ECC7C003ECE5C4DA9C72A84FC
:1026C00013858700AE8497A00000E780E0FCA16539
:1026D0002A899D0548089770FFFFE780603E9305B3
:1026E000803EB345B902480893F5F50F9790FFFF78
:1026F000E780C021014781465008A6852285977052
:10270000FFFFE780406105611703FFFF6700239C1F
:102710001703FFFFE702639997000000E780A0F826
:102720001703FFFF6700A39A1703FFFFE702E39772
:1027300001117C00AE843ECAA165B70707002A8458
:102740003ECC48087C00938575033ECE9770FFFF12
:10275000E78000371C44480883C5B700BD899790BF
:10276000FFFFE780A01A500801478146A685228511
:102770009770FFFFE780205A05611703FFFF67008E
:1027800003951703FFFFE70243922A84AE84970064
:102790000000E78000EEA685228597000000E78014
:1027A000E0F81703FFFF670083921703FFFFE702BC
:1027B000C38F97000000E78060F71703FFFF6700F3
:1027C00003911703FFFFE702438E0329C50141115F
:1027D000630809022A843285B2849790FFFFE7805C
:1027E00080202AC626859790FFFFE780E021832777
:1027F00049002A8691C7DC4781C7B2452285829766
:1028000041011703FFFF6700838C1703FFFFE702F7
:10281000C389444D91CC2A8432859790FFFFE7808D
:10282000A01EDC40AA8589C79C4799C32285829750
:102830001703FFFF6700A3891703FFFFE702438524
:10284000032AC5014111630D0A062E89AA84954504
:10285000328532849770FFFFE78080268545228588
:102860009790FFFFE7804004AA89CA852285979048
:10287000FFFFE780A00B83274A008DCBDC439DC779
:1028800022859790FFFFE780A00083274A00104031
:1028900083564400DC437115A307A100B2961307C9
:1028A000F1004E86CA852685829701C523800900DE
:1028B00001A88345F10022859790FFFFE780C0FEC5
:1028C000410117F3FEFF6700E37F17F3FEFFE70206
:1028D000C37D65711C083EC2B70780013EC41C0859
:1028E00032893EC62A84AE8497000000E780A0EDBE
:1028F0004A859790FFFFE78020118357A1008DC381
:10290000AA855000228597000000E78020F3014748
:1029100081465000A68522859770FFFFE780A03F83
:10292000596117F3FEFF6700837A17F3FEFFE70292
:10293000237665711C088329C5013EC2B707800153
:102940003EC41C082A84AE8432893EC6970000002B
:10295000E780E0EB638A09024A859790FFFFE780F2
:10296000A00A8357A100AA8585C35000228597003D
:102970000000E780A0EC014781465000A685228533
:102980009770FFFFE7802039596117F3FEFF67005A
:10299000637317F3FEFFE702437165711C083EC2C3
:1029A000B70780013EC42A841C0832853EC6AE8427
:1029B0009790FFFFE78040058357A1008DC3AA854C
:1029C0005000228597000000E78040E701478146DC
:1029D0005000A68522859770FFFFE780C0335961BC
:1029E00017F3FEFF6700A36E17F3FEFFE702E36B2A
:1029F000444D81EC8347450093B71700B307F0407F
:102A00003E8517F3FEFF6700836C1845FD576DDBAD
:102A100097070000938747032A845CCB9705000043
:102A20009385A5C21385840097A00000E78060C449
:102A300080C003474400814761F71737FF1F2327F2
:102A4000973C7DBF17F3FEFFE70283648329C5012E
:102A500041110329850081476387090A032409017D
:102A600091452A8A22859770FFFFE780600585459A
:102A700022859790FFFFE78020E38945AA8A228577
:102A80009790FFFFE78040E2AA849770FFFFE780FE
:102A9000400A83A749002A8B8DCB9C439DC7228582
:102AA0009790FFFFE780C0DE83A74900A306A1003F
:102AB0001040835644009C431307D100B296D6853C
:102AC0001306E1005285829709CD83570B002380BE
:102AD000F400A183A380F40023800A00A306010070
:102AE00039A88357E10022852380F4008345D10073
:102AF000A183A380F4009790FFFFE780E0DA83478B
:102B0000D100B337F0000347B900920701453D9B60
:102B1000D98FA305F900410117F3FEFF6700835A1F
:102B200017F3FEFFE702635841110DED9737FF1FC2
:102B30009387C72D804315C80440130984009DC99D
:102B40005C4099C79C4B89C726852EC68297B245A3
:102B50009307803EB385F5024A8597A00000E78081
:102B600060C121A0404DAA8469F8410117F3FEFF1E
:102B70006700E3554A8597A00000E780E0C15C400C
:102B8000EDD7DC4BFDD326858297C5B717F3FEFF43
:102B9000E702A3512A8432859790FFFFE780A0E4E3
:102BA000AA85228597000000E780C0F717F3FEFF93
:102BB0006700E35117F3FEFFE702234F2A84AE8438
:102BC00097000000E780C0FCA685228597000000E2
:102BD000E78060AD17F3FEFF6700634F0841335590
:102BE000B5000589828017F3FEFFE702034C173416
:102BF000FF1F1304A4231C5C0111231701008D8304
